S01800004343534D6F64756C65535733305765622E73726563A2
S31508008000000001207DD8000849CF000851CF00089C
S3150800801059CF000861CF000869CF000800000000AA
S3150800802000000000000000000000000071CF0008FA
S315080080307DCF00080000000089CF000895CF000812
S31508008040C5D80008C5D80008C5D80008C5D800088E
S31508008050C5D80008C5D80008C5D80008C5D800087E
S31508008060C5D80008C5D80008C5D80008C5D800086E
S31508008070C5D80008C5D80008C5D80008C5D800085E
S31508008080C5D80008C5D80008C5D80008C5D800084E
S31508008090A1CF0008C5D80008C5D80008C5D800086B
S315080080A0C5D80008C5D80008C5D80008C5D800082E
S315080080B0C5D80008B5CF0008C5D80008C5D8000837
S315080080C0C5D80008C5D80008C5D80008C5D800080E
S315080080D0C5D80008C9CF0008DDCF0008F1CF0008D1
S315080080E0C5D80008C5D80008C5D800080000000093
S315080080F00000000000000000000000000000000072
S315080081000000000000000000C5D80008C5D8000817
S31508008110C5D8000805D00008C5D80008C5D8000885
S31508008120C5D80008C5D80008C5D80008C5D80008AD
S31508008130C5D80008C5D80008C5D8000819D0000851
S31508008140C5D800082DD00008C5D80008C5D800082D
S315080081500000000000000000000000000000000011
S315080081600000000000000000000000000000000001
S3150800817000000000000000000000000000000000F1
S3150800818000000000000000000000000000000000E1
S3150800819000000000000000000000000000000000D1
S315080081A000000000000000000000000000000000C1
S315080081B000000000000000000000000000000000B1
S315080081C000000000000000000000000000000000A1
S315080081D00000000000000000000000000000000091
S309080081E05FF8E0F165
S315080081E810B5054C237833B9044B13B10448AFF3DB
S315080081F800800123237010BDD8000020000000006D
S315080082080840010808B5034B1BB103490348AFF3F7
S31508008218008008BD00000000DC00002008400108B6
S3150800822881F0004102E000BF83F0004330B54FEA11
S3150800823841044FEA430594EA050F08BF90EA020F7E
S315080082481FBF54EA000C55EA020C7FEA645C7FEA11
S31508008258655C00F0E2804FEA5454D4EB5555B8BF34
S315080082686D420CDD2C4480EA020281EA030382EAA5
S31508008278000083EA010180EA020281EA0303362D37
S3150800828888BF30BD11F0004F4FEA01314FF4801C0A
S315080082984CEA113102D0404261EB410113F0004F1C
S315080082A84FEA03334CEA133302D0524263EB4303D3
S315080082B894EA050F00F0A780A4F10104D5F1200E71
S315080082C80DDB02FA0EFC22FA05F2801841F10001CC
S315080082D803FA0EF2801843FA05F359410EE0A5F1A0
S315080082E820050EF1200E012A03FA0EFC28BF4CF0D1
S315080082F8020C43FA05F3C01851EBE37101F0004587
S3150800830807D54FF0000EDCF1000C7EEB00006EEB93
S315080083180101B1F5801F1BD3B1F5001F0CD349081D
S315080083285FEA30004FEA3C0C04F101044FEA445274
S3150800833812F5800F80F09A80BCF1004F08BF5FEAFB
S31508008348500C50F1000041EB045141EA050130BDDB
S315080083585FEA4C0C404141EB0101013C28BFB1F5ED
S31508008368801FE9D291F0000F04BF01460020B1FA38
S3150800837881F308BF2033A3F10B03B3F120020CDA0B
S315080083880C3208DD02F1140CC2F10C0201FA0CF0E9
S3150800839821FA02F10CE002F11402D8BFC2F1200C4E
S315080083A801FA02F120FA0CFCDCBF41EA0C01904004
S315080083B8E41AA2BF01EB0451294330BD6FEA04044D
S315080083C81F3C1CDA0C340EDC04F11404C4F1200238
S315080083D820FA04F001FA02F340EA030021FA04F34A
S315080083E845EA030130BDC4F10C04C4F1200220FAA1
S315080083F802F001FA04F340EA0300294630BD21FADF
S3150800840804F0294630BD94F0000F83F4801306BFA4
S3150800841881F480110134013D4EE77FEA645C18BF98
S315080084287FEA655C29D094EA050F08BF90EA020F2F
S3150800843805D054EA000C04BF1946104630BD91EA27
S31508008448030F1EBF0021002030BD5FEA545C05D12A
S315080084584000494128BF41F0004130BD14F5800469
S315080084683CBF01F5801130BD01F0004545F0FE41DD
S3150800847841F470014FF0000030BD7FEA645C1ABF12
S31508008488194610467FEA655C1CBF0B46024650EA49
S31508008498013406BF52EA033591EA030F41F4002175
S315080084A830BD00BF90F0000F04BF0021704730B5FB
S315080084B84FF4806404F132044FF000054FF00001D0
S315080084C850E700BF90F0000F04BF0021704730B591
S315080084D84FF4806404F1320410F0004548BF404266
S315080084E84FF000013EE700BF42004FEAE2014FEABB
S315080084F831014FEA02701FBF12F07F4393F07F4F96
S3150800850881F06051704732F07F4208BF704793F098
S315080085187F4F04BF41F40021704730B54FF46074AB
S3150800852801F0004521F000411CE700BF50EA0102AE
S3150800853808BF704730B54FF000050AE050EA010257
S3150800854808BF704730B511F0004502D5404261EBC7
S3150800855841014FF4806404F132045FEA915C3FF408
S31508008568D8AE4FF003025FEADC0C18BF03325FEAA5
S31508008578DC0C18BF033202EBDC02C2F1200300FA56
S3150800858803FC20FA02F001FA03FE40EA0E0021FA7B
S3150800859802F11444BDE600BF70B54FF0FF0C4CF469
S315080085A8E06C1CEA11541DBF1CEA135594EA0C0F1B
S315080085B895EA0C0F00F0DEF82C4481EA030621EA56
S315080085C84C5123EA4C5350EA013518BF52EA033591
S315080085D841F4801143F4801338D0A0FB02CE4FF043
S315080085E80005E1FB02E506F00042E0FB03E54FF073
S315080085F80006E1FB03569CF0000F18BF4EF0010E6B
S31508008608A4F1FF04B6F5007F64F5407404D25FEA66
S315080086184E0E6D4146EB060642EAC62141EA555119
S315080086284FEAC52040EA5E504FEACE2EB4F1FD0C5B
S3150800863888BFBCF5E06F1ED8BEF1004F08BF5FEAD9
S31508008648500E50F1000041EB045170BD06F000468B
S3150800865846EA010140EA020081EA0301B4EB5C0438
S31508008668C2BFD4EB0C0541EA045170BD41F4801130
S315080086784FF0000E013C00F3AB8014F1360FDEBF55
S31508008688002001F0004170BDC4F10004203C35DA31
S315080086980C341BDC04F11404C4F1200500FA05F3B4
S315080086A820FA04F001FA05F240EA020001F0004255
S315080086B821F0004110EBD37021FA04F642EB0601CB
S315080086C85EEA430E08BF20EAD37070BDC4F10C04F5
S315080086D8C4F1200500FA04F320FA05F001FA04F2B9
S315080086E840EA020001F0004110EBD37041F10001A5
S315080086F85EEA430E08BF20EAD37070BDC4F12005B0
S3150800870800FA05F24EEA020E20FA04F301FA05F217
S3150800871843EA020321FA04F001F0004121FA04F2BF
S3150800872820EA020000EBD3705EEA430E08BF20EA8F
S31508008738D37070BD94F0000F0FD101F000464000C9
S3150800874841EB010111F4801F08BF013CF7D041EA4B
S31508008758060195F0000F18BF704703F0004652004F
S3150800876843EB030313F4801F08BF013DF7D043EA20
S315080087780603704794EA0C0F0CEA135518BF95EAD6
S315080087880C0F0CD050EA410618BF52EA4306D1D15D
S3150800879881EA030101F000414FF0000070BD50EA7C
S315080087A8410606BF1046194652EA430619D094EA06
S315080087B80C0F02D150EA013613D195EA0C0F05D1F0
S315080087C852EA03361CBF104619460AD181EA030144
S315080087D801F0004141F0FE4141F470014FF00000FC
S315080087E870BD41F0FE4141F4780170BD70B54FF097
S315080087F8FF0C4CF4E06C1CEA11541DBF1CEA135517
S3150800880894EA0C0F95EA0C0F00F0A7F8A4EB0504F8
S3150800881881EA030E52EA03354FEA013100F08880EF
S315080088284FEA03334FF0805545EA131343EA1263B8
S315080088384FEA022245EA111545EA10654FEA00266D
S315080088480EF000419D4208BF964244F1FD0404F526
S31508008858407402D25B084FEA3202B61A65EB030582
S315080088685B084FEA32024FF480104FF4002CB6EB3F
S31508008878020E75EB030E22BFB61A754640EA0C00BF
S315080088885B084FEA3202B6EB020E75EB030E22BFFF
S31508008898B61A754640EA5C005B084FEA3202B6EB40
S315080088A8020E75EB030E22BFB61A754640EA9C00FF
S315080088B85B084FEA3202B6EB020E75EB030E22BFCF
S315080088C8B61A754640EADC0055EA060E18D04FEA8D
S315080088D8051545EA16754FEA06164FEAC30343EA2D
S315080088E852734FEAC2025FEA1C1CC0D111F4801FFA
S315080088F80BD141EA00014FF000004FF0004CB6E7F3
S3150800890811F4801F04BF01430020B4F1FD0C88BF91
S31508008918BCF5E06F3FF6AFAEB5EB030C04BFB6EB9C
S31508008928020C5FEA500C50F1000041EB045170BD8F
S315080089380EF0004E4EEA113114EB5C04C2BFD4EBBC
S315080089480C0541EA045170BD41F480114FF0000E40
S31508008958013C90E645EA060E8DE60CEA135594EABC
S315080089680C0F08BF95EA0C0F3FF43BAF94EA0C0FBF
S315080089780AD150EA01347FF434AF95EA0C0F7FF434
S3150800898825AF104619462CE795EA0C0F06D152EA88
S3150800899803353FF4FDAE1046194622E750EA41066C
S315080089A818BF52EA43067FF4C5AE50EA41047FF47D
S315080089B80DAF52EA43057FF4EBAE12E74FEA4102E0
S315080089C8B2F1E04324BFB3F5001CDCF1FE5C0DD917
S315080089D801F0004C4FEAC0024CEA5070B2F1004F61
S315080089E840EB830008BF20F00100704711F0804F64
S315080089F821D113F13872BCBF01F00040704741F429
S31508008A0880114FEA5252C2F11802C2F1200C10FA2C
S31508008A180CF320FA02F018BF40F001004FEAC12310
S31508008A284FEAD32303FA0CFC40EA0C0023FA02F3B4
S31508008A384FEA4303CCE77FEA625307D150EA01338A
S31508008A481EBF4FF0FE4040F44000704701F000405A
S31508008A5840F0FE4040F40000704700BF80F0004038
S31508008A6802E000BF81F0004142001FBF5FEA4103F0
S31508008A7892EA030F7FEA226C7FEA236C6AD04FEAF0
S31508008A881262D2EB1363C1BFD21841404840414035
S31508008A98B8BF5B42192B88BF704710F0004F40F4E7
S31508008AA8000020F07F4018BF404211F0004F41F403
S31508008AB8000121F07F4118BF494292EA030F3FD0CF
S31508008AC8A2F1010241FA03FC10EB0C00C3F12003E2
S31508008AD801FA03F100F0004302D5494260EB400071
S31508008AE8B0F5000F13D3B0F1807F06D340084FEADC
S31508008AF8310102F10102FE2A51D2B1F1004F40EBD1
S31508008B08C25008BF20F0010040EA03007047490038
S31508008B1840EB0000013A28BFB0F5000FEDD2B0FAD5
S31508008B2880FCACF1080CB2EB0C0200FA0CF0AABFF8
S31508008B3800EBC25052421843BCBFD0401843704796
S31508008B4892F0000F81F4000106BF80F4000001329C
S31508008B58013BB5E74FEA41037FEA226C18BF7FEA73
S31508008B68236C21D092EA030F04D092F0000F08BFB5
S31508008B780846704790EA010F1CBF0020704712F09C
S31508008B887F4F04D1400028BF40F00040704712F1DB
S31508008B9800723CBF00F50000704700F0004343F040
S31508008BA8FE4040F4000070477FEA226216BF084676
S31508008BB87FEA23630146420206BF5FEA412390EA39
S31508008BC8010F40F4800070474FF0000304E000BF2F
S31508008BD810F0004348BF40425FEA000C08BF7047E0
S31508008BE843F0964301464FF000001CE050EA0102A4
S31508008BF808BF70474FF000030AE000BF50EA0102B9
S31508008C0808BF704711F0004302D5404261EB4101A5
S31508008C185FEA010C02BF84460146002043F0B643CA
S31508008C2808BFA3F18053A3F50003BCFA8CF2083AEF
S31508008C38A3EBC25310DB01FA02FC634400FA02FCF8
S31508008C48C2F12002BCF1004F20FA02F243EB0200FF
S31508008C5808BF20F00100704702F1200201FA02FC61
S31508008C68C2F1200250EA4C0021FA02F243EB020054
S31508008C7808BF20EADC7070474FF0FF0C1CEAD05298
S31508008C881EBF1CEAD15392EA0C0F93EA0C0F6FD059
S31508008C981A4480EA010C400218BF5FEA41211ED037
S31508008CA84FF0006343EA501043EA5111A0FB013123
S31508008CB80CF00040B1F5000F3EBF490041EAD371F8
S31508008CC85B0040EA010062F17F02FD2A1DD8B3F174
S31508008CD8004F40EBC25008BF20F00100704790F0E3
S31508008CE8000F0CF0004C08BF49024CEA502040EA35
S31508008CF851207F3AC2BFD2F1FF0340EAC2507047FB
S31508008D0840F400004FF00003013A5DDC12F1190F38
S31508008D18DCBF00F000407047C2F10002410021FAAA
S31508008D2802F1C2F1200200FA02FC5FEA310040F1C2
S31508008D38000053EA4C0308BF20EADC70704792F03B
S31508008D48000F00F0004C02BF400010F4000F013A73
S31508008D58F9D040EA0C0093F0000F01F0004C02BF6E
S31508008D68490011F4000F013BF9D041EA0C018FE7DD
S31508008D780CEAD15392EA0C0F18BF93EA0C0F0AD0E3
S31508008D8830F0004C18BF31F0004CD8D180EA010009
S31508008D9800F00040704790F0000F17BF90F0004FA2
S31508008DA8084691F0000F91F0004F14D092EA0C0F84
S31508008DB801D142020FD193EA0C0F03D14B0218BF17
S31508008DC8084608D180EA010000F0004040F0FE405D
S31508008DD840F40000704740F0FE4040F440007047F9
S31508008DE84FF0FF0C1CEAD0521EBF1CEAD15392EA78
S31508008DF80C0F93EA0C0F69D0A2EB030280EA010C68
S31508008E0849024FEA402037D04FF0805343EA111100
S31508008E1843EA10130CF000408B4238BF5B0042F15E
S31508008E287D024FF4000C8B4224BF5B1A40EA0C0003
S31508008E38B3EB510F24BFA3EB510340EA5C00B3EB35
S31508008E48910F24BFA3EB910340EA9C00B3EBD10F23
S31508008E5824BFA3EBD10340EADC001B0118BF5FEA75
S31508008E681C1CE0D1FD2A3FF650AF8B4240EBC2509E
S31508008E7808BF20F0010070470CF0004C4CEA50205F
S31508008E887F32C2BFD2F1FF0340EAC250704740F4AE
S31508008E9800004FF00003013A37E792F0000F00F0A0
S31508008EA8004C02BF400010F4000F013AF9D040EA1E
S31508008EB80C0093F0000F01F0004C02BF490011F4B2
S31508008EC8000F013BF9D041EA0C0195E70CEAD153AA
S31508008ED892EA0C0F08D142027FF47DAF93EA0C0F91
S31508008EE87FF470AF084676E793EA0C0F04D14B0275
S31508008EF83FF44CAF08466EE730F0004C18BF31F027
S31508008F08004CCAD130F000427FF45CAF31F0004320
S31508008F187FF43CAF5FE700BF4FF0FF3C06E000BFB9
S31508008F284FF0010C02E000BF4FF0010C4DF804CDDC
S31508008F384FEA40024FEA41037FEA226C18BF7FEAEC
S31508008F48236C11D001B052EA530C18BF90EA010FEE
S31508008F5858BFB2EB030088BFC81738BF6FEAE1707D
S31508008F6818BF40F0010070477FEA226C02D15FEA19
S31508008F78402C05D17FEA236CE4D15FEA412CE1D085
S31508008F885DF8040B704700BF844608466146FFE74C
S31508008F980FB5FFF7C9FF002848BF10F1000F0FBD2E
S31508008FA84DF808EDFFF7F4FF0CBF012000205DF827
S31508008FB808FB00BF4DF808EDFFF7EAFF34BF0120AC
S31508008FC800205DF808FB00BF4DF808EDFFF7E0FF45
S31508008FD894BF012000205DF808FB00BF4DF808ED96
S31508008FE8FFF7D2FF94BF012000205DF808FB00BFF9
S31508008FF84DF808EDFFF7C8FF34BF012000205DF8DB
S3150800900808FB00BF4FEA4002B2F1FE4F0FD34FF0FC
S315080090189E03B3EB12620DD94FEA002343F00043CF
S3150800902810F0004F23FA02F018BF404270474FF07D
S315080090380000704712F1610F01D1420205D110F004
S31508009048004008BF6FF0004070474FF000007047B7
S3150800905853B94AB9002908BF00281CBF4FF0FF3189
S315080090684FF0FF3000F08CB9ADF1080C6DE904CE6D
S3150800907800F006F8DDF804E0DDE9022304B07047DD
S315080090882DE9F047089D8E4604468846002B4AD1A6
S315080090988A42174662D9B2FA82F64EB1C6F1200359
S315080090A801FA06F820FA03F3B74043EA0808B44079
S315080090B84FEA174EB8FBFEF11FFA87FC0EFB11881C
S315080090C801FB0CF2230C43EA08439A4209D9FB1818
S315080090D801F1FF3080F0EB809A4240F2E8800239CD
S315080090E83B449A1AB2FBFEF00EFB102200FB0CFC5E
S315080090F8A3B243EA02439C4509D9FB1800F1FF329B
S3150800910880F0D7809C4540F2D4803B44023840EA38
S3150800911801400021A3EB0C031DB10022F340C5E969
S315080091280032BDE8F0878B4205D90DB1C5E90001C3
S3150800913800210846F5E7B3FA83F1002946D17345B5
S3150800914802D3824200F20881841A6EEB03020120D8
S315080091589046002DE5D0C5E90048E2E7002A00F068
S315080091689180B2FA82F6002E40F0A5808A1A01216B
S31508009178030C4FEA174E80B2BCB2B2FBFEFC0EFBDC
S315080091881C2243EA024304FB0CF29A4207D9FB184D
S315080091980CF1FF3802D29A4200F2E380C4469B1AC1
S315080091A8B3FBFEF20EFB123302FB04F440EA034358
S315080091B89C4207D9FB1802F1FF3002D29C4200F202
S315080091C8CD8002461B1B42EA0C40A5E7C1F12006E2
S315080091D88B4022FA06F71F432EFA06FA4FEA174972
S315080091E8BAFBF9F80EFA01FE20FA06F309FB18AAE3
S315080091F81FFA87FC43EA0E0300FA01FE08FB0CF087
S315080092081C0C44EA0A44A04202FA01F20AD93C199B
S3150800921808F1FF3A80F09E80A04240F29B80A8F1B0
S3150800922802083C44241A98B2B4FBF9F309FB134420
S3150800923803FB0CFC40EA0444A44509D93C1903F18C
S31508009248FF3080F08580A44540F28280023B3C448A
S3150800925843EA0840A4EB0C04A0FB028C6445434689
S31508009268E14664D361D05DB1BEEB030264EB090441
S3150800927804FA06F622FA01F31E43CC40C5E900644F
S3150800928800214EE7B1FBF2FC010C41EA0E4180B21F
S3150800929840EA01423B46B1FBF7F138463C46B84638
S315080092A8BE462026A2EB080241EA0C4165E70146BC
S315080092B817E710462BE7C6F120012EFA01FCB7403E
S315080092C80EFA06FE20FA01F141EA0E014FEA174E98
S315080092D8BCFBFEF8BCB20EFB18CC08FB04F90A0C5A
S315080092E842EA0C42B04091454FEA104380B23ED953
S315080092F8BA1808F1FF3C01D291451FD8A2EB09021A
S31508009308B2FBFEF909FB04F80EFB192A8AB242EAEF
S315080093180A42424529D2BA1809F1FF31C2D2424552
S31508009328C0D2A9F102013A44BCE7C6459BD2B8EBBC
S3150800933802036CEB070C0138E14694E7A7EB090929
S315080093484A44B2FBFEF9A8F1020C09FB04F8DBE76C
S3150800935803467DE7D04665E70846FAE63B44023AFF
S3150800936830E7ACF1020C3B4419E749469AE7A2EB09
S315080093780902B2FBFEF9C44609FB04F8C4E700BFB4
S31508009388704700BF80B584B000AF3B1D00221A6045
S315080093985A609A60184B194A1A60174B00229A6045
S315080093A8154B00221A73144B00221A75124B4FF4E8
S315080093B86022DA61104B00225A600F4B01221A61AB
S315080093C80D4804F003FB0346002B01D001F012FBFD
S315080093D808237B600123BB600023FB603B1D1946FD
S315080093E8054804F0B7FD0346002B01D001F002FB3F
S315080093F800BF1037BD4680BDF40000200024014098
S3150800940880B58AB000AF786007F1180300221A60A1
S315080094185A609A60DA607B681B681F4A934237D19C
S315080094281E4B9B691D4A43F4007393611B4B9B694A
S3150800943803F400737B617B69184B9B69174A43F0F1
S3150800944804039361154B9B6903F004033B613B696D
S31508009458124B9B69114A43F0080393610F4B9B69AA
S3150800946803F00803FB60FB681823BB610323FB6151
S3150800947807F1180319460A4806F0F0F80323BB61F2
S315080094880323FB6107F118031946064806F0E6F8B0
S3150800949800BF2837BD4680BD0024014000100240A1
S315080094A800080140000C014080B582B000AF0346B1
S315080094B80A46FB711346BB71FB79072B50D801A2E4
S315080094C852F823F0ED940008FD9400080D9500085D
S315080094D81D9500082D9500083D9500084B95000830
S315080094E85B950008BB791A464FF48071214806F047
S315080094F850FA36E0BB791A464FF400711D4806F053
S3150800950848FA2EE0BB791A464FF48061194806F0E6
S3150800951840FA26E0BB791A464FF40061154806F06A
S3150800952838FA1EE0BB791A464FF48051114806F0FE
S3150800953830FA16E0BB791A4608210F4806F029FAC8
S315080095480FE0BB791A464FF400410C4806F021FA99
S3150800955807E0BB791A460821094806F01AFA00E016
S3150800956800BFFB790749BA79CA5400BF0837BD4610
S3150800957880BD00BF001801400010014000080140E6
S31508009588001401402401002080B483B000AF0346CC
S31508009598FB71FB79034AD35C18460C37BD4680BC79
S315080095A8704700BF2401002080B582B000AF03468B
S315080095B8FB71FB79062B3BD801A252F823F000BFB2
S315080095C8E5950008F1950008FD9500080996000834
S315080095D815960008219600082D96000802211748B6
S315080095E806F0C0F9034624E00421144806F0BAF93F
S315080095F803461EE08021124806F0B4F9034618E02F
S315080096088021104806F0AEF9034612E010210E48EC
S3150800961806F0A8F903460CE008210B4806F0A2F95B
S31508009628034606E00221064806F09CF9034600E0D0
S31508009638002318460837BD4680BD00BF000801400C
S315080096480018014000140140000C014080B500AF25
S31508009658154804F013FE00210020FFF725FF002116
S315080096680120FFF721FF00210220FFF71DFF002137
S315080096780320FFF719FF00210420FFF715FF012132
S315080096880520FFF711FF01210620FFF70DFF00212E
S315080096980720FFF709FF054803F094FB044803F081
S315080096A891FB00BF80BD00BFF400002030010020F8
S315080096B85801002090B587B000AF78600C4B7B61E5
S315080096C80C4B3B6179697868FFF7CCF903461C4669
S315080096D839697869FFF7D0FA034619462046FFF72D
S315080096E87FFB0346FB60FB6818461C37BD4690BDE2
S315080096F800007A443211803BB0B586B000AFF860F6
S31508009708B9607A603B60F868FEF7DCFE1CA3D3E90B
S315080097180023FFF76BF802460B4614461D46B86841
S31508009728FEF7E2FE02460B4620462946FEF734FFB8
S3150800973802460B4610461946FFF740F903467B6171
S3150800974879687869FFF74AFC0346002B01D00E4B67
S3150800975810E079697868FFF785F903461946786944
S31508009768FFF73EFB034619463868FFF785FA0346AE
S315080097783B613B6918461837BD46B0BDAFF3008054
S315080097880000000000FEAF40000080BF80B588B02A
S3150800979800AF0346FB7100F09BF8FB79002B03D05A
S315080097A8082000F053F802E0092000F04FF8224894
S315080097B804F0E4F94FF0FF311F4804F0B9FA1E48DF
S315080097C804F0BCFBF8611C4804F086FAFB79002B08
S315080097D801D0012200E0002213469B001344DB0057
S315080097E8164A1344FA691146184603F010FBB8617D
S315080097F8BB69B3F57A6F03D900F076F8142317E036
S315080098080F4B7B610F4B3B610F4BFB60FB683A695B
S315080098187969B869FFF770FF03461846FFF74AFFE4
S31508009828B86000F061F8B868FFF7ECFB03461BB2AE
S3150800983818462037BD4680BDF400002030010020B8
S31508009848333353400000A04000007A4480B586B000
S3150800985800AF78607B68FB6001233B6103237B616B
S3150800986807F10C031946064804F074FB0346002B57
S3150800987801D001F0BFF800BF1837BD4680BD00BF4C
S31508009888F400002080B483B000AFEFF310833B6088
S315080098983B687B6072B600BF0C4B1B78DBB2002BAB
S315080098A806D07B68002B01D162B600BF002308E00A
S315080098B8064B01221A707B68002B01D162B600BFDD
S315080098C8012318460C37BD4680BC70472C0100207A
S315080098D880B500AF00BFFFF7D5FF0346002BFAD0C7
S315080098E800BF00BF80BD000080B483B000AFEFF3AF
S315080098F810833B603B687B6072B600BF064B00224C
S315080099081A707B68002B01D162B600BF00BF0C37FE
S31508009918BD4680BC704700BF2C01002080B500AF4B
S31508009928174B184A1A60164B08225A60144B00221D
S315080099389A60134B0022DA60114B4FF460221A61C1
S315080099480F4B4FF480125A610D4B00221A760C4BB6
S3150800995801225A760A4B01229A76094B0122DA76AF
S31508009968074B00221A77064B01225A77044804F057
S3150800997833FD0346002B01D001F03CF800BF80BD3B
S31508009988800100200064004080B500AF174B184AD4
S315080099981A60164B10225A60144B00229A60134B11
S315080099A80022DA60114B4FF460221A610F4B4FF40C
S315080099B880125A610D4B00221A760C4B01225A76F0
S315080099C80A4B01229A76094B0122DA76074B0022BE
S315080099D81A77064B01225A77044804F0FDFC034619
S315080099E8002B01D001F006F800BF80BDA8010020B1
S315080099F80068004080B58EB000AF786007F1200394
S31508009A0800221A605A609A60DA607B681B68614AA5
S31508009A18934253D1604B1B6801335F4A13605E4B10
S31508009A281B68012B0BD15D4BDB695C4A43F000735D
S31508009A38D3615A4BDB6903F00073FB61FB69574B2B
S31508009A489B69564A43F020039361544B9B6903F07C
S31508009A582003BB61BB6901233B6200237B620023A9
S31508009A68BB6207F1200319464D4805F0F7FD0223A6
S31508009A783B6202237B620323FB6207F12003194634
S31508009A88474805F0EBFD474B5B683B633B6B23F4A4
S31508009A98C0433B633B6B43F0E0633B633B6B43F478
S31508009AA8C0433B633F4A3B6B5360002200211420A6
S31508009AB805F03FFC142005F058FC67E07B681B6836
S31508009AC8394A934262D1354BDB69344A43F080639D
S31508009AD8D361324BDB6903F080637B617B692E4B6C
S31508009AE81B6801332C4A13602B4B1B68012B0BD1BF
S31508009AF82A4BDB69294A43F00073D361274BDB6994
S31508009B0803F000733B613B69244B9B69234A43F086
S31508009B1808039361214B9B6903F00803FB60FB6804
S31508009B2820233B6200237B620023BB6207F12003E4
S31508009B3819461E4805F092FD40233B6202237B62C4
S31508009B480323FB6207F120031946184805F086FD2A
S31508009B58144B5B687B637B6B43F0E0637B637B6BCF
S31508009B6843F480037B630F4A7B6B53600022002112
S31508009B783F2005F0DEFB3F2005F0F7FB0022002119
S31508009B88412005F0D6FB412005F0EFFB00BF38372A
S31508009B98BD4680BD00640040D00100200010024088
S31508009BA8001401400000014000680040000C014014
S31508009BB880B400AF084B00221A70074B00225A706F
S31508009BC8054B002262F06902DA7300221A7400BF94
S31508009BD8BD4680BC704700BFD401002080B500AFE1
S31508009BE81A4B5A781A4B1B789A4206D0174B5A784A
S31508009BF8174B1A70154B00221A70164B1B7B002B35
S31508009C0803D0124B07225A770EE0124B5B7B002BC8
S31508009C1803D00E4B0A225A7706E00C4B9B7F002B83
S31508009C2802D10A4B00225A77084B5B7F0021184657
S31508009C3800F078FD0346002B06D0044B5B7F1A46D6
S31508009C480021054809F074F900BF80BDD401002039
S31508009C58F4010020240700202040010880B500AF41
S31508009C680F4B5B7F002B03D0022000F01FF816E08D
S31508009C780C4B1B78002B07D10B4B1B78002B03D0FA
S31508009C88012000F013F80AE0064B1B78022B06D1D0
S31508009C98034B5B7F002B02D1012000F007F880BD3B
S31508009CA8D4010020F3010020C20E002080B582B03E
S31508009CB800AF0346FB71414B1B78FA799A4203D1E8
S31508009CC83F4AFB79537075E03C4AFB7913703B4B66
S31508009CD81B78002B03D13B49072000F0CBFB374BF9
S31508009CE81B78012B03D13849072000F0C3FB334BF7
S31508009CF81B78022B03D13549072000F0BBFB2F4BF5
S31508009D081B78032B03D13249072000F0B3FB2B4BF2
S31508009D181B78042B03D12F49072000F0ABFB274BF0
S31508009D281B78052B03D12C49072000F0A3FB234BEE
S31508009D381B78062B03D12949072000F09BFB1F4BEC
S31508009D481B78072B03D12649072000F093FB1B4BEA
S31508009D581B78082B03D12349072000F08BFB174BE8
S31508009D681B78092B03D12049072000F083FB134BE6
S31508009D781B780A2B03D11D49072000F07BFB0F4BE4
S31508009D881B780B2B03D11A49072000F073FB0B4BE2
S31508009D981B780C2B03D11749072000F06BFB074BE0
S31508009DA81B780D2B03D11449072000F063FB044ADE
S31508009DB8FB7953700837BD4680BD00BFF301002004
S31508009DC8D4010020344001084840010860400108D1
S31508009DD87840010890400108AC400108CC400108C9
S31508009DE8EC4001080C410108244101083C410108DE
S31508009DF854410108704101088841010880B584B0BA
S31508009E0800AF78600023FB607868FFF71FFD0948F4
S31508009E1803F0B4FE0A21074803F08AFF054804F050
S31508009E288DF8F860034803F057FFFB6818461037A3
S31508009E38BD4680BDF400002080B485B000AFF86048
S31508009E48B9607A60FA68BB689A4205DBFA687B6883
S31508009E589A4201DC012300E0002318461437BD4660
S31508009E6880BC704780B483B000AF7860124B1B780B
S31508009E78002B08D1114A7B6813600F4B01221A7010
S31508009E880E4B1B6812E00D4B1B687A68D31A2622FC
S31508009E9802FB03F3002B00DAFF331B121A46074BA3
S31508009EA81B681344054A1360044B1B6818460C378D
S31508009EB8BD4680BC704700BF00020020FC01002098
S31508009EC880B582B000AF78600B46FB70FB78052B2F
S31508009ED84AD801A252F823F0F99E0008079F0008FD
S31508009EE81F9F0008379F00084F9F0008659F0008B6
S31508009EF87B6842F20F72934238DD00237EE042F611
S31508009F08041241F64C517868FFF796FF0346002B72
S31508009F182ED0012372E041F64C5241F2941178682A
S31508009F28FFF78AFF0346002B24D0022366E041F296
S31508009F38941240F2DC517868FFF77EFF0346002B3F
S31508009F481AD003235AE040F6C4122E497868FFF758
S31508009F5873FF0346002B11D004234FE07B682A4A77
S31508009F6893420DDA052349E000BF0AE000BF08E07E
S31508009F7800BF06E000BF04E000BF02E000BF00E043
S31508009F8800BF7B6842F6F722934201DD002335E0DD
S31508009F9842F210724FF4FA517868FFF74DFF0346FC
S31508009FA8002B01D0012329E041F6583241F28831C5
S31508009FB87868FFF741FF0346002B01D002231DE00E
S31508009FC84FF47A624FF4FA617868FFF735FF03466B
S31508009FD8002B01D0032311E04FF4FA620B49786885
S31508009FE8FFF72AFF0346002B01D0042306E07B6807
S31508009FF8074A934201DA052300E00623184608377C
S3150800A008BD4680BD24FAFFFFFDD6FFFF18FCFFFFFB
S3150800A01815D3FFFF80B483B000AF0346FB71FB7905
S3150800A028052B07D1064B1B780A2B01D8642302E0B7
S3150800A0383C2300E00A2318460C37BD4680BC704707
S3150800A0480102002080B584B000AF0023FB6000231E
S3150800A058BB6000237B600420FFF7D0FEF860FB682E
S3150800A06840F6E44203FB02F20D4BA3FB0213D21A95
S3150800A07852081344DB0ABB60BB68A3F2BB634FF400
S3150800A0887A7202FB03F3074A82FB03129211DB1763
S3150800A098D31A7B607B6818461037BD4680BD00BF5B
S3150800A0A8010110007FE0077E80B500AF0E4B1B68E4
S3150800A0B89F229A620C4B1B6840F2C112DA620A4B5D
S3150800A0C81B684FF4E1729A63074B1B6840F2C71284
S3150800A0D85A630421044806F087FF0021024806F05F
S3150800A0E835FE00BF80BD00BFC80E002080B485B00D
S3150800A0F800AF0346FB71FB794FF4E17202FB03F3E9
S3150800A1080B4A82FB03125211DB17D31AFB60094A62
S3150800A118FB791370084B1B68FA689A63064B1B6829
S3150800A12801225A6300BF1437BD4680BC704700BF7A
S3150800A1381F85EB5101020020C80E002080B400AF2D
S3150800A148024B1B781846BD4680BC704701020020A2
S3150800A15890B585B000AF224B1B68FB6003F008FC7E
S3150800A168B860204B1B78062B02D01E4B1B7832E0B2
S3150800A1781D4B1B781946F868FFF7A2FE0346FB71C4
S3150800A188194B1B78FA799A4207D1174B1A78174B45
S3150800A1981A70174ABB6813601BE0144B1B78FA79C8
S3150800A1A89A4206D0114AFB791370114ABB681360A4
S3150800A1B80FE00F4B1B68BA68D41A0C4B1B78184665
S3150800A1C8FFF728FF03469C4203D3084B1A78064B29
S3150800A1D81A70054B1B7818461437BD4690BD00BF44
S3150800A1E8FC010020040000200500002006000020CD
S3150800A1F80402002080B582B000AF78607B681B68CF
S3150800A2080E4A934216D17B681B7F012B12D1FFF7A2
S3150800A21839FB0346002B0CD0FFF714FF0346084A00
S3150800A2281360074B1B681846FFF71CFEFFF75CFB15
S3150800A23800E000BF0837BD4680BD00BF00040040E7
S3150800A248F801002080B500AF064B074A1A60054892
S3150800A25805F0A5F80346002B01D000F0CBFB00BF9C
S3150800A26880BD00BF080200200030024080B485B0D7
S3150800A27800AF78607B681B68094A93420BD1094B83
S3150800A2885B69084A43F040035361064B5B6903F070
S3150800A2984003FB60FB6800BF1437BD4680BC7047A7
S3150800A2A8003002400010024080B584B000AFF86064
S3150800A2B8B9607A607B689BB21946B86800F006F8F8
S3150800A2C87B6818461037BD4680BD000080B485B047
S3150800A2D800AF78600B467B8072B600BF0023FB810F
S3150800A2E845E0284BB3F804349BB2B3F5806F18D30E
S3150800A2F8244BB3F802349BB201335A42C3F3090319
S3150800A308C2F3090258BF53429AB21E4BA3F8022455
S3150800A3181C4BB3F804349BB2013B9AB2194BA3F809
S3150800A3280424FB897A681344164AB2F8002492B2C0
S3150800A3381978144B9954134BB3F800349BB201336C
S3150800A3485A42C3F30903C2F3090258BF53429AB2E1
S3150800A3580C4BA3F800240B4BB3F804349BB2013317
S3150800A3689AB2084BA3F80424FB890133FB81FA89BE
S3150800A3787B889A42B5D362B600BF00BF1437BD467C
S3150800A38880BC70471002002080B483B000AF72B654
S3150800A39800BF064BB3F80434FB8062B600BFFB88DF
S3150800A3A818460C37BD4680BC704700BF100200200F
S3150800A3B880B582B000AF72B600BF2D4BB3F804342F
S3150800A3C89BB2002B02D162B600BF4EE0284BB3F809
S3150800A3D80434FB80FB88802B01D98023FB80244B1F
S3150800A3E8B3F802349BB2C3F58063BB80FA88BB888E
S3150800A3F89A4201D9BB88FB801D4BB3F804349BB23B
S3150800A408FA889A420CD11A4BB3F802349BB21A4608
S3150800A418174B1344F9885022184602F0E5F90BE061
S3150800A428134BB3F802349BB21A46114B1344F988F6
S3150800A4385122184602F0D8F90D4BB3F802349AB2ED
S3150800A448FB8813449BB2C3F309039AB2084BA3F8D3
S3150800A4580224074BB3F804349AB2FB88D31A9AB283
S3150800A468034BA3F8042462B600BF0837BD4680BD6F
S3150800A478100200200EB480B585B000AF0346FB7104
S3150800A488154AFB79137007F12003BB60BB68FA69A4
S3150800A4987E21124808F0D0FDF860FB68002B01DA27
S3150800A4A8FB6812E0FB687D2B01DD7E23FB60FB68F9
S3150800A4B80133094A0021D154FB689BB202339BB287
S3150800A4C819460548FFF702FFFB6818461437BD46C4
S3150800A4D8BDE8804003B0704718060020190600201A
S3150800A4E880B58AB000AF07F1140300221A605A60D3
S3150800A4F89A60DA607D4B9B697C4A43F01003936146
S3150800A5087A4B9B6903F010033B613B69774B9B6960
S3150800A518764A43F004039361744B9B6903F004037A
S3150800A528FB60FB68714B9B69704A43F008039361AB
S3150800A5386E4B9B6903F00803BB60BB686B4B9B6952
S3150800A5486A4A43F040039361684B9B6903F04003EA
S3150800A5587B607B68654B9B69644A43F0200393617B
S3150800A568624B9B6903F020033B603B680022382155
S3150800A5785F4805F00EFA00224FF4F8515D4805F0D9
S3150800A58808FA00224FF400415B4805F002FA002257
S3150800A59818215A4805F0FDF900228021584805F087
S3150800A5A8F8F938237B610123BB610023FB61022389
S3150800A5B83B6207F1140319464D4805F04FF8022384
S3150800A5C87B610023BB610023FB6107F1140319466D
S3150800A5D8494805F043F804237B610023BB6102233D
S3150800A5E8FB6107F114031946434805F037F844F2A6
S3150800A5F882037B610023BB610023FB6107F1140317
S3150800A60819463C4805F02AF84FF4F8537B610123AC
S3150800A618BB610023FB6102233B6207F11403194659
S3150800A628344805F01BF84FF400437B610123BB61EE
S3150800A6380023FB6102233B6207F1140319462E48DF
S3150800A64805F00CF818237B610123BB610023FB6125
S3150800A65802233B6207F114031946284804F0FEFF53
S3150800A66880237B610023BB610023FB6107F1140388
S3150800A6781946224804F0F2FF18237B610023BB61C0
S3150800A6880023FB6107F1140319461D4804F0E6FF89
S3150800A69880237B610123BB610023FB6102233B62A4
S3150800A6A807F114031946164804F0D8FF4FF4407307
S3150800A6B87B611223BB6103233B6207F11403194626
S3150800A6C80F4804F0CBFF0F4B5B687B627B6A43F04D
S3150800A6D8E0637B627B6A43F002037B62094A7B6A12
S3150800A6E8536000BF2837BD4680BD00BF0010024032
S3150800A6F800100140001801400008014000140140FC
S3150800A708000C01400000014080B400AF034B044A26
S3150800A7189A6000BFBD4680BC704700BF00ED00E0E8
S3150800A7280080000880B485B000AF03460A46FB716E
S3150800A7381346BB71BB791F2B01D900230EE00023F2
S3150800A748FB73BB79084AD35CFA799A4201D001238C
S3150800A758FB73BB790449FA79CA54FB7B1846143744
S3150800A768BD4680BC704700BF9806002080B584B0F7
S3150800A77800AF786003F0FCF8B8607B68FB60FB689C
S3150800A788B3F1FF3F0ED00E4B1B781A46FB681344ED
S3150800A798FB6007E001F02CF9FFF760FA01F010F802
S3150800A7A801F0A8FE03F0E4F80246BB68D31AFA6873
S3150800A7B89A42EFD800BF00BF1037BD4680BD00BF1C
S3150800A7C87400002080B500AF0320FEF7EDFE0346AF
S3150800A7D8002B02D1024B01221A7000BF80BD00BFB0
S3150800A7E8D401002080B500AF0B4804F015F8FFF730
S3150800A7F895F8094803F0CCFF0346002B01D000F072
S3150800A808F9F80221044804F074FA0346002B01D02B
S3150800A81800F0F0F800BF80BD8001002080B582B046
S3150800A82802AFFFF771FF03F04BF805F0D7F800F011
S3150800A83871F8FFF755FEFEF7A5FDFFF76FF8FFF766
S3150800A848A3F801F05BF802F0F7FC02F075FEFFF7D3
S3150800A858F9FC02F01DFE02F045FE02F097FE02F032
S3150800A86875FCFEF7F3FE00F08BFF4FF4967003F0C5
S3150800A87889F801F0DBFA01F029FE21490720FFF7DC
S3150800A888F9FD01F0FFFD1F4B1B889BB21A461E49AE
S3150800A8980720FFF7EFFD1B4B9B781A461B49072035
S3150800A8A8FFF7E8FD174B9B889BB21A46154BDB88C2
S3150800A8B89BB21946134B1B899BB200930B46144946
S3150800A8C80720FFF7D7FDFFF78DFF00F07DFAFFF7A2
S3150800A8D86FF900F087FB00F025FC0A20FFF746FF12
S3150800A8E800F08EF8FFF77AF900F010FE0A20FFF755
S3150800A8F83DFFFFF767FF3220FFF738FF00BFE8E79D
S3150800A908D4410108B80E0020E8410108FC410108B5
S3150800A9181042010880B59CB000AF07F13803382209
S3150800A9280021184608F096FB07F1240300221A604E
S3150800A9385A609A60DA601A613B1D2022002118467F
S3150800A94808F088FB0523BB634FF480333B64042374
S3150800A9587B640123BB640123FB644FF48033FB63E8
S3150800A9680223BB654FF48033FB654FF4E0133B665F
S3150800A97802237B664FF4C063BB664023FB6607F178
S3150800A9883803184605F0FAF80346002B01D000F0FC
S3150800A99831F80F237B620223BB620023FB624FF464
S3150800A9A880633B6300237B6307F12403022118466F
S3150800A9B805F0FAFB0346002B01D000F01BF8032329
S3150800A9C87B604FF48073BB604FF40043FB603B1D0C
S3150800A9D8184605F0DFFD0346002B01D000F00AF8FB
S3150800A9E8034B01221A6000BF7037BD4680BD00BF01
S3150800A9F87000424280B400AF72B600BF00BFFDE7E0
S3150800AA082DE9B04384B000AF2E4B00221A712E4BA5
S3150800AA185B78082B04D12B4B012283F8242003E00A
S3150800AA28284B002283F8242002F0A2FFF860254B61
S3150800AA389B68FA68D31ABB60224AFB689360224B64
S3150800AA48D3F80330BA6802FB03F3204AA2FB0323B0
S3150800AA589B097B601B4BD3E90423796800200C46C5
S3150800AA68054612EB040843EB0509164BC3E90489A6
S3150800AA78144BD3E90423164BA3FB0223DB0A114A1A
S3150800AA889361104B93F82430002B08D00D4B9A6924
S3150800AA980C4BDB69D31A0C4AC2F807300CE00A4B90
S3150800AAA80022DA7100221A7200225A7200229A7259
S3150800AAB8044B9B69034AD36100BF1037BD46BDE8FE
S3150800AAC8B08300BFB8060020D4010020D34D621019
S3150800AAD8C5B3A29180B582B000AF0346FB71064A9A
S3150800AAE8FB79D37102F044FF0346034A136100BF9A
S3150800AAF80837BD4680BD00BF2407002080B500AFD3
S3150800AB0802F036FF0246024B1B69D31A184680BD67
S3150800AB182407002080B584B000AF7860884B894A3E
S3150800AB280121786803F0C4FF0346002B40F004812E
S3150800AB38844B5B68BB603B7A002B40F0FC8002F0D4
S3150800AB4817FF0346804A1360BB7A03F03F03DBB25C
S3150800AB58022B05D17D4B7A4A92E8030083E8030065
S3150800AB68BB7A03F03F03DBB2042B19D1784B744A3E
S3150800AB7892E8030083E80300754B1B791A46754B60
S3150800AB88DA61734B1A7A734B83F82020704BDA799B
S3150800AB98704B83F821206E4B9A796E4B83F82220E6
S3150800ABA8BB7A03F03F03DBB2062B23D16A4B644A10
S3150800ABB892E8030083E80300674B5B781A46664BFE
S3150800ABC81B781B0213441A46634B9A60624BDB7860
S3150800ABD81A46614B9B781B0213441A465E4BDA6089
S3150800ABE85D4B5B791A465C4B1B791B0213441A4664
S3150800ABF8594B1A61BB7A03F03F03DBB2082B05D120
S3150800AC08564B4F4A92E8030083E80300BB7A03F0E1
S3150800AC183F03DBB2092B40F08F80514B484A92E834
S3150800AC28030083E803004E4BDB791A464C4BDA607F
S3150800AC384B4BDA684A4B9B791B021343484AD36045
S3150800AC48474BDA68464B5B791B041343444AD3607F
S3150800AC58434BDA68424B1B791B061343404AD360B9
S3150800AC683F4BDB781A463E4B9A603D4B9A683C4BFD
S3150800AC789B781B0213433A4A9360394B9A68384BB8
S3150800AC885B781B041343364A9360354B9A68344BF2
S3150800AC981B781B061343324A9360314B9B68314A2B
S3150800ACA8A2FB03239B09FB812D4BDB682E4AA2FBDB
S3150800ACB803235B09BB81274AFB895380254ABB893D
S3150800ACC89380FB89132B8CBF01230023DBB21A461A
S3150800ACD8204B9A721F4B01221A721D4B1A791D4B6B
S3150800ACE89A711C4BDB79012B26D91A4B5A881F4BAC
S3150800ACF8A3F81320174BB3F904309AB21B4BA3F8E1
S3150800AD0815201A4BB3F815309BB21A46174BB3F8E9
S3150800AD1813309BB202FB03F3154A82FB0312921007
S3150800AD28DB17D31A1A46114BC3F80320094B9A7A2C
S3150800AD380E4B1A7600E000BF1037BD4680BD00BF2F
S3150800AD48680700204C07002048070020E006002076
S3150800AD58EC06002024070020F80600200C0700202F
S3150800AD6814070020D34D62101F85EB51D40100202B
S3150800AD786766666680B58AB000AF0E237B610023D6
S3150800AD88BB610123FB6100233B6000237B60002332
S3150800AD98BB600023FB6000233B6101233B62012360
S3150800ADA83B610E237B623B461946064803F010FCB6
S3150800ADB80346002B01D0FFF71DFE00BF2837BD4606
S3150800ADC880BD00BFA801002080B500AF134803F076
S3150800ADD823FDFEF7D9FDFFF7CDFF104803F0D8FC91
S3150800ADE810210E4803F085FF242200210C4808F09C
S3150800ADF831F90B4B0022DA7102F0BAFD0346084A0C
S3150800AE081361074B47F230525A61054B00221A76EE
S3150800AE180021002000F006F800BF80BDA801002028
S3150800AE282407002080B584B000AF03460A46FB71A4
S3150800AE381346BB7107F1080308220021184608F0D3
S3150800AE4809F9FB79002B15D10D4B1B7A002B13D06A
S3150800AE58BB79002B0CBF01230023DBB23B72F979BF
S3150800AE6807F108031A22F02000F066F81420FFF705
S3150800AE787DFC02E000BF00E000BF1037BD4680BD7C
S3150800AE882407002080B586B000AF0346FB710B4641
S3150800AE98BB8013467B8007F1080308220021184661
S3150800AEA808F0D8F8FB79002B40D1BB88952B01D838
S3150800AEB89623BB801F4B1B7E002B06D1BB88B3F598
S3150800AEC8FA7F02D340F2F313BB807B88642202FB25
S3150800AED803F37B61BB884FF47A7202FB03F33B6189
S3150800AEE87B691B0EDBB23B737B691B0CDBB27B737E
S3150800AEF87B691B0ADBB2BB737B69DBB2FB733B69F5
S3150800AF081B0EDBB23B723B691B0CDBB27B723B69DF
S3150800AF181B0ADBB2BB723B69DBB2FB72F97907F134
S3150800AF2808031C22F02000F007F800E000BF1837D5
S3150800AF38BD4680BD2407002080B58CB000AF3B60B5
S3150800AF480346FB710B46BB7113467B71FB7987F881
S3150800AF582830BB7987F829307B7903F03F03DAB2C2
S3150800AF6897F82A3062F3050387F82A307B8D0A2278
S3150800AF7862F389137B850A2387F82F30BB6A7B61BE
S3150800AF880023FB610423BB6108233B621EE01448C7
S3150800AF9803F05AFD0346002B0ED007F10C0307F100
S3150800AFA810013A680E4803F080FC034687F82E30ED
S3150800AFB897F82E30002B0ED00120FFF7D7FB97F90C
S3150800AFC82F30DBB2013BDBB287F82F3097F92F30E9
S3150800AFD8002BDCDC00E000BF3037BD4680BD00BF73
S3150800AFE8A801002080B582B000AF3B4600221A604F
S3150800AFF85A603B4604220021F020FFF79DFF1420E3
S3150800B008FFF7B4FB3B4606220021F020FFF794FF22
S3150800B0181420FFF7ABFB3B4609220021F020FFF777
S3150800B0288BFF1420FFF7A2FB3A4BB3F81B309BB2F1
S3150800B038394AA2FB0323DB089BB21A46354BB3F8F9
S3150800B04813309BB202FB03F31A46344B5B699A42E8
S3150800B05811D9324B5A6913469B0013445B001A46AA
S3150800B0682C4BB3F813309BB2B2FBF3F39AB2294BC5
S3150800B078A3F8112006E0274BB3F81B309AB2254BE4
S3150800B088A3F81120234BB3F811309BB240F2325281
S3150800B098934208D91F4B002242F032025A74002202
S3150800B0A842F005029A741B4BB3F811309BB21A4644
S3150800B0B8184BB3F80F309BB202FB03F3184A82FB0E
S3150800B0C803129210DB17D31A1A46124BC3F80B2031
S3150800B0D8124B5B7A002B18D00E4BB3F80F309BB285
S3150800B0E80C4AB2F8112092B219460020FFF7CAFE98
S3150800B0F81420FFF73BFB074BB3F813309BB2B3F5A5
S3150800B108F57F02D9054B01221A7600BF0837BD46D6
S3150800B11880BD00BFD4010020CDCCCCCC24070020AC
S3150800B1286766666698B500AF02F022FC0246B44B1D
S3150800B1381B68D31AB3F5FA7F20D9B24B00221A72C4
S3150800B148B04B00229A72B04B00221A71AE4B0022FD
S3150800B1581A72AD4B0022DA71AB4B00229A71AB4BCF
S3150800B16800229A60A94B0022DA60A84B00221A61CD
S3150800B178A74B0022DA60A64B00229A60A14B1B7ADD
S3150800B188002B03D09F4B1B78002B0CD1A14B002218
S3150800B198DA7400221A759F4B00225A7500229A758E
S3150800B1A89C4B00221A769B4B9B7F002B0CD00121C7
S3150800B1B80420FEF779F902F0DBFB0346964A13608A
S3150800B1C8904B01221A7010E002F0D2FB0246924B0D
S3150800B1D81B68D31A4EF66022934206D9002104202A
S3150800B1E8FEF762F9874B00221A700520FEF7DCF98C
S3150800B1F803461A46834BDA72824B1B7A002B07D012
S3150800B208804B1B7B002B03D17E4B1B78002B02D16E
S3150800B2187C4B00225A727B4BDB79092B00F255814D
S3150800B22801A252F823F000BF59B200088DB20008EF
S3150800B238A9B20008E1B200082FB3000871B30008E4
S3150800B248DBB3000885B4000835B40008BFB40008A5
S3150800B2586C4B00225A7000210320FEF725F9694B2A
S3150800B2681B7A002B00F03581664B1B78002B00F003
S3150800B2783081644B1B7B002B40F02B810120FFF7A4
S3150800B28829FC26E1FFF73AFC0346B3F57A6F40F244
S3150800B29822815C4B01225A720220FFF71BFC1AE135
S3150800B2A8584B00221A7600210320FEF7FDF8554B65
S3150800B2B85B7A002B03D10020FFF70CFC1CE1554BE9
S3150800B2C8DB7D002B00F0098101210020FFF7AAFD8C
S3150800B2D80320FFF7FFFB00E14A4B9B7A002B0CD0B3
S3150800B2E8484B5B7A002B08D002F042FB03464B4AD0
S3150800B2F813600420FFF7EEFBF1E0FFF7FFFB0346B8
S3150800B30842F21072934240F2EA803E4B01225A7387
S3150800B318404B0A225A770020FFF7DCFB40490420F5
S3150800B328FFF7A8F8DBE001210320FEF7BDF8354B47
S3150800B338DB7A002B03D00520FFF7CCFBD1E0FFF71B
S3150800B348DDFB0346B3F57A7F40F2CB802D4B01220D
S3150800B3581A73304B07225A770620FFF7BBFB314989
S3150800B3680420FFF787F8BCE02A4BDB7D002B03D0C7
S3150800B378244B5B7A002B03D10620FFF7ABFBBBE017
S3150800B3880520FEF711F903461C460320FEF7FCF8CC
S3150800B39803469C4217D002F0EBFA0246224B1B687A
S3150800B3A8D31AB3F57A7F40F29E801A4B07225A774A
S3150800B3B8144B01221A730620FFF78CFB194904203F
S3150800B3C8FFF758F88FE002F0D3FA0346164A1360D7
S3150800B3D889E0104B00225A7400229A740D4BB3F870
S3150800B3E815309BB21D2B06D9FFF788FB034641F299
S3150800B3F88832934279D90820FFF76CFB75E000BFBD
S3150800B4084807002024070020EC060020F80600203C
S3150800B41814070020D40100207007002074070020B4
S3150800B428284201083842010878070020002103202D
S3150800B438FEF73AF8314BDB7A002B07D100210020BA
S3150800B448FFF7F0FC0720FFF745FB50E0FFF756FB30
S3150800B4580346B3F57A7F4AD9284B01221A73284B33
S3150800B46807225A7700210020FFF7DCFC0720FFF7A0
S3150800B47831FB24490420FEF7FDFF38E01F4B9B7A71
S3150800B488002B03D10920FFF725FB32E0FFF736FB2F
S3150800B498034642F2107293422BD9184B01225A736B
S3150800B4A8174B0A225A770020FFF714FB164904207F
S3150800B4B8FEF7E0FF1DE0FFF721FB0346B3F57A6FB9
S3150800B4C819D90220FFF706FB15E00020FFF702FB53
S3150800B4D812E000BF10E000BF0EE000BF0CE000BF9E
S3150800B4E80AE000BF08E000BF06E000BF04E000BFAE
S3150800B4F802E000BF00E000BF00BF98BD2407002097
S3150800B508D4010020384201085842010880B500AF26
S3150800B518344B5B7F002B03D0334800F01FF95FE0FC
S3150800B528304B5B780D2B57D801A252F823F000BF91
S3150800B53871B5000879B5000881B5000889B500080D
S3150800B54891B5000899B50008A1B50008A9B500087D
S3150800B558B1B50008B9B50008C1B50008C9B50008ED
S3150800B568D1B50008D9B50008204800F0F7F837E043
S3150800B5781F4800F0F3F833E01B4800F0EFF82FE017
S3150800B5881C4800F0EBF82BE01A4800F0E7F827E02B
S3150800B598194800F0E3F823E0174800F0DFF81FE041
S3150800B5A8154800F0DBF81BE0134800F0D7F817E059
S3150800B5B8124800F0D3F813E0104800F0CFF80FE06F
S3150800B5C80E4800F0CBF80BE00C4800F0C7F807E087
S3150800B5D8084800F0C3F803E0044800F0BFF800BFC5
S3150800B5E880BD00BFD40100204400002008000020C8
S3150800B5F814000020200000202C000020380000201D
S3150800B60880B487B000AFF860B96011461A460B4691
S3150800B618FB801346BB80FA88BB889A4201D9BB8847
S3150800B628FB80BB88002B01D10123BB80FA8813460F
S3150800B6381B029A1ABB8892FBF3F3FB82FB681B78FA
S3150800B6481A46FB8AC3F1FF0303FB02F2BB681B78A1
S3150800B6581946FB8A01FB03F31344204A82FB0312AB
S3150800B6681A44D211DB17D31ADAB23B6A1A70FB6886
S3150800B6785B781A46FB8AC3F1FF0303FB02F2BB6831
S3150800B6885B781946FB8A01FB03F31344134A82FBCA
S3150800B69803121A44D211DB17D31ADAB23B6A5A7064
S3150800B6A8FB689B781A46FB8AC3F1FF0303FB02F281
S3150800B6B8BB689B781946FB8A01FB03F31344074AC0
S3150800B6C882FB03121A44D211DB17D31ADAB23B6A81
S3150800B6D89A7000BF1C37BD4680BC70478180808041
S3150800B6E880B483B000AF78607B681B781A466423F9
S3150800B6F802FB03F3174A82FB03121A44D211DB171B
S3150800B708D21A154B1B689A637B685B781A466423BA
S3150800B71802FB03F30F4A82FB03121A44D211DB1702
S3150800B728D21A0D4B1B68DA637B689B781A46642322
S3150800B73802FB03F3074A82FB03121A44D211DB17EA
S3150800B748D21A054B1B681A6400BF0C37BD4680BC65
S3150800B758704700BF81808080100F002080B483B0B6
S3150800B76800AF7860054B7A681068516803C3128978
S3150800B7781A8000BF0C37BD4680BC70478407002076
S3150800B78880B582B000AF00233B7100237B7100238C
S3150800B798BB710421094805F027FC0821074805F06C
S3150800B7A823FC0C21054805F01FFC3B1D1846FFF72E
S3150800B7B897FF00BF0837BD4680BD00BF100F0020A1
S3150800B7C880B582B002AF02F0D3F80246464B1B6832
S3150800B7D8D31A142B40F2858002F0CAF80346424A67
S3150800B7E81360424B5B8801339AB2404B5A803F4BF1
S3150800B7F81B78032B67D801A252F823F015B800085E
S3150800B80847B8000873B80008A5B80008374B5A881F
S3150800B818374BDB781946374B00930B46344936487D
S3150800B828FFF7EEFE314B5B88314AD27893424ED900
S3150800B8382E4B01221A702D4B00225A8047E02B4BBB
S3150800B8482B4A04331268114619800233120C1A70EF
S3150800B858264B5B88264A127993423AD9234B022209
S3150800B8681A70224B00225A8033E0204B5A88204B04
S3150800B8785B7919461F4B00930B461F491C48FFF76F
S3150800B888BFFE1A4B5B881A4A5279934223D9174B3B
S3150800B89803221A70154B00225A801CE0134B144ACF
S3150800B8A8043307321188927819809A700F4B5B888F
S3150800B8B80F4A9279934210D90C4B00221A700B4BF7
S3150800B8C800225A8009E0094B00221A7006E000BFD8
S3150800B8D804E000BF02E000BF00E000BF0548FFF72C
S3150800B8E8FFFE00BFBD4680BD900700207C070020EC
S3150800B8F884070020800700208B07002080B500AF4A
S3150800B9080A4B0B4A1A60094B4FF0FF325A60074B2D
S3150800B9184FF480729A60054805F0C0F80346002B74
S3150800B92801D0FFF767F800BF80BD00BF9407002065
S3150800B9380028004080B584B000AF78607B681B6833
S3150800B9480B4A934210D104F03DF80A4BDB69094AC1
S3150800B95843F00063D361074BDB6903F00063FB60C0
S3150800B968FB68054B01221A6000BF1037BD4680BD2B
S3150800B97800280040001002403C04424280B400AF50
S3150800B988BFF34F8F00BF064BDB6803F4E062044938
S3150800B998044B1343CB60BFF34F8F00BF00BFFDE7CF
S3150800B9A800ED00E00400FA0580B582B000AF7860C3
S3150800B9B80B467B807B680B4A93420FD10A4B0022C1
S3150800B9C81A707B88002B0AD07B88B3F5807F06D847
S3150800B9D87B881946054800F0E5FC00E000BF0837F3
S3150800B9E8BD4680BD30100020CC090020CC070020B9
S3150800B9F880B500AFAA4B1B78002B11D1A94806F0D1
S3150800BA089CFE0346202B0BD14FF48072A649A54805
S3150800BA1806F074FA0346002B02D1A14B01221A70CC
S3150800BA28FEF796FB03461A46A04B1A70A04B1B78DE
S3150800BA38002B03D09E4B1A789E4B1A7001F098FF7C
S3150800BA4802469D4B1B68D31A0A2B53D901F090FF5F
S3150800BA5802469A4B1B68D31AC72B06D900F01CFB5B
S3150800BA6801F086FF0346954A1360954B1B78002B11
S3150800BA7808D094490420FEF7FDFC00F0AEFA904B76
S3150800BA8800221A708A4B1B78012B03D0884B5B7FE0
S3150800BA98002B13D001F06CFF02468B4B1B68D31A98
S3150800BAA8B3F57A7F0AD901F063FF0346864A13601D
S3150800BAB886490520FEF7DEFC00F08FFA844B1B78D2
S3150800BAC80C2B03D0824B1B780B2B13D101F050FF9C
S3150800BAD802467D4B1B68D31AB3F57A7F0AD901F05B
S3150800BAE847FF0346784A13607A490520FEF7C2FCE1
S3150800BAF800F073FA784B1B78002B07D10121052033
S3150800BB08FDF7D2FC0020FEF7D1F8FEE0734B1B7850
S3150800BB18042B00F2FA8001A252F823F039BB000878
S3150800BB2859BB00089DBB0008DBBB00082BBC0008F6
S3150800BB3800210520FDF7B8FC0220FEF7B7F85C4B94
S3150800BB485B7F002B40F0A880644B01221A70A3E0A3
S3150800BB5801210520FDF7A8FC0120FEF7A7F8534B9D
S3150800BB681B78012B03D0514B1B78022B02D15B4B58
S3150800BB7802221A704E4B5B7F002B00F08F804C4BCD
S3150800BB885B7F1A4656490420FEF774FC534B00227D
S3150800BB981A7083E001210520FDF786FC0420FEF7CC
S3150800BBA885F8434B1B78022B06D14E490720FEF72A
S3150800BBB861FC4A4B03221A703C4B1B78002B40F059
S3150800BBC89F8049490720FEF755FC444B01221A7005
S3150800BBD896E001210520FDF767FC3D4B1B78022BF3
S3150800BBE803D80320FEF762F804E0394B1B78184699
S3150800BBF8FEF75CF82D4B1B78002B06D13A4907202F
S3150800BC08FEF738FC354B01221A70384B1B78002B87
S3150800BC1878D037490720FEF72DFC304B04221A70D6
S3150800BC2870E000210520FDF73FFC0D20FEF73EF8E1
S3150800BC3801F09EFE02462F4B1B68D31AB3F57A7F8E
S3150800BC481AD901F095FE03462A4A1360274B1B7832
S3150800BC58002B0AD0254B1B78FF2B0DD0234B1B78BE
S3150800BC68013BDAB2214B1A7006E023490720FEF792
S3150800BC7801FC1A4B01221A701C4B1B78002B43D166
S3150800BC880A4B1B78012B3FD11C490720FEF7F2FB0C
S3150800BC98124B02221A7037E000BF36E000BF34E0C4
S3150800BCA8CC09002030100020CC0700204F000020C7
S3150800BCB8D4010020C8070020C0070020300A002049
S3150800BCC8CD0900206C420108C407002080420108FB
S3150800BCD82C0A002098420108C20E002050000020B5
S3150800BCE8B4420108DC42010800430108CE090020D5
S3150800BCF810430108340A0020204301084843010874
S3150800BD0800BF02E000BF00E000BF3F4B1B78002BD6
S3150800BD181FD03E4B1B68002B08D001F029FE0246AF
S3150800BD283A4B1B68D31AB3F5FA6F08D33849042077
S3150800BD38FEF7A0FB01F01CFE0346344A1360354B98
S3150800BD480022DA75344B00221A706420FEF7CEF901
S3150800BD5844E0324B1B68002B23D001F009FE02464B
S3150800BD682E4B1B68D31AB3F5FA6F1AD9284904203B
S3150800BD78FEF780FB244B01221A7001F0F9FD0346F1
S3150800BD88264A136001F0F4FD0346204A1360214B46
S3150800BD980022DA75204B00221A706420FEF7A6F9ED
S3150800BDA81CE01F4B1B78012B03D11A4B0022DA75AE
S3150800BDB814E01C4B1B78002B14BF01230023DBB2AD
S3150800BDC81A46144BDA75134BDB7D002B06D1114B3B
S3150800BDD85B78032B02D10F4B0022DA75124B1B78BE
S3150800BDE8012B07D0104B1B78022B03D00E4B1B7860
S3150800BDF8032B03D1074B01229A7703E0054B002250
S3150800BE089A7700BF00BF80BDD8090020DC0900204A
S3150800BE1884430108D40100202C0A0020D4090020F4
S3150800BE28C8070020C90700204F00002080B500AFCA
S3150800BE38FEF73AF96420FEF759F90D4B4FF47A7272
S3150800BE481A800B4B96225A80094B40F232529A8036
S3150800BE58074B0A22DA80064B47F230529A6000F0FE
S3150800BE68B3F804490720FEF705FB00BF80BD00BFED
S3150800BE78A80700209843010880B485B000AF786009
S3150800BE880B467B804FF6FF73FB810023BB8122E0BC
S3150800BE98BB897A6813441B781A46FB895340FB8189
S3150800BEA80023FB7211E0FB8903F00103002B06D07F
S3150800BEB8FB895B089AB20D4B5340FB8102E0FB896C
S3150800BEC85B08FB81FB7A0133FB72FB7A072BEAD9FD
S3150800BED8BB890133BB81BA897B889A42D8D3FB8947
S3150800BEE818461437BD4680BC704700BF01A0FFFF3F
S3150800BEF880B586B000AFB9607B600346FB7313460E
S3150800BF08BB81BB890333FB82FA8A3B8C9A4201D9E7
S3150800BF18002329E07B68FA7B1A70BB89002B09D0B5
S3150800BF28BB68002B06D07B680133BA89B9681846FE
S3150800BF3807F00BF9BB8901339BB219467868FFF7F6
S3150800BF489BFF0346BB82BB8901337A681344BA8AC6
S3150800BF58D2B21A70BB8A1B0A99B2BB8902337A68AD
S3150800BF681344CAB21A70FB8A18461837BD4680BDEC
S3150800BF7880B586B002AF03463960FB711346BB80AD
S3150800BF88BA88F8794FF4807300930C4B3968FFF731
S3150800BF98AFFF0346FB81FB89002B06D0FA894FF4CD
S3150800BFA87A730649064805F0E9FE01F0E1FC0346FE
S3150800BFB8044A136000BF1037BD4680BDCC08002070
S3150800BFC830100020C007002080B500AF00220021ED
S3150800BFD85220FFF7CDFF00BF80BD80B500AF002215
S3150800BFE800215320FFF7C4FF00BF80BD80B582B08B
S3150800BFF800AF01F0BDFC78601E4B1B687A68D31A3F
S3150800C0083B601C4A7B6813601B4BB3F813309BB222
S3150800C0181A46194BB3F815309BB202FB03F3174AB5
S3150800C02882FB03129210DB17D31A1A46144B1A60AE
S3150800C038134B1B683A6802FB03F3124AA2FB032355
S3150800C0489A09114B1B6813440F4A13600F4B1B7848
S3150800C058012B02D10C4B00221A600B4B1B680C4AA9
S3150800C068A2FB0323DB0A0B4A136000BF0837BD4649
S3150800C07880BD00BF380A0020D401002067666666BE
S3150800C088B4070020D34D6210B80700202C0A0020F8
S3150800C098C5B3A291BC07002080B500AFFFF7A6FF7D
S3150800C0A8FEF74CF803461A462A4B1A702A4BDA7AD0
S3150800C0B8284B5A70294BB3F813309AB2254B5A8035
S3150800C0C8264BB3F815309AB2224B9A80244B1B6834
S3150800C0D8204AC2F80630234B1B681E4AC2F80A30A3
S3150800C0E8214B1B78032B04D1204B1A78194BDA7489
S3150800C0F802E0184B0022DA741D4B1A88154B9A82EF
S3150800C1081B4B5A88134BDA82194B9A88114B1A8398
S3150800C118174BDA880F4B5A83154B9B680D4AD36120
S3150800C128144B1A780B4B9A740A4A002343F07F4338
S3150800C13843F47F0343F43B4343F0A003D38100232E
S3150800C14843F00D031382202202495020FFF710FFFF
S3150800C15800BF80BDE009002024070020D401002084
S3150800C168B4070020BC070020500000204F0000201C
S3150800C178A8070020D009002080B483B000AF034682
S3150800C188FB71FB79403B092B2AD801A252F823F008
S3150800C198C1C10008C5C10008C9C10008CDC1000849
S3150800C1A8D1C10008D5C10008D9C10008DDC10008F9
S3150800C1B8E1C10008E5C10008012313E0012311E0E5
S3150800C1C801230FE001230DE001230BE0042309E016
S3150800C1D8012307E02C2305E0012303E0002301E0FF
S3150800C1E84FF6FF7318460C37BD4680BC704700BF2C
S3150800C1F8F0B58BB000AF03463960FB711346BB80B8
S3150800C20801F0B6FB03465B4A13605B4B00221A70C3
S3150800C2185A4B00221A60FB79403B092B00F2A3808F
S3150800C22801A252F823F000BF59C2000887C20008C5
S3150800C238A1C20008C3C2000857C30008DDC2000827
S3150800C248FBC2000809C300084DC3000863C30008F9
S3150800C2583B68FB60FB681B7887F8273097F8273018
S3150800C268642B02D9642387F82730454A97F827307C
S3150800C278137097F827301846FDF738FF76E03B68BD
S3150800C2883B613B691B78002B14BF01230023DBB2F3
S3150800C2981A463C4B1A7069E03B687B617B691B78D8
S3150800C2A8002B62D038490520FEF7E4F8FFF78CFE24
S3150800C2B80A2001F067FBFFF761FB3B68BB61BB69B6
S3150800C2C81B78002B14BF01230023DBB21A462F4B19
S3150800C2D81A704BE03B68FB61FB691B889AB22C4BCA
S3150800C2E8A3F80F20FB695B889AB2294BA3F81B2091
S3150800C2F83CE03B683B623B6A1A78264B1A7035E085
S3150800C308254A3B681C46164604F1200C3546234642
S3150800C318186859689A68DB680FC51034103664457A
S3150800C328F4D13346224610685168926807C31A4BF7
S3150800C3385B881A4AA2FB0323DB089BB2DAB2144BC2
S3150800C3489A7013E03B681A78154B1A700EE00C4B76
S3150800C3581B781846FDF7CAFE08E001F009FB0346F4
S3150800C368044A136002E000BF00E000BF00BF2C3794
S3150800C378BD46F0BDD4090020D8090020DC090020F4
S3150800C3884E000020C9070020A4430108CF09002051
S3150800C398D4010020D0090020000A0020CDCCCCCC3E
S3150800C3A82C0A002080B586B000AF78600B467B80E3
S3150800C3B87B88022B01D800235AE07B681B78FB751B
S3150800C3C87B88033BBB827B88023B7A6813441B78CD
S3150800C3D81AB27B88013B79680B441B781BB21B028F
S3150800C3E81BB213431BB27B82BB8A01339BB2194625
S3150800C3F87868FFF741FD03463B827A8A3B8A9A4268
S3150800C40805D01D490420FEF735F8002330E0FB7DEA
S3150800C4181846FFF7B1FE0346FB81FB894FF6FF7204
S3150800C428934207D1FB7D1A4614490520FEF722F8E0
S3150800C43800231DE0FA89BB8A9A4207D0FB7D1A4673
S3150800C4480F490420FEF716F8002311E0BB8A002BD3
S3150800C45807D07B68591CBA8AFB7D1846FFF7C8FEC1
S3150800C46805E0FB7D002200211846FFF7C1FE0123DF
S3150800C47818461837BD4680BDBC430108D043010895
S3150800C488E443010880B400AF0E4B1B681B689AB2D8
S3150800C4980D4B1A800B4B1B685A790B4B9A70094B34
S3150800C4A81B681A79084BDA70074B01229A80064BE3
S3150800C4B80022DA80044B06221A8100BFBD4680BCDA
S3150800C4C8704700BF00000020B80E002080B500AFF6
S3150800C4D84FF404720021054806F0BCFD4FF40472B7
S3150800C4E80021034806F0B6FD00BF80BD3C0A0020BF
S3150800C4F84C0C002080B500AF2A4B93F84230DBB2CB
S3150800C508202B0AD1284B93F80832DBB2002B04D12A
S3150800C518FF222649234805F0F1FC254B93F84230BB
S3150800C528DBB2202B04D1FF222249214805F0E6FC7C
S3150800C5381C4B93F84130DBB2212B19D11A4BD3F88F
S3150800C5480C32002B14D001F013FA0246164BD3F816
S3150800C5580C32D31A642B0BD9124805F02DFD00228C
S3150800C5681021154803F015FA0F4B0022C3F80C22C0
S3150800C5780D4B93F80832DBB2002B11D0094B93F810
S3150800C5884130DBB2212B0BD00C4800F0EDF9FF2225
S3150800C5980649044805F0B2FC034B002283F8082232
S3150800C5A800BF80BDE80F00203C0A00203C0B002095
S3150800C5B8580F00204C0D0020001401403C0C0020A8
S3150800C5C880B582B000AF78600B467B807B681A68B6
S3150800C5D8224B1B689A4216D17B881A46204921485D
S3150800C5E800F08EF90346002B04D1142200210020FE
S3150800C5F800F0FAF81C4B00221A70FF22184917484F
S3150800C60805F07CFC25E07B681A68184B1B689A427B
S3150800C61814D17B881A461649164800F071F903465C
S3150800C628002B05D0104B01221A70134800F09CF90C
S3150800C638FF220F490D4805F061FC0AE07B681A6875
S3150800C6480E4B1B689A4204D17B8819467868FFF70F
S3150800C658ABF900BF0837BD4680BD00BFE80F00200C
S3150800C6683C0B00203C0A00205C0E0020580F0020D6
S3150800C6784C0D00204C0C00204C0E002030100020D9
S3150800C68880B582B000AF78607B681A68084B1B686B
S3150800C6989A4208D100221021064803F07AF9064B77
S3150800C6A80022C3F80C2200BF0837BD4680BD00BF6C
S3150800C6B8E80F0020001401403C0A002080B485B029
S3150800C6C800AF78600B467B804FF0FF33FB60002392
S3150800C6D87B8121E07B897A6813441B781A46FB68B4
S3150800C6E85340FB6000237B7210E0FB6803F00103EC
S3150800C6F8002B05D0FB685A080D4B5340FB6002E037
S3150800C708FB685B08FB607B7A01337B727B7A072BB5
S3150800C718EBD97B8901337B817A897B889A42D9D37D
S3150800C728FB68DB4318461437BD4680BC704700BF14
S3150800C7382083B8ED80B588B000AFF8607A601A46ED
S3150800C7480B467B8113467B720023FB83FB8B5A1CA3
S3150800C758FA831A467B6813447A7A1A70FB68002BA0
S3150800C76819D00023BB8312E0BB8BFA681A44FB8BEB
S3150800C778591CF98319467B680B4412781A70FB8B87
S3150800C788FA2B01D900232AE0BB8B0133BB83BA8B6A
S3150800C7987B899A42E8D3FB8B19467868FFF78EFFA0
S3150800C7A803463B6107F110037B610023BB6112E076
S3150800C7B8BB697A691A44FB8B591CF98319467B6845
S3150800C7C80B4412781A70FB8BFE2B01D9002306E05E
S3150800C7D8BB690133BB61BB69032BE9DDFB8B1846D3
S3150800C7E82037BD4680BD000080B584B000AF7860AC
S3150800C7F80B467B8013467B707B787988154A786860
S3150800C808FFF798FF0346FB81FB89002B1ED0124BC6
S3150800C81893F84130DBB2212B07D10F4805F0CCFB42
S3150800C828002210210D4803F0B4F8012210210B4804
S3150800C83803F0AFF8FB891A460649074805F029FBAD
S3150800C84801F096F80346034AC2F80C3200BF1037BF
S3150800C858BD4680BD3C0A0020E80F002000140140B0
S3150800C86880B588B000AFF8600B467A607B817B8913
S3150800C878042B01D800233FE07B89B3F5807F01D9D3
S3150800C888002339E07B89043BFB83FB8BFA68134456
S3150800C8981B781946FB8B0133FA6813441B781B026D
S3150800C8A841EA0302FB8B0233F9680B441B781B0425
S3150800C8B81A43FB8B0333F9680B441B781B0613438F
S3150800C8C8BB61FB8B1946F868FFF7F8FE7861BA6909
S3150800C8D87B699A4201D000230EE0FB685A1C7B68E4
S3150800C8E85A60FB681A787B681A70FB8BDBB2013BC7
S3150800C8F8DAB27B685A70012318462037BD4680BDD0
S3150800C90880B584B000AFF860B9601346FB80FB6851
S3150800C91803F50072FB881946B868FFF7A1FF0346B6
S3150800C928002B01D1002304E0FB68012283F80822C2
S3150800C938012318461037BD4680BD000080B400AFF5
S3150800C948BFF34F8F00BF064BDB6803F4E062044968
S3150800C958044B1343CB60BFF34F8F00BF00BFFDE7FF
S3150800C96800ED00E00400FA0580B584B000AF7860F1
S3150800C9781323FB737B681B78C22B00F3CC80B02B80
S3150800C9880FDA602B42D0602B00F3C580502B43D0BA
S3150800C998502B00F3C080012B00F0A680402B2DD029
S3150800C9A8B9E0B03B122B00F2B68001A252F823F088
S3150800C9B827CA00081FCB00081FCB00081FCB000892
S3150800C9C81FCB0008CFCA00081FCB00081FCB0008DA
S3150800C9D81FCB00081FCB00081FCB00081FCB000879
S3150800C9E81FCB00081FCB00081FCB00081FCB000869
S3150800C9F865CA0008C9CA00089DCA000800F0B2F846
S3150800CA08402258214B48FFF7EFFE8FE060220A21A3
S3150800CA184948FFF7E9FE89E0FDF7CAFC86E07B6826
S3150800CA285B780B2B17D17B685A68444B106851689A
S3150800CA3803C31189927A19809A70414B01221A7098
S3150800CA483E4BD3F803303D4A3E490720FDF712FD11
S3150800CA581223FB7362E01323FB735FE07B685B7842
S3150800CA68012B14D17B685B681B781A464FF47A73D6
S3150800CA7802FB03F31A46344B5A61334B5B691A4671
S3150800CA8832490720FDF7F6FC1223FB7346E0132309
S3150800CA98FB7343E07B685B78012B0ED17B685B6888
S3150800CAA81A782B4B1A702A4B1B781A4629490720DD
S3150800CAB8FDF7E0FC1223FB7330E01323FB732DE02C
S3150800CAC81323FB732AE0122200210020FFF78CFEAD
S3150800CAD800BF214B93F84130DBB2212BF9D00A204D
S3150800CAE800F050FFFFF72AFF7B685B78092B0FD108
S3150800CAF87B685A68194B1068516803C3127A1A700A
S3150800CB08174B1B78DBB2012B0FD01223FB7305E0FA
S3150800CB181323FB7302E01323FB7300BFFB7B1A4640
S3150800CB2800210020FFF760FE00E000BF1037BD4671
S3150800CB3880BD00BF600E0020B80E002060000020EF
S3150800CB48C20E0020044401082407002018440108DE
S3150800CB58D40100202C440108E80F002054000020C6
S3150800CB685C0E002080B500AF8F4B9A788F4B9A7071
S3150800CB788D4BD3F807308D4AC2F803308A4BB3F881
S3150800CB880F309AB2894BA3F80720874BB3F81B30A6
S3150800CB989AB2864BA3F80920834BB3F813309AB296
S3150800CBA8824BA3F80B20804BB3F815309AB27F4B0B
S3150800CBB8A3F80D207C4B1A7E7C4BDA737A4B5A7F86
S3150800CBC87A4B5A70784B5A78784B1A70774B0022FA
S3150800CBD81A7400225A74754B00229A74734B0022F1
S3150800CBE8DA7400221A750420FCF7CEFC034603F013
S3150800CBF80103D9B26D4A537D61F3000353750320C7
S3150800CC08FCF7C2FC034603F00103D9B2674A537D11
S3150800CC1861F3410353750020FCF7B6FC034603F09D
S3150800CC280103D9B2614A537D61F3820353755F4A9A
S3150800CC38537D23F0080353750320FCF7B5FC034618
S3150800CC48002B0CBF01230023D9B2584A537D61F340
S3150800CC5804135375FDF798FB0346002B14BF0123ED
S3150800CC680023D9B2514A537D61F3451353754F4A88
S3150800CC78537D23F0400353754D4B1B7A03F001038C
S3150800CC88D9B24A4A537D61F3C71353750020FCF796
S3150800CC987DFD03465AB2454B5A760120FCF776FDC8
S3150800CCA803465AB2414B9A76414BDB695AB23F4B17
S3150800CCB8DA763E4B00221A773C4B00225A773B4BD2
S3150800CCC800229A770022DA77384B002283F8202048
S3150800CCD8384B9B689AB2354BA3F82120354BDB684D
S3150800CCE89AB2324BA3F82320324B1B699AB22F4BC0
S3150800CCF8A3F82520112200212F4806F0ABF92B4B63
S3150800CD08002283F83820294B002283F8392000228C
S3150800CD1883F83A20254B002283F83B20002283F823
S3150800CD283C2004220021254806F094F91F4B0022CE
S3150800CD3883F84120002283F84220002283F8432002
S3150800CD48002283F84420194B002283F84720174B02
S3150800CD58002283F84620154B002283F84520134BFA
S3150800CD68002283F84820002283F849200F4B002226
S3150800CD7883F84A2008220021114806F06BF90B4B64
S3150800CD88002283F85320094B002283F854200022F6
S3150800CD9883F85520054B002283F85620002283F88D
S3150800CDA8572000BF80BD00BFD4010020600E0020B8
S3150800CDB824070020F8060020870E00209D0E002074
S3150800CDC8AB0E002080B485B000AF78607B68002B76
S3150800CDD818D07B6800221A607B6800229A807B68D4
S3150800CDE80022DA800023FB8108E0FA897B68023290
S3150800CDF8002143F82210FB890133FB81FB89072BA5
S3150800CE08F3D900E000BF1437BD4680BC704780B42C
S3150800CE1885B000AF786039607B68002B01D13B6824
S3150800CE2856E07B68DB88072B27D87B689B881A46D9
S3150800CE387B680232396843F822107B681A683B68AF
S3150800CE481A447B681A607B689B8801339AB27B68A8
S3150800CE589A807B689B88072B02D97B6800229A8070
S3150800CE687B68DB8801339AB27B68DA807B681B6843
S3150800CE787A68D28893FBF2F32AE07B689B881A467D
S3150800CE887B68023253F82230FB607B689B881A4617
S3150800CE987B680232396843F822107B681A68396851
S3150800CEA8FB68CB1A1A447B681A607B689B8801332F
S3150800CEB89AB27B689A807B689B88072B02D97B681D
S3150800CEC800229A807B681B68002B00DA0733DB1080
S3150800CED818461437BD4680BC7047000080B485B034
S3150800CEE800AF154B9B69144A43F001039361124B33
S3150800CEF89B6903F00103BB60BB680F4BDB690E4AED
S3150800CF0843F08053D3610C4BDB6903F080537B6095
S3150800CF187B680A4B5B68FB60FB6823F0E063FB6091
S3150800CF28FB6843F00073FB60044AFB68536000BF64
S3150800CF381437BD4680BC7047001002400000014007
S3150800CF4880B400AF00BFFDE780B400AF00BFFDE7BF
S3150800CF5880B400AF00BFFDE780B400AF00BFFDE7AF
S3150800CF6880B400AF00BFFDE780B400AF00BFBD4680
S3150800CF7880BC704780B400AF00BFBD4680BC704710
S3150800CF8880B400AF00BFBD4680BC704780B500AF0F
S3150800CF9800F0DCFC00BF80BD80B500AF024801F098
S3150800CFA8CDFE00BF80BD00BF8001002080B500AF60
S3150800CFB8024804F0C3F800BF80BD00BFC80E0020B1
S3150800CFC880B500AF024805F00BF900BF80BD00BF69
S3150800CFD8A00F002080B500AF024805F001F900BF90
S3150800CFE880BD00BFE80F002080B500AF024805F0F5
S3150800CFF8F7F800BF80BD00BF3010002080B500AF2D
S3150800D008024805F0EDF800BF80BD00BF580F0020A4
S3150800D01880B500AF024801F091FE00BF80BD00BF91
S3150800D028A801002080B500AF024801F087FE00BFBE
S3150800D03880BD00BFA801002080B586B000AFF860A3
S3150800D048B9607A6000237B610AE0AFF30080014685
S3150800D058BB685A1CBA60CAB21A707B6901337B610D
S3150800D0687A697B689A42F0DB7B6818461837BD46AA
S3150800D07880BD80B483B000AF78604FF0FF331846A0
S3150800D0880C37BD4680BC704780B483B000AF786063
S3150800D09839603B684FF400525A60002318460C372B
S3150800D0A8BD4680BC704780B483B000AF7860012362
S3150800D0B818460C37BD4680BC704780B485B000AFAB
S3150800D0C8F860B9607A60002318461437BD4680BCF4
S3150800D0D87047000080B586B000AF7860144A154BD3
S3150800D0E8D31A7B617B693B61134B1B68002B02D102
S3150800D0F8114B124A1A60104B1A687B6813443A692E
S3150800D1089A4207D205F0F4FF03460C221A604FF03C
S3150800D118FF3309E0084B1B68FB60074B1A687B68F6
S3150800D1281344054A1360FB6818461837BD4680BD80
S3150800D1380000012000040000C40E0020C8110020C9
S3150800D14880B400AF00BFBD4680BC704780B58EB0BE
S3150800D15800AF07F1280300221A605A609A60DA605D
S3150800D16807F1200300221A605A603B1D00221A6044
S3150800D1785A609A60DA601A615A619A612C4B2D4A8C
S3150800D1881A602B4B00225A60294B00229A60284BBA
S3150800D1984FF6FF72DA60264B00221A61244B0022EA
S3150800D1A89A61234803F083FD0346002B01D0FDF757
S3150800D1B821FC4FF48053BB6207F1280319461C4823
S3150800D1C804F06EF90346002B01D0FDF713FC184846
S3150800D1D803F0B2FE0346002B01D0FDF70BFC002333
S3150800D1E83B6200237B6207F120031946104804F0C6
S3150800D1F8FDFC0346002B01D0FDF7FCFB60237B6092
S3150800D2080023BB600023FB6000237B613B1D0422CF
S3150800D2181946074804F082F80346002B01D0FDF7A3
S3150800D228E9FB034800F0CEF800BF3837BD4680BD95
S3150800D238C80E00200004004080B58EB000AF07F184
S3150800D248280300221A605A609A60DA6007F12003F8
S3150800D25800221A605A603B1D00221A605A609A60BA
S3150800D268DA601A615A619A61374B384A1A60364B3E
S3150800D2784FF434725A60344B00229A60324B642257
S3150800D288DA60314B00221A612F4B00229A612E4828
S3150800D29803F00DFD0346002B01D0FDF7ABFB4FF459
S3150800D2A88053BB6207F128031946274804F0F8F8A3
S3150800D2B80346002B01D0FDF79DFB234803F03CFEEF
S3150800D2C80346002B01D0FDF795FB00233B6200239C
S3150800D2D87B6207F1200319461B4804F087FC0346BE
S3150800D2E8002B01D0FDF786FB60237B600023BB601B
S3150800D2F80023FB6000237B613B1D04221946124864
S3150800D30804F00CF80346002B01D0FDF773FB3B1D10
S3150800D318082219460C4804F001F80346002B01D0E8
S3150800D328FDF768FB3B1D0C221946074803F0F6FF74
S3150800D3380346002B01D0FDF75DFB034800F042F8D1
S3150800D34800BF3837BD4680BD100F002000080040D2
S3150800D35880B584B000AF78607B681B68164A93422C
S3150800D36814D1164BDB69154A43F00203D361134BF4
S3150800D378DB6903F00203FB60FB68002200211D201D
S3150800D38801F0D7FF1D2001F0F0FF10E07B681B684D
S3150800D3980B4A93420BD1094BDB69084A43F004034D
S3150800D3A8D361064BDB6903F00403BB60BB6800BFA7
S3150800D3B81037BD4680BD00BF00040040001002407B
S3150800D3C80008004080B58AB000AF786007F11403FA
S3150800D3D800221A605A609A60DA607B681B68264AD7
S3150800D3E8934218D1254B9B69244A43F00403936159
S3150800D3F8224B9B6903F004033B613B6980237B61ED
S3150800D4080223BB6102233B6207F1140319461C4831
S3150800D41802F024F92BE07B681B681A4A934226D146
S3150800D428164B9B69154A43F020039361134B9B6976
S3150800D43803F02003FB60FB684FF460437B6102231B
S3150800D448BB6102233B6207F1140319460E4802F032
S3150800D45805F90E4B5B687B627B6A43F0E0637B6287
S3150800D4687B6A43F480537B62084A7B6A536000BF31
S3150800D4782837BD4680BD00BF0004004000100240A2
S3150800D488000801400008004000140140000001405F
S3150800D49880B500AF114B124A1A60104B4FF416525A
S3150800D4A85A600E4B00229A600C4B0022DA600B4B2E
S3150800D4B800221A61094B0C225A61084B00229A610C
S3150800D4C8064B0022DA61054804F008FC0346002BDF
S3150800D4D801D0FDF78FFA00BF80BD00BF580F0020A6
S3150800D4E80050004080B500AF114B124A1A60104B25
S3150800D4F84FF4E1325A600E4B00229A600C4B002218
S3150800D508DA600B4B00221A61094B0C225A61084B48
S3150800D51800229A61064B0022DA61054804F0DEFB10
S3150800D5280346002B01D0FDF765FA00BF80BD00BF92
S3150800D538A00F00200038014080B500AF114B124AF1
S3150800D5481A60104B4FF4E1325A600E4B00229A606B
S3150800D5580C4B0022DA600B4B00221A61094B0C228D
S3150800D5685A61084B00229A61064B0022DA6105487F
S3150800D57804F0B4FB0346002B01D0FDF73BFA00BFC5
S3150800D58880BD00BFE80F00200044004080B500AF0A
S3150800D598114B124A1A60104B4FF4E1325A600E4B7F
S3150800D5A800229A600C4B0022DA600B4B00221A61A3
S3150800D5B8094B0C225A61084B00229A61064B002235
S3150800D5C8DA61054804F08AFB0346002B01D0FDF70B
S3150800D5D811FA00BF80BD00BF301000200048004087
S3150800D5E880B592B000AF786007F1300300221A6060
S3150800D5F85A609A60DA607B681B68954A934245D1F7
S3150800D608944BDB69934A43F48013D361914BDB69E6
S3150800D61803F48013FB62FB6A8E4B9B698D4A43F0C1
S3150800D628100393618B4B9B6903F01003BB62BB6ABB
S3150800D638884B9B69874A43F020039361854B9B690E
S3150800D64803F020037B627B6A4FF480533B63022313
S3150800D6587B630323FB6307F1300319467E4801F011
S3150800D668FDFF04233B6300237B630023BB6307F1A9
S3150800D67830031946794801F0F1FF002200213520C8
S3150800D68801F057FE352001F070FEDCE07B681B6868
S3150800D698734A93423AD16F4B9B696E4A43F4804367
S3150800D6A893616C4B9B6903F480433B623B6A694B05
S3150800D6B89B69684A43F004039361664B9B6903F0C8
S3150800D6C80403FB61FB694FF400733B6302237B6326
S3150800D6D80323FB6307F130031946624801F0BEFFCE
S3150800D6E84FF480633B6300237B630023BB6307F126
S3150800D6F8300319465B4801F0B1FF002200212520B6
S3150800D70801F017FE252001F030FE9CE07B681B68B7
S3150800D718554A934246D14F4BDB694E4A43F4003388
S3150800D728D3614C4BDB6903F40033BB61BB69494BD6
S3150800D7389B69484A43F020039361464B9B6903F06B
S3150800D74820037B617B6920233B6302237B630323D6
S3150800D758FB6307F130031946404801F07FFF402371
S3150800D7683B6300237B630023BB6307F13003194639
S3150800D7783A4801F073FF3D4B5B683B643B6C43F0EA
S3150800D788E0633B643B6C43F008033B64374A3B6CF5
S3150800D798536000220021262001F0CBFD262001F047
S3150800D7A8E4FD50E07B681B68314A93424BD1294B0C
S3150800D7B8DB69284A43F48023D361264BDB6903F4E3
S3150800D7C880233B613B69234B9B69224A43F010033C
S3150800D7D89361204B9B6903F01003FB60FB684FF4C9
S3150800D7E880633B6302237B630323FB6307F13003F0
S3150800D7F81946194801F032FF4FF400633B630023CA
S3150800D8087B630023BB6307F130031946124801F00E
S3150800D81825FF164B5B687B647B6C23F030037B64BF
S3150800D8287B6C43F0E0637B647B6C43F010037B649A
S3150800D8380E4A7B6C536000220021272001F079FDEF
S3150800D848272001F092FD00BF4837BD4680BD00BFBE
S3150800D858005000400010024000100140001401402A
S3150800D868003801400008014000440040000001401B
S3150800D87800480040FFF764FC0B480C490C4A002393
S3150800D88802E0D458C4500433C4188C42F9D3094A60
S3150800D898094C002301E013600432A242FBD305F0C9
S3150800D8A82DFCFCF7BBFF704700000020D4000020C1
S3150800D8B8DC440108D8000020C8110020FEE7000053
S3150800D8C880B500AF084B1B68074A43F0100313607E
S3150800D8D8032001F023FD0F2000F008F8FFF7FEFAF1
S3150800D8E80023184680BD00BF0020024080B582B0DC
S3150800D8F800AF7860124B1A68124B1B7819464FF41A
S3150800D9087A73B3FBF1F3B2FBF3F3184601F03BFD68
S3150800D9180346002B01D001230EE07B680F2B0AD89B
S3150800D928002279684FF0FF3001F003FD064A7B684C
S3150800D9381360002300E0012318460837BD4680BD5A
S3150800D9486C000020740000207000002080B400AF2E
S3150800D958054B1B781A46054B1B681344034A136084
S3150800D96800BFBD4680BC70477400002078100020B0
S3150800D97880B400AF024B1B681846BD4680BC70478A
S3150800D9887810002080B584B000AF7860FFF7F0FF04
S3150800D998B8607B68FB60FB68B3F1FF3F05D00A4BAC
S3150800D9A81B781A46FB681344FB6000BFFFF7E0FFC5
S3150800D9B80246BB68D31AFA689A42F7D800BF00BF6E
S3150800D9C81037BD4680BD00BF7400002080B586B0FC
S3150800D9D800AF78600023FB7500233B610023BB601A
S3150800D9E80023FB607B68002B01D10123BEE07B681E
S3150800D9F89B68002B7B689B6A002B09D17B680022F1
S3150800DA08DA627B68002283F824207868FBF7F8FC3A
S3150800DA18786800F0F1FB0346FB757B689B6A03F0A0
S3150800DA281003002B40F09980FB7D002B40F0958071
S3150800DA387B689B6A23F4885323F0020343F00202A7
S3150800DA487B689A627B685A687B68DB691A437B68D5
S3150800DA581B7B5B001343BA681343BB607B689B68F0
S3150800DA68B3F5807F03D07B689B68012B02D14FF4FE
S3150800DA78807300E000233A6913433B617B681B7D8A
S3150800DA88012B19D17B681B7B002B09D17B689B6905
S3150800DA98013B5A033B69134343F400633B610BE0BC
S3150800DAA87B689B6A43F020027B689A627B68DB6A1C
S3150800DAB843F001027B68DA627B681B685B6823F4BB
S3150800DAC869417B681B683A690A435A607B681B6820
S3150800DAD89A68284B13407A681268B9680B439360AA
S3150800DAE87B689B68B3F5807F03D07B689B68012BAE
S3150800DAF804D17B681B69013B1B05FB607B681B68B7
S3150800DB08DB6A23F470017B681B68FA680A43DA62E1
S3150800DB187B681B689A68184B1340BA689A420BD1F7
S3150800DB287B680022DA627B689B6A23F0030343F06A
S3150800DB3801027B689A6218E07B689B6A23F01203E5
S3150800DB4843F010027B689A627B68DB6A43F001023D
S3150800DB587B68DA620123FB7507E07B689B6A43F0FA
S3150800DB6810027B689A620123FB75FB7D18461837F5
S3150800DB78BD4680BDFDF7E1FFFE0E1FFF80B584B0E8
S3150800DB8800AF78600023FB737B6893F82430012B79
S3150800DB9801D1022398E07B68012283F8242078685B
S3150800DBA800F0D0FA0346FB73FB7B002B40F0878016
S3150800DBB87B689B6A23F4407323F0010343F480725D
S3150800DBC87B689A627B681B68414A934205D1414B38
S3150800DBD85B6803F47023002B15D17B689B6A23F4D2
S3150800DBE880127B689A627B681B685B6803F48063AB
S3150800DBF8002B26D07B689B6A23F4405343F4805253
S3150800DC087B689A621DE07B689B6A43F480127B688E
S3150800DC189A627B681B682F4A934204D07B681B6804
S3150800DC282B4A93420DD12B4B5B6803F48063002B78
S3150800DC3807D07B689B6A23F4405343F480527B6879
S3150800DC489A627B689B6A03F48053002B06D07B682C
S3150800DC58DB6A23F006027B68DA6202E07B68002248
S3150800DC68DA627B68002283F824207B681B686FF0D9
S3150800DC7802021A607B681B689B6803F46023B3F585
S3150800DC88602F13D17B681B68114A934205D1114B43
S3150800DC985B6803F47023002B08D17B681B689A68B5
S3150800DCA87B681B6842F4A0029A600CE07B681B68D4
S3150800DCB89A687B681B6842F480129A6003E07B685E
S3150800DCC8002283F82420FB7B18461037BD4680BD02
S3150800DCD8002801400024014080B584B000AF786070
S3150800DCE80023FB737B6893F82430012B01D10223A8
S3150800DCF81AE07B68012283F82420786800F07CFA09
S3150800DD080346FB73FB7B002B09D17B689B6A23F4CC
S3150800DD18885323F0010343F001027B689A627B6803
S3150800DD28002283F82420FB7B18461037BD4680BDA1
S3150800DD3890B587B000AF7860396000237B6100230F
S3150800DD48FB6000233B61FFF713FE78617B681B685D
S3150800DD589B6803F48073002B0BD07B689B6A43F09F
S3150800DD6820027B689A627B68002283F824200123B4
S3150800DD78D3E07B681B685B6803F48073002B31D19A
S3150800DD887B681B68DB6A03F47003002B2AD121E041
S3150800DD983B68B3F1FF3F1DD03B68002B07D0FFF760
S3150800DDA8E7FD02467B69D31A3A689A4212D27B681B
S3150800DDB81B681B6803F00203002B0BD17B689B6A60
S3150800DDC843F004027B689A627B68002283F8242061
S3150800DDD80323A2E07B681B681B6803F00203002B79
S3150800DDE8D6D070E04F4B1C68022002F005FD0346AA
S3150800DDF8B4FBF3F27B681B6819694B4B0B40002B85
S3150800DE0818D17B681B68D968484B0B40002B11D181
S3150800DE187B681B681969464B0B40002B08D17B6841
S3150800DE281B68D968434B0B40002B01D1142320E00B
S3150800DE3829231EE07B681B6819693D4B0B40002B9C
S3150800DE4806D17B681B68D9683A4B0B40002B0DD066
S3150800DE587B681B681969384B0B40002B08D17B680F
S3150800DE681B68D968344B0B40002B01D1542300E0BA
S3150800DE78FC2302FB03F33B6121E03B68B3F1FF3F58
S3150800DE881AD03B68002B07D0FFF772FD02467B695C
S3150800DE98D31A3A689A420FD2FB683A699A420BD95A
S3150800DEA87B689B6A43F004027B689A627B68002257
S3150800DEB883F82420032330E0FB680133FB60FB6802
S3150800DEC83A699A42D9D87B681B686FF012021A60B9
S3150800DED87B689B6A43F400727B689A627B681B6856
S3150800DEE89B6803F46023B3F5602F15D17B681B7B09
S3150800DEF8002B11D17B689B6A23F480727B689A622F
S3150800DF087B689B6A03F48053002B05D17B689B6A60
S3150800DF1843F001027B689A62002318461C37BD46FF
S3150800DF2890BD00BF6C000020244992242449920021
S3150800DF3892244912922449004992240080B483B055
S3150800DF4800AF78607B681B68DB6C18460C37BD46E3
S3150800DF5880BC704780B485B000AF7860396000230C
S3150800DF68FB730023BB607B6893F82430012B01D12F
S3150800DF780223DCE07B68012283F824203B685B687F
S3150800DF88062B1CD87B681B68596B3B685A6813466E
S3150800DF989B001344053B1F2202FA03F3DB4319408F
S3150800DFA83B6818683B685A6813469B001344053B48
S3150800DFB800FA03F27B681B680A435A633CE03B682D
S3150800DFC85B680C2B1CD87B681B68196B3B685A68FE
S3150800DFD813469B001344233B1F2202FA03F3DB4331
S3150800DFE819403B6818683B685A6813469B001344EF
S3150800DFF8233B00FA03F27B681B680A431A631BE093
S3150800E0087B681B68D96A3B685A6813469B001344A1
S3150800E018413B1F2202FA03F3DB4319403B681868A1
S3150800E0283B685A6813469B001344413B00FA03F2BF
S3150800E0387B681B680A43DA623B681B68092B1CD98C
S3150800E0487B681B68D9683B681A6813465B001344E3
S3150800E0581E3B072202FA03F3DB4319403B6898681C
S3150800E0683B681A6813465B0013441E3B00FA03F222
S3150800E0787B681B680A43DA6019E07B681B681969BC
S3150800E0883B681A6813465B001344072202FA03F32F
S3150800E098DB4319403B6898683B681A6813465B0077
S3150800E0A8134400FA03F27B681B680A431A613B6843
S3150800E0B81B68102B03D03B681B68112B32D17B6871
S3150800E0C81B681D4A934225D17B681B689B6803F425
S3150800E0D80003002B26D17B681B689A687B681B6837
S3150800E0E842F400029A603B681B68102B1AD1134B3E
S3150800E0F81B68134AA2FB03239A0C13469B00134476
S3150800E1085B00BB6002E0BB68013BBB60BB68002BD9
S3150800E118F9D107E07B689B6A43F020027B689A621C
S3150800E1280123FB737B68002283F82420FB7B1846AF
S3150800E1381437BD4680BC7047002401406C00002097
S3150800E14883DE1B4380B584B000AF78600023FB608C
S3150800E1580023BB607B681B689B6803F00103012BDF
S3150800E16840D07B681B689A687B681B6842F0010286
S3150800E1789A601F4B1B681F4AA2FB03239B0CBB60B4
S3150800E18802E0BB68013BBB60BB68002BF9D1FFF70F
S3150800E198EFFBF8601FE0FFF7EBFB0246FB68D31AB4
S3150800E1A8022B18D97B681B689B6803F00103012BAF
S3150800E1B811D07B689B6A43F010027B689A627B6879
S3150800E1C8DB6A43F001027B68DA627B68002283F81F
S3150800E1D82420012307E07B681B689B6803F001037A
S3150800E1E8012BD8D1002318461037BD4680BD00BF7D
S3150800E1F86C00002083DE1B4380B584B000AF7860CE
S3150800E2080023FB607B681B689B6803F00103012BEE
S3150800E2182ED17B681B689A687B681B6822F0010206
S3150800E2289A60FFF7A5FBF8601BE0FFF7A1FB02461B
S3150800E238FB68D31A022B14D97B681B689B6803F002
S3150800E2480103012B0DD17B689B6A43F010027B689A
S3150800E2589A627B68DB6A43F001027B68DA6201230B
S3150800E26807E07B681B689B6803F00103012BDCD079
S3150800E278002318461037BD4680BD000090B587B004
S3150800E28800AF78600023FB750023FB607B6893F872
S3150800E2982430012B01D1022397E07B68012283F8F9
S3150800E2A824207868FFF7A8FF0346FB757868FFF708
S3150800E2B849FF0346FB75FB7D002B40F081807B6890
S3150800E2C89B6A23F4885323F0020343F002027B680F
S3150800E2D89A62404B1C68022002F08EFA0346B4FB89
S3150800E2E8F3F35B00FB6002E0FB68013BFB60FB683D
S3150800E2F8002BF9D17B681B689A687B681B6842F013
S3150800E30808029A60FFF734FB38611BE0FFF730FB19
S3150800E31802463B69D31A0A2B14D97B681B689B6883
S3150800E32803F00803002B0DD07B689B6A23F01203C1
S3150800E33843F010027B689A627B68002283F82420DF
S3150800E348012342E07B681B689B6803F00803002BDF
S3150800E358DCD17B681B689A687B681B6842F00402F4
S3150800E3689A60FFF705FB38611BE0FFF701FB0246D9
S3150800E3783B69D31A0A2B14D97B681B689B6803F078
S3150800E3880403002B0DD07B689B6A23F0120343F025
S3150800E39810027B689A627B68002283F8242001238E
S3150800E3A813E07B681B689B6803F00403002BDCD129
S3150800E3B87B689B6A23F0030343F001027B689A6231
S3150800E3C87B68002283F82420FB7D18461C37BD4647
S3150800E3D890BD00BF6C00002080B584B000AF78609F
S3150800E3E87B68002B01D10123EDE07B6893F8203088
S3150800E3F8DBB2002B02D17868FBF7FCFA7B681B684E
S3150800E4081A687B681B6842F001021A60FFF7B0FABF
S3150800E418F86012E0FFF7ACFA0246FB68D31A0A2B33
S3150800E4280BD97B685B6A43F400327B685A627B685F
S3150800E438052283F820200123C5E07B681B685B68F2
S3150800E44803F00103002BE5D07B681B681A687B6814
S3150800E4581B6822F002021A60FFF78AFAF86012E0CF
S3150800E468FFF786FA0246FB68D31A0A2B0BD97B688C
S3150800E4785B6A43F400327B685A627B68052283F834
S3150800E488202001239FE07B681B685B6803F0020372
S3150800E498002BE5D17B681B7E012B08D17B681B689E
S3150800E4A81A687B681B6842F080021A6007E07B6876
S3150800E4B81B681A687B681B6822F080021A607B68EA
S3150800E4C85B7E012B08D17B681B681A687B681B680A
S3150800E4D842F040021A6007E07B681B681A687B6886
S3150800E4E81B6822F040021A607B689B7E012B08D1C4
S3150800E4F87B681B681A687B681B6842F020021A60EA
S3150800E50807E07B681B681A687B681B6822F020028C
S3150800E5181A607B68DB7E012B08D17B681B681A6842
S3150800E5287B681B6822F010021A6007E07B681B6884
S3150800E5381A687B681B6842F010021A607B681B7FA2
S3150800E548012B08D17B681B681A687B681B6842F030
S3150800E55808021A6007E07B681B681A687B681B68EC
S3150800E56822F008021A607B685B7F012B08D17B685A
S3150800E5781B681A687B681B6842F004021A6007E081
S3150800E5887B681B681A687B681B6822F004021A6095
S3150800E5987B689A687B68DB681A437B681B691A4339
S3150800E5A87B685B6942EA03017B685B685A1E7B687D
S3150800E5B81B680A43DA617B6800225A627B68012273
S3150800E5C883F82020002318461037BD4680BD000072
S3150800E5D880B487B000AF786039607B681B687B6158
S3150800E5E87B6893F82030FB74FB7C012B03D0FB7CFB
S3150800E5F8022B40F0BE80654B7B617B69D3F80032FD
S3150800E60843F001027B69C3F800227B69D3F800321C
S3150800E61823F47C527B69C3F800227B69D3F800226D
S3150800E6283B685B6A1B021A437B69C3F800223B688E
S3150800E6385B6903F01F03012202FA03F3FB607B6997
S3150800E648D3F81C22FB68DB431A407B69C3F81C22F3
S3150800E6583B68DB69002B23D17B69D3F80C22FB685E
S3150800E668DB431A407B69C3F80C223B68DB6819044C
S3150800E6783B685B689BB23A68526919437B694832BA
S3150800E68843F832103B689B6819043B681B689AB2C2
S3150800E6983B685B690A4379694833DB000B445A606F
S3150800E6A83B68DB69012B22D17B69D3F80C22FB680E
S3150800E6B81A437B69C3F80C223B681B6819043B6834
S3150800E6C85B689BB23A68526919437B69483243F8D2
S3150800E6D832103B689B6819043B68DB689AB23B684A
S3150800E6E85B690A4379694833DB000B445A603B681F
S3150800E6F89B69002B09D17B69D3F80422FB68DB43A5
S3150800E7081A407B69C3F8042207E07B69D3F8042218
S3150800E718FB681A437B69C3F804223B681B69002B0C
S3150800E72809D17B69D3F81422FB68DB431A407B6955
S3150800E738C3F8142207E07B69D3F81422FB681A4346
S3150800E7487B69C3F814223B681B6A012B07D17B69CE
S3150800E758D3F81C22FB681A437B69C3F81C227B6919
S3150800E768D3F8003223F001027B69C3F8002200239C
S3150800E77806E07B685B6A43F480227B685A62012359
S3150800E78818461C37BD4680BC704700BF0064004069
S3150800E79880B584B000AF78607B6893F82030DBB228
S3150800E7A8012B2ED17B68022283F820207B681B6800
S3150800E7B81A687B681B6822F001021A60FFF7D8F806
S3150800E7C8F86012E0FFF7D4F80246FB68D31A0A2B5A
S3150800E7D80BD97B685B6A43F400327B685A627B68AC
S3150800E7E8052283F82020012312E07B681B685B68F2
S3150800E7F803F00103002BE5D17B6800225A62002347
S3150800E80806E07B685B6A43F400227B685A62012348
S3150800E81818461037BD4680BD80B584B000AF78600D
S3150800E8287B6893F82030DBB2022B33D17B681B68F0
S3150800E8381A687B681B6842F001021A60FFF798F8A5
S3150800E848F86012E0FFF794F80246FB68D31A0A2B19
S3150800E8580BD97B685B6A43F400327B685A627B682B
S3150800E868052283F8202001231BE07B681B685B6868
S3150800E87803F00103002BE5D07B681B681A687B68E0
S3150800E8881B6822F002021A607B68012283F820209E
S3150800E898002306E07B685B6A43F480127B685A6249
S3150800E8A8012318461037BD4680BD80B489B000AF2D
S3150800E8B8F860B9607A603B60FB6893F82030FB77AC
S3150800E8C8FB681B689B68BB61FB7F012B03D0FB7F3A
S3150800E8D8022B40F0AD80BB6903F08063002B0AD198
S3150800E8E8BB6903F00063002B05D1BB6903F08053AD
S3150800E8F8002B00F09580BB691B0E03F003037B61B0
S3150800E90801227B699A403B681A60BB689B68002BA2
S3150800E9180DD1BB681B685A05BB68DB68F9680968C6
S3150800E9281A437B6918331B010B441A600FE0BB684E
S3150800E9385B68DA00BB689B681A43BB68DB68F968DA
S3150800E94809681A437B6918331B010B441A60FB686C
S3150800E9581968BB681A697B6918331B010B440433A9
S3150800E9681A60BB681B7D012B11D1FB681A687B6985
S3150800E97818331B01134404331B68FA68116843F4F7
S3150800E98880727B6918331B010B4404331A607B6851
S3150800E99807331B781A067B6806331B781B041A4349
S3150800E9A87B6805331B781B0213437A68043212788E
S3150800E9B81046FA68116843EA00027B691B010B4492
S3150800E9C803F5C6731A607B6803331B781A067B68D7
S3150800E9D802331B781B041A437B6801331B781B0216
S3150800E9E813437A6812781046FA68116843EA0002EF
S3150800E9F87B691B010B4403F5C4731A60FB681A6824
S3150800EA087B6918331B0113441B68FA68116843F0BD
S3150800EA1801027B6918331B010B441A6000230EE0B8
S3150800EA28FB685B6A43F40012FB685A62012306E036
S3150800EA38FB685B6A43F48022FB685A62012318461E
S3150800EA482437BD4680BC704780B485B000AF78606F
S3150800EA580023FB607B6893F82030FB72FB7A012B56
S3150800EA6802D0FB7A022B1DD17B681B689B6803F0D2
S3150800EA788063002B02D0FB680133FB607B681B6848
S3150800EA889B6803F00063002B02D0FB680133FB6028
S3150800EA987B681B689B6803F08053002B02D0FB68D1
S3150800EAA80133FB60FB6818461437BD4680BC7047BF
S3150800EAB880B487B000AFF860B9607A603B60FB68DD
S3150800EAC893F82030FB75FB7D012B03D0FB7D022BC9
S3150800EAD840F00381BB68002B0ED1FB681B68DB6816
S3150800EAE803F00303002B16D1FB685B6A43F4001294
S3150800EAF8FB685A620123F7E0FB681B681B6903F089
S3150800EB080303002B07D1FB685B6A43F40012FB6812
S3150800EB185A620123E8E0FB681A68BB681B331B01C5
S3150800EB2813441B6803F004027B689A607B689B6839
S3150800EB38002B0CD1FB681A68BB681B331B011344EE
S3150800EB481B685B0DC3F30A027B681A600BE0FB6857
S3150800EB581A68BB681B331B0113441B68DB0823F0C0
S3150800EB6860427B685A60FB681A68BB681B331B01DE
S3150800EB7813441B6803F002027B68DA60FB681A68AC
S3150800EB88BB681B331B01134404331B6803F00803D3
S3150800EB98002B03D07B6808221A610BE0FB681A6809
S3150800EBA8BB681B331B01134404331B6803F00F02AD
S3150800EBB87B681A61FB681A68BB681B331B01134418
S3150800EBC804331B681B0ADAB27B689A61FB681A6801
S3150800EBD8BB681B331B01134404331B681B0C9AB20E
S3150800EBE87B685A61FB681A68BB681B01134403F5FE
S3150800EBF8DC731B68DAB23B681A70FB681A68BB686C
S3150800EC081B01134403F5DC731B681A0A3B680133B6
S3150800EC18D2B21A70FB681A68BB681B01134403F55D
S3150800EC28DC731B681A0C3B680233D2B21A70FB688D
S3150800EC381A68BB681B01134403F5DC731B681A0EB4
S3150800EC483B680333D2B21A70FB681A68BB681B01A3
S3150800EC58134403F5DE731A683B680433D2B21A7094
S3150800EC68FB681A68BB681B01134403F5DE731B6847
S3150800EC781A0A3B680533D2B21A70FB681A68BB6869
S3150800EC881B01134403F5DE731B681A0C3B6806332D
S3150800EC98D2B21A70FB681A68BB681B01134403F5DD
S3150800ECA8DE731B681A0E3B680733D2B21A70BB6844
S3150800ECB8002B08D1FB681B68DA68FB681B6842F0FA
S3150800ECC82002DA6007E0FB681B681A69FB681B689C
S3150800ECD842F020021A61002306E0FB685B6A43F4E7
S3150800ECE88022FB685A62012318461C37BD4680BC39
S3150800ECF8704780B485B000AF786039607B6893F850
S3150800ED082030FB73FB7B012B02D0FB7B022B09D13E
S3150800ED187B681B6859697B681B683A680A435A61A5
S3150800ED28002306E07B685B6A43F480227B685A62A4
S3150800ED38012318461437BD4680BC704780B58AB08B
S3150800ED4800AF786000237B627B681B685B693B625F
S3150800ED587B681B685B68FB617B681B689B68BB6193
S3150800ED687B681B68DB687B617B681B681B693B6182
S3150800ED787B681B689B69FB603B6A03F00103002BF1
S3150800ED887CD0BB6903F00103002B23D07B681B6882
S3150800ED9801229A60BB6903F00203002B03D0786846
S3150800EDA800F083F916E0BB6903F00403002B04D0CE
S3150800EDB87B6A43F400637B620CE0BB6903F00803D3
S3150800EDC8002B04D07B6A43F480537B6202E07868A0
S3150800EDD800F086F9BB6903F48073002B24D07B689E
S3150800EDE81B684FF480729A60BB6903F40073002BA2
S3150800EDF803D0786800F062F916E0BB6903F480630B
S3150800EE08002B04D07B6A43F400537B620CE0BB6991
S3150800EE1803F40063002B04D07B6A43F480437B62C7
S3150800EE2802E0786800F065F9BB6903F48033002BC3
S3150800EE3824D07B681B684FF480329A60BB6903F458
S3150800EE480033002B03D0786800F041F916E0BB6957
S3150800EE5803F48023002B04D07B6A43F400437B62C7
S3150800EE680CE0BB6903F40023002B04D07B6A43F447
S3150800EE7880337B6202E0786800F044F93B6A03F065
S3150800EE880803002B0CD07B6903F01003002B07D06E
S3150800EE987B6A43F400737B627B681B681022DA601E
S3150800EEA83B6A03F00403002B0BD07B6903F00803C5
S3150800EEB8002B06D07B681B680822DA60786800F0A1
S3150800EEC833F93B6A03F00203002B09D07B681B68F9
S3150800EED8DB6803F00303002B02D0786800F01BF9FF
S3150800EEE83B6A03F04003002B0CD03B6903F0100380
S3150800EEF8002B07D07B6A43F480637B627B681B68B8
S3150800EF0810221A613B6A03F02003002B0BD03B69D9
S3150800EF1803F00803002B06D07B681B6808221A61D1
S3150800EF28786800F00AF93B6A03F01003002B09D049
S3150800EF387B681B681B6903F00303002B02D07868FB
S3150800EF48FBF7E8FD3B6A03F40033002B0BD0FB699B
S3150800EF5803F01003002B06D07B681B6810225A6042
S3150800EF68786800F0F3F83B6A03F48033002B0BD07B
S3150800EF78FB6903F00803002B06D07B681B68082288
S3150800EF885A60786800F0EBF83B6A03F40043002BF4
S3150800EF987BD0FB6903F00403002B72D03B6A03F4A9
S3150800EFA88073002B08D0FB6803F00103002B03D0FD
S3150800EFB87B6A43F001037B623B6A03F40073002B08
S3150800EFC808D0FB6803F00203002B03D07B6A43F0E2
S3150800EFD802037B623B6A03F48063002B08D0FB6854
S3150800EFE803F00403002B03D07B6A43F004037B6217
S3150800EFF83B6A03F40063002B43D0FB6803F07003F5
S3150800F008002B3ED0FB6803F07003602B2BD0602BD7
S3150800F0182ED8502B22D0502B2AD8402B19D0402B2B
S3150800F02826D8302B10D0302B22D8102B02D0202BE4
S3150800F03805D01DE07B6A43F008037B6219E07B6A0A
S3150800F04843F010037B6214E07B6A43F020037B627B
S3150800F0580FE07B6A43F040037B620AE07B6A43F071
S3150800F06880037B6205E07B6A43F480737B6200E079
S3150800F07800BF7B681B689A697B681B6822F0700268
S3150800F0889A617B681B6804225A607B6A002B08D041
S3150800F0987B685A6A7B6A1A437B685A62786800F002
S3150800F0A867F800BF2837BD4680BD80B483B000AF77
S3150800F0B8786000BF0C37BD4680BC704780B483B003
S3150800F0C800AF786000BF0C37BD4680BC704780B477
S3150800F0D883B000AF786000BF0C37BD4680BC704768
S3150800F0E880B483B000AF786000BF0C37BD4680BCDB
S3150800F0F8704780B483B000AF786000BF0C37BD4650
S3150800F10880BC704780B483B000AF786000BF0C3706
S3150800F118BD4680BC704780B483B000AF786000BF36
S3150800F1280C37BD4680BC704780B483B000AF7860A2
S3150800F13800BF0C37BD4680BC704780B483B000AFAB
S3150800F148786000BF0C37BD4680BC704780B483B072
S3150800F15800AF786000BF0C37BD4680BC704780B4E6
S3150800F16883B000AF786000BF0C37BD4680BC7047D7
S3150800F17880B483B000AF786000BF0C37BD4680BC4A
S3150800F1887047000080B485B000AF78607B6803F0EC
S3150800F1980703FB600C4BDB68BB60BA684FF6FF03D6
S3150800F1A81340BB60FB681A02BB68134343F0BF638E
S3150800F1B843F40033BB60044ABB68D36000BF143706
S3150800F1C8BD4680BC704700BF00ED00E080B400AFC4
S3150800F1D8044BDB681B0A03F007031846BD4680BCC8
S3150800F1E8704700BF00ED00E080B483B000AF034667
S3150800F1F8FB7197F90730002B0BDBFB7903F01F022D
S3150800F208064997F907305B09012000FA02F241F826
S3150800F218232000BF0C37BD4680BC704700E100E0DC
S3150800F22880B483B000AF03463960FB7197F907309D
S3150800F238002B0ADB3B68DAB20C4997F9073012014A
S3150800F248D2B20B4483F800230AE03B68DAB20849CD
S3150800F258FB7903F00F03043B1201D2B20B441A766A
S3150800F26800BF0C37BD4680BC704700BF00E100E010
S3150800F27800ED00E080B489B000AFF860B9607A6044
S3150800F288FB6803F00703FB61FB69C3F10703042B5B
S3150800F29828BF0423BB61FB690433062B02D9FB6923
S3150800F2A8033B00E000237B614FF0FF32BB6902FA9B
S3150800F2B803F3DA43BB681A407B699A404FF0FF317B
S3150800F2C87B6901FA03F3D9437B680B401343184655
S3150800F2D82437BD4680BC704780B582B000AF7860D9
S3150800F2E87B68013BB3F1807F01D301230FE00A4A0B
S3150800F2F87B68013B53600F214FF0FF30FFF790FF03
S3150800F308054B00229A60044B07221A600023184608
S3150800F3180837BD4680BD00BF10E000E080B582B062
S3150800F32800AF78607868FFF72DFF00BF0837BD463D
S3150800F33880BD80B586B000AF0346B9607A60FB73B6
S3150800F34800237B61FFF742FF78617A68B9687869B4
S3150800F358FFF790FF024697F90F3011461846FFF750
S3150800F3685FFF00BF1837BD4680BD80B582B000AFC5
S3150800F3780346FB7197F907301846FFF735FF00BFB4
S3150800F3880837BD4680BD80B582B000AF786078681A
S3150800F398FFF7A2FF034618460837BD4680BD80B565
S3150800F3A882B000AF78607B68002B01D101230EE09C
S3150800F3B87B685B79DBB2002B05D17B6800221A7162
S3150800F3C87868FAF753FF7B6801225A7100231846B2
S3150800F3D80837BD4680BD80B485B000AF7860002385
S3150800F3E8FB737B6893F82130DBB2022B08D07B6865
S3150800F3F804229A637B68002283F82020012320E0F0
S3150800F4087B681B681A687B681B6822F00E021A60FC
S3150800F4187B681B681A687B681B6822F001021A60F9
S3150800F4287B681A6C7B68DB6B012101FA02F25A6069
S3150800F4387B68012283F821207B68002283F8202034
S3150800F448FB7B18461437BD4680BC704780B584B028
S3150800F45800AF78600023FB737B6893F82130DBB232
S3150800F468022B05D07B6804229A630123FB73D6E036
S3150800F4787B681B681A687B681B6822F00E021A608C
S3150800F4887B681B681A687B681B6822F001021A6089
S3150800F4987B681B681A46644B9A4258D97B681B686E
S3150800F4A8624A93424FD07B681B68614A934248D0A8
S3150800F4B87B681B685F4A934240D07B681B685E4A34
S3150800F4C8934238D07B681B685C4A934230D07B6885
S3150800F4D81B685B4A934228D07B681B68524A93424A
S3150800F4E820D07B681B68574A934219D07B681B68EB
S3150800F4F8554A934212D07B681B68544A93420AD0ED
S3150800F5087B681B68524A934202D14FF480531BE02A
S3150800F5184FF4803318E04FF4807315E0102313E096
S3150800F528012311E04FF080730EE04FF480130BE0CF
S3150800F5384FF4803308E04FF4805305E04FF48073A6
S3150800F54802E0102300E00123424A536057E07B6833
S3150800F5581B68364A93424FD07B681B68344A9342E5
S3150800F56848D07B681B68334A934240D07B681B683F
S3150800F578314A934238D07B681B68304A934230D068
S3150800F5887B681B682E4A934228D07B681B68264AE4
S3150800F598934220D07B681B682A4A934219D07B6815
S3150800F5A81B68294A934212D07B681B68274A9342EC
S3150800F5B80AD07B681B68264A934202D14FF48053C7
S3150800F5C81BE04FF4803318E04FF4807315E01023DE
S3150800F5D813E0012311E04FF080730EE04FF4801317
S3150800F5E80BE04FF4803308E04FF4805305E04FF4FE
S3150800F5F8807302E0102300E00123174A53607B68F2
S3150800F608012283F821207B68002283F820207B6862
S3150800F6185B6B002B03D07B685B6B78689847FB7B32
S3150800F62818461037BD4680BD8000024008000240D3
S3150800F6381C000240300002404400024058000240C4
S3150800F6486C000240080402401C04024030040240D0
S3150800F65844040240000402400000024080B48BB013
S3150800F66800AF7860396000237B6200233B6269E15A
S3150800F67801227B6A02FA03F3FB613B681B68FA6995
S3150800F6881340BB61BA69FB699A4240F058813B68E6
S3150800F6985B689A4A93425ED0984A934275D8984AC4
S3150800F6A8934258D0964A93426FD8964A934252D074
S3150800F6B8944A934269D8944A93424CD0924A9342C0
S3150800F6C863D8924A934246D0904A93425DD8122B01
S3150800F6D82AD8122B59D801A252F823F05FF7000846
S3150800F6E839F700084BF700088DF7000893F7000864
S3150800F6F893F7000893F7000893F7000893F70008AC
S3150800F70893F7000893F7000893F7000893F700089B
S3150800F71893F7000893F7000893F7000893F700088B
S3150800F72841F7000855F70008794A934213D02CE0A8
S3150800F7383B68DB683B6229E03B68DB6804333B626D
S3150800F74824E03B68DB6808333B621FE03B68DB68FC
S3150800F7580C333B621AE03B689B68002B02D10423F2
S3150800F7683B6213E03B689B68012B05D108233B6283
S3150800F7787B68FA691A6109E008233B627B68FA69BB
S3150800F7885A6103E000233B6200E000BFBB69FF2B18
S3150800F79801D87B6801E07B6804337B61BB69FF2B72
S3150800F7A802D87B6A9B0002E07B6A083B9B003B61A8
S3150800F7B87B691A680F213B6901FA03F3DB431A4090
S3150800F7C8396A3B6901FA03F31A437B691A603B688D
S3150800F7D85B6803F08053002B00F0B1804D4B9B69A2
S3150800F7E84C4A43F0010393614A4B9B6903F00103B2
S3150800F7F8BB60BB68484A7B6A9B08023352F82330C9
S3150800F808FB607B6A03F003039B000F2202FA03F3EB
S3150800F818DB43FA681340FB607B68404A934213D07F
S3150800F8287B683F4A93420DD07B683E4A934207D08D
S3150800F8387B683D4A934201D1032306E0042304E08A
S3150800F848022302E0012300E000237A6A02F0030299
S3150800F85892009340FA681343FB602F497B6A9B081A
S3150800F8680233FA6841F823203B685B6803F480137F
S3150800F878002B06D02D4B9A682C49BB6913438B601D
S3150800F88806E02A4B9A68BB69DB43284913408B6014
S3150800F8983B685B6803F40013002B06D0234BDA6831
S3150800F8A82249BB691343CB6006E0204BDA68BB697B
S3150800F8B8DB431E491340CB603B685B6803F400339F
S3150800F8C8002B06D0194B5A681849BB6913434B6075
S3150800F8D806E0164B5A68BB69DB43144913404B606C
S3150800F8E83B685B6803F48033002B21D00F4B1A68FA
S3150800F8F80E49BB6913430B6021E000BF00003210B4
S3150800F908000031100000221000002110000012101B
S3150800F91800001110001002400000014000080140D4
S3150800F928000C014000100140001401400004014089
S3150800F9380B4B1A68BB69DB43094913400B607B6AA2
S3150800F94801337B623B681A687B6A22FA03F3002B49
S3150800F9587FF48EAE00BF00BF2C37BD4680BC70470B
S3150800F9680004014080B485B000AF78600B467B8000
S3150800F9787B689A687B881340002B02D00123FB73A7
S3150800F98801E00023FB73FB7B18461437BD4680BC91
S3150800F998704780B483B000AF78600B467B80134607
S3150800F9A87B707B78002B03D07A887B681A6103E022
S3150800F9B87B881A047B681A6100BF0C37BD4680BC71
S3150800F9C87047000080B400AF034B01221A6000BFDD
S3150800F9D8BD4680BC704700BF20000E4280B582B085
S3150800F9E800AFFDF7C5FF7860604B1B685F4A43F0B8
S3150800F9F80103136008E0FDF7BBFF02467B68D31ACC
S3150800FA08022B01D90323ACE0584B1B6803F0020309
S3150800FA18002BF0D0554B1B6823F0F803534A43F0E4
S3150800FA2880031360FDF7A4FF7860504B00225A60E4
S3150800FA380AE0FDF79DFF02467B68D31A41F2883231
S3150800FA48934201D903238CE0484B5B6803F00C0307
S3150800FA58002BEED1464B474A1A60474B1B68184697
S3150800FA68FDF744FF0346002B01D0012379E0FDF793
S3150800FA787FFF78603D4B1B683C4A23F08073136010
S3150800FA8808E0FDF775FF02467B68D31A022B01D9F1
S3150800FA98032366E0354B1B6803F00073002BF0D18F
S3150800FAA8324B00225A60FDF763FF78602F4B1B68BC
S3150800FAB82E4A23F41023136008E0FDF759FF02467F
S3150800FAC87B68D31A642B01D903234AE0274B1B68A2
S3150800FAD803F40033002BF0D1244B1B68234A23F484
S3150800FAE880231360FDF744FF7860204B1B681F4A84
S3150800FAF823F08063136008E0FDF73AFF02467B6847
S3150800FB08D31A642B01D903232BE0184B1B6803F07F
S3150800FB180063002BF0D1FDF72BFF7860134B1B68A9
S3150800FB28124A23F08053136008E0FDF721FF0246C6
S3150800FB387B68D31A642B01D9032312E00B4B1B6885
S3150800FB4803F00053002BF0D1084B0022DA62074B6A
S3150800FB585B6A064A43F080735362044B00229A6034
S3150800FB68002318460837BD4680BD00BF001002406E
S3150800FB786C00002000127A007000002080B586B05C
S3150800FB8800AF78607B68002B01D1012304E37B680A
S3150800FB981B6803F00103002B00F08780924B5B6813
S3150800FBA803F00C03042B0CD08F4B5B6803F00C0393
S3150800FBB8082B12D18C4B5B6803F48033B3F5803F6E
S3150800FBC80BD1894B1B6803F40033002B6CD07B6878
S3150800FBD89B68002B68D10123DEE27B689B68B3F536
S3150800FBE8803F06D1804B1B687F4A43F480331360F5
S3150800FBF82EE07B689B68002B0CD17B4B1B687A4AE6
S3150800FC0823F480331360784B1B68774A23F48023E0
S3150800FC1813601DE07B689B68B3F5A02F0CD1724B67
S3150800FC281B68714A43F4802313606F4B1B686E4A3E
S3150800FC3843F4803313600BE06B4B1B686A4A23F462
S3150800FC4880331360684B1B68674A23F48023136064
S3150800FC587B689B68002B13D0FDF78AFE386108E09D
S3150800FC68FDF786FE02463B69D31A642B01D903239E
S3150800FC7892E25D4B1B6803F40033002BF0D014E0C6
S3150800FC88FDF776FE386108E0FDF772FE02463B6925
S3150800FC98D31A642B01D903237EE2534B1B6803F45A
S3150800FCA80033002BF0D100E000BF7B681B6803F027
S3150800FCB80203002B63D04C4B5B6803F00C03002B44
S3150800FCC80BD0494B5B6803F00C03082B1CD1464B39
S3150800FCD85B6803F48033002B16D1434B1B6803F08B
S3150800FCE80203002B05D07B685B69012B01D0012331
S3150800FCF852E23D4B1B6823F0F8027B689B69DB00E0
S3150800FD08394913430B603AE07B685B69002B20D0BE
S3150800FD18364B01221A60FDF72BFE386108E0FDF71D
S3150800FD2827FE02463B69D31A022B01D9032333E27D
S3150800FD382D4B1B6803F00203002BF0D02A4B1B68D7
S3150800FD4823F0F8027B689B69DB00274913430B609D
S3150800FD5815E0264B00221A60FDF70AFE386108E00E
S3150800FD68FDF706FE02463B69D31A022B01D903237F
S3150800FD7812E21D4B1B6803F00203002BF0D17B68C7
S3150800FD881B6803F00803002B3AD07B68DB69002B55
S3150800FD9819D0174B01221A60FDF7EAFD386108E009
S3150800FDA8FDF7E6FD02463B69D31A022B01D9032360
S3150800FDB8F2E10D4B5B6A03F00203002BF0D0012039
S3150800FDC800F0CAFB1CE00A4B00221A60FDF7D0FDBA
S3150800FDD838610FE0FDF7CCFD02463B69D31A022BC2
S3150800FDE808D90323D8E100BF0010024000004242A8
S3150800FDF8800442429B4B5B6A03F00203002BE9D15D
S3150800FE087B681B6803F00403002B00F0A680002318
S3150800FE18FB75944BDB6903F08053002B0DD1914B8E
S3150800FE28DB69904A43F08053D3618E4BDB6903F054
S3150800FE388053BB60BB680123FB758B4B1B6803F4B7
S3150800FE488073002B18D1884B1B68874A43F4807344
S3150800FE581360FDF78DFD386108E0FDF789FD024658
S3150800FE683B69D31A642B01D9032395E17E4B1B689A
S3150800FE7803F48073002BF0D07B681B69012B06D12D
S3150800FE88784B1B6A774A43F0010313622DE07B68B7
S3150800FE981B69002B0CD1734B1B6A724A23F00103AA
S3150800FEA81362704B1B6A6F4A23F0040313621CE043
S3150800FEB87B681B69052B0CD16A4B1B6A694A43F098
S3150800FEC804031362674B1B6A664A43F0010313620D
S3150800FED80BE0644B1B6A634A23F001031362614B08
S3150800FEE81B6A604A23F0040313627B681B69002BAC
S3150800FEF815D0FDF73DFD38610AE0FDF739FD0246E4
S3150800FF083B69D31A41F28832934201D9032343E164
S3150800FF18544B1B6A03F00203002BEED014E0FDF7DE
S3150800FF2827FD38610AE0FDF723FD02463B69D31A27
S3150800FF3841F28832934201D903232DE1494B1B6AC2
S3150800FF4803F00203002BEED1FB7D012B05D1454BAF
S3150800FF58DB69444A23F08053D3617B68DB6A002B4C
S3150800FF6800F08C803F4B5B6803F48033B3F5803F21
S3150800FF780ED13C4B5B6803F00C03082B08D1394BB0
S3150800FF88DB6A03F48033B3F5803F01D1012303E12B
S3150800FF987B68DB6A022B4ED1324B1B6803F0805311
S3150800FFA8002B09D02F4BDB6A03F0F0027B685B6BEA
S3150800FFB89A4201D00123EFE02C4B00221A60FDF784
S3150800FFC8D7FC386108E0FDF7D3FC02463B69D31A2B
S3150800FFD8642B01D90323DFE0224B1B6803F0006377
S3150800FFE8002BF0D11F4BDB6A23F0F0027B685B6BB2
S3150800FFF81C491343CB621B4BDB6A23F470627B688C
S315080100081B6B18491343CB62184B01221A60FDF77B
S31508010018AFFC386108E0FDF7ABFC02463B69D31A29
S31508010028642B01D90323B7E00E4B1B6803F0006361
S31508010038002BF0D022E00B4BDB6A0A4A23F4803303
S31508010048D3620A4B00221A60FDF792FC38610FE069
S31508010058FDF78EFC02463B69D31A642B08D903239C
S315080100689AE000BF00100240007000406800424252
S315080100784B4B1B6803F00063002BE9D17B681B6AAD
S31508010088002B00F08880464B5B6803F00C03082BAD
S3150801009868D07B681B6A022B4DD1424B00221A6035
S315080100A8FDF766FC386108E0FDF762FC02463B6924
S315080100B8D31A022B01D903236EE0394B1B6803F0C7
S315080100C80073002BF0D17B685B6AB3F5803F0FD1CB
S315080100D8334BDA6A7B685B6831491343CB62304B29
S315080100E8DB6A23F00F027B68DB682D491343CB6271
S315080100F82B4B5B6823F474127B68596A7B689B6A85
S315080101080B43274913434B60264B01221A60FDF717
S315080101182FFC386108E0FDF72BFC02463B69D31A28
S31508010128022B01D9032337E01D4B1B6803F0007323
S31508010138002BF0D02FE01B4B00221A60FDF718FCA4
S31508010148386108E0FDF714FC02463B69D31A022B0D
S3150801015801D9032320E0124B1B6803F00073002B17
S31508010168F0D118E07B681B6A012B01D1012313E042
S315080101780B4B5B68FB60FB6803F480327B685B6A40
S315080101889A4206D1FB6803F470127B689B6A9A4205
S3150801019801D0012300E0002318461837BD4680BD63
S315080101A8001002406000424280B584B000AF786012
S315080101B839607B68002B01D10123D0E06A4B1B68A3
S315080101C803F007033A689A4210D9674B1B6823F06C
S315080101D8070265493B6813430B60634B1B6803F0C9
S315080101E807033A689A4201D00123B8E07B681B687D
S315080101F803F00203002B20D07B681B6803F0040375
S31508010208002B05D0594B5B68584A43F4E0635360A1
S315080102187B681B6803F00803002B05D0534B5B6802
S31508010228524A43F460535360504B5B6823F0F0021B
S315080102387B689B684D4913434B607B681B6803F0D1
S315080102480103002B40D07B685B68012B07D1474B1C
S315080102581B6803F40033002B15D101237FE07B6863
S315080102685B68022B07D1414B1B6803F00073002B0F
S3150801027809D1012373E03D4B1B6803F00203002BE8
S3150801028801D101236BE0394B5B6823F003027B68D4
S315080102985B68364913434B60FDF76AFBF8600AE069
S315080102A8FDF766FB0246FB68D31A41F28832934288
S315080102B801D9032353E02D4B5B6803F00C027B68D5
S315080102C85B689B009A42EBD1274B1B6803F007032F
S315080102D83A689A4210D2244B1B6823F0070222492E
S315080102E83B6813430B60204B1B6803F007033A6806
S315080102F89A4201D0012332E07B681B6803F00403A4
S31508010308002B08D0194B5B6823F4E0627B68DB682D
S31508010318164913434B607B681B6803F00803002BD7
S3150801032809D0124B5B6823F460527B681B69DB00B2
S315080103380E4913434B6000F021F802460B4B5B68E4
S315080103481B0903F00F030A49CB5C22FA03F3094A8E
S315080103581360094B1B681846FDF7C8FA00231846A7
S315080103681037BD4680BD00BF00200240001002407C
S31508010378404401086C000020700000202DE9B04FA8
S315080103888EB000AF0023FB620023BB6200237B63A8
S3150801039800237B6200233B6300233B620023FB6146
S315080103A84E4B5B68FB62FB6A03F00C03042B02D015
S315080103B8082B03D089E04A4B3B6389E0FB6A9B0C0F
S315080103C803F00F02474B9B5C7B62FB6A03F480339D
S315080103D8002B72D0414BDB6A03F00F02424B9B5C40
S315080103E8BB623E4BDB6A03F48033002B53D03B4B8D
S315080103F8DB6A1B0903F00F0301333B62374BDB6AE0
S315080104081B0A03F00F030233FB61FB6900229A46B4
S3150801041893467B6A00223B617A613B6903FB0BF2CF
S315080104287B690AFB03F313443A69AAFB02010B44E5
S3150801043819462B4B03FB01F2002300FB03F3134474
S31508010448274AA0FB02452B441D463B6A0022BB608E
S31508010458FA60BB6A00223B607A60D7E902010B465B
S31508010468D7E900AB524602FB03F25B4684460CFB0E
S3150801047803F3134402465146A2FB01894B449946A4
S3150801048842464B4620462946F8F7E2FD02460B4600
S3150801049813467B6307E07B6A114A03FB02F2BB6AD0
S315080104A8B2FBF3F37B630F4B5B7B1A467B6A93427A
S315080104B808D17B6B5B087B6304E07B6A0B4A02FB0A
S315080104C803F37B637B6B3B6302E0094B3B6300BF2A
S315080104D83B6B18463837BD46BDE8B08F0010024059
S315080104E840787D01584401086844010800093D001F
S315080104F800127A0080B400AF024B1B681846BD4645
S3150801050880BC70476C00002080B500AFFFF7F2FF8A
S315080105180246054B5B681B0A03F007030349CB5CD4
S3150801052822FA03F3184680BD001002405044010818
S3150801053880B500AFFFF7DEFF0246054B5B68DB0AAD
S3150801054803F007030349CB5C22FA03F3184680BD77
S31508010558001002405044010880B485B000AF7860A5
S315080105680A4B1B680A4AA2FB03235B0A7A6802FB41
S3150801057803F3FB6000BFFB685A1EFA60002BF9D12A
S3150801058800BF00BF1437BD4680BC70476C00002009
S31508010598D34D621080B588B000AF786000237B61BF
S315080105A800233B610023FB617B681B6803F0010399
S315080105B8002B7DD00023FB768B4BDB6903F0805338
S315080105C8002B0DD1884BDB69874A43F08053D361E9
S315080105D8854BDB6903F08053FB60FB680123FB76D7
S315080105E8824B1B6803F48073002B18D17F4B1B6859
S315080105F87E4A43F480731360FDF7BAF9786108E017
S31508010608FDF7B6F902467B69D31A642B01D9032388
S31508010618E5E0764B1B6803F48073002BF0D0724B28
S315080106281B6A03F440733B613B69002B2ED07B6838
S315080106385B6803F440733A699A4227D06A4B1B6A86
S3150801064823F440733B616A4B01221A60684B002206
S315080106581A60654A3B6913623B6903F00103002B7B
S3150801066814D0FDF785F978610AE0FDF781F90246A4
S315080106787B69D31A41F28832934201D90323AEE042
S31508010688594B1B6A03F00203002BEED0564B1B6A23
S3150801069823F440727B685B68534913430B62FB7EFC
S315080106A8012B05D1504BDB694F4A23F08053D3619F
S315080106B87B681B6803F00203002B08D04A4B5B686A
S315080106C823F440427B689B68474913434B607B6820
S315080106D81B6803F00403002B08D0434BDB6A23F499
S315080106E800327B68DB6840491343CB627B681B6829
S315080106F803F00803002B08D03B4BDB6A23F480225E
S315080107087B681B6938491343CB62374BDB6A03F4A9
S315080107180033002B05D1344BDB6A03F48023002B05
S3150801072801D00123FB61FB69012B48D12E4B1B68BC
S3150801073803F08053002B38D12B4B1B6803F08063D9
S31508010748002B09D0284BDB6A03F0F0027B689B690A
S315080107589A4201D0012342E0234BDB6A23F0F002D7
S315080107687B689B6920491343CB621F4BDB6A23F4D9
S3150801077870427B685B691C491343CB621D4B012296
S315080107881A60FDF7F5F8786108E0FDF7F1F8024611
S315080107987B69D31A642B01D9032320E0124B1B6802
S315080107A803F00053002BF0D009E00F4BDB6A03F482
S315080107B870427B685B699A4201D001230FE07B6826
S315080107C81B6803F01003002B08D0074B5B6823F45A
S315080107D880027B68DB69044913434B60002318468A
S315080107E82037BD4680BD00BF00100240007000409A
S315080107F8400442427000424280B58AB000AF786030
S315080108080023FB6100237B620023BB6100237B6114
S3150801081800233B610023FB600023BB6000233B6286
S315080108287B68013B0F2B00F21D8101A252F823F0C8
S31508010838ED090108510A01086D0A01084B09010861
S315080108486D0A01086D0A01086D0A01089D09010862
S315080108586D0A01086D0A01086D0A01086D0A010881
S315080108686D0A01086D0A01086D0A01087908010867
S31508010878834B5B68BB60824B1B6803F08073002B54
S3150801088800F0F280BB689B0C03F00F037D4AD35C2A
S31508010898BB61BB6803F48033002B3BD0784BDB6A1A
S315080108A803F00F03784AD35CFB61754BDB6A03F4E3
S315080108B88033002B1CD0724BDB6A1B0903F00F032C
S315080108C80133FB606E4BDB6A1B0A03F00F03023325
S315080108D87B616E4AFB68B2FBF3F37A6903FB02F2A2
S315080108E8FB69B2FBF3F2BB6902FB03F37B6207E020
S315080108F8664AFB69B2FBF3F2BB6902FB03F37B6247
S31508010908604B5B7B1A46BB69934208D17B6A5B08D5
S315080109187B6204E0BB695E4A02FB03F37B62584BC0
S315080109285B6803F48003B3F5800F02D17B6A3B62E7
S315080109389AE07B6A5B00574AA2FB03235B083B6282
S3150801094892E04F4BDB6A03F40033002B03D1FFF720
S3150801095815FD38628AE04A4B1B6803F08053002B61
S3150801096800F08480464BDB6A1B0903F00F03013349
S31508010978FB60434BDB6A1B0B03F00F0302333B6136
S31508010988424AFB68B2FBF3F33A6902FB03F35B00DD
S315080109983B626BE03A4BDB6A03F48023002B03D1F5
S315080109A8FFF7ECFC386263E0354B1B6803F08053AC
S315080109B8002B5DD0324BDB6A1B0903F00F030133A9
S315080109C8FB602F4BDB6A1B0B03F00F0302333B61FA
S315080109D82E4AFB68B2FBF3F33A6902FB03F35B00A1
S315080109E83B6245E0264B1B6ABB60BB6803F4407350
S315080109F8B3F5807F08D1BB6803F00203002B03D047
S31508010A084FF400433B621EE0BB6803F44073B3F539
S31508010A18007F09D11A4B5B6A03F00203002B03D046
S31508010A2849F640433B620EE0BB6803F44073B3F5ED
S31508010A38407F1FD1124B1B6803F40033002B19D0D2
S31508010A48154B3B6216E015E0FFF772FD02460C4BA3
S31508010A585B689B0B03F0030301335B00B2FBF3F3FB
S31508010A683B6208E000BF06E000BF04E000BF02E001
S31508010A7800BF00E000BF3B6A18462837BD4680BD5F
S31508010A8800100240784401088844010840787D012D
S31508010A9800093D00ABAAAAAAF0FA020080B584B0FB
S31508010AA800AF78600023FB607B68002B01D1012326
S31508010AB87AE07B685B7CDBB2002B05D17B68002278
S31508010AC81A747868FAF736FF7B6802225A747868C6
S31508010AD800F070F80346002B04D07B6804225A7488
S31508010AE8012361E0786800F092F80346002B04D0E8
S31508010AF87B6804225A74012356E07B681B685A6886
S31508010B087B681B6822F007025A607B689B68002B82
S31508010B1805D0274B1B6B264A23F001031363244B85
S31508010B28DB6A23F460727B689B6821491343CB62AD
S31508010B387B685B68B3F1FF3F03D07B685B68FB6042
S31508010B480EE00120FFF758FEF860FB68002B04D178
S31508010B587B6804225A74012326E0FB68013BFB6083
S31508010B68FB681A0C7B681B6802F00F029A607B689F
S31508010B781B68FA6892B2DA60786800F070F803467A
S31508010B88002B04D07B6804225A7401230CE07B6885
S31508010B980022DA737B6801225A737B6801229A73E9
S31508010BA87B6801225A74002318461037BD4680BD52
S31508010BB8006C004080B584B000AF78600023FB6004
S31508010BC87B68002B01D101231DE07B681B685A68E5
S31508010BD87B681B6822F008025A60FCF7C9FEF860B0
S31508010BE809E0FCF7C5FE0246FB68D31AB3F57A7F16
S31508010BF801D9032307E07B681B685B6803F00803D0
S31508010C08002BEED0002318461037BD4680BD80B5A7
S31508010C1884B000AF78600023FB60FCF7A9FEF86092
S31508010C2809E0FCF7A5FE0246FB68D31AB3F57A7FF5
S31508010C3801D903230FE07B681B685B6803F020036F
S31508010C48002BEED07B681B685A687B681B6842F0E4
S31508010C5810025A60002318461037BD4680BD80B574
S31508010C6884B000AF78600023FB607B681B685A680C
S31508010C787B681B6822F010025A60FCF779FEF86057
S31508010C8809E0FCF775FE0246FB68D31AB3F57A7FC5
S31508010C9801D9032307E07B681B685B6803F0200317
S31508010CA8002BEED0002318461037BD4680BD80B507
S31508010CB882B000AF78607B68002B01D1012341E03F
S31508010CC87B6893F83D30DBB2002B06D17B6800229E
S31508010CD883F83C207868FCF73BFB7B68022283F89B
S31508010CE83D207B681A687B6804331946104600F06C
S31508010CF8C3FC7B68012283F846207B68012283F8B6
S31508010D083E207B68012283F83F207B68012283F80D
S31508010D1840207B68012283F841207B68012283F8F9
S31508010D2842207B68012283F843207B68012283F8E5
S31508010D3844207B68012283F845207B68012283F8D1
S31508010D483D20002318460837BD4680BD80B584B0C6
S31508010D5800AF786039600023FB733B68002B09D123
S31508010D687B6893F83E30DBB2012B14BF01230023BD
S31508010D78DBB222E03B68042B09D17B6893F83F3044
S31508010D88DBB2012B14BF01230023DBB215E03B6854
S31508010D98082B09D17B6893F84030DBB2012B14BFC5
S31508010DA801230023DBB208E07B6893F84130DBB204
S31508010DB8012B14BF01230023DBB2002B01D0012329
S31508010DC8AEE03B68002B04D17B68022283F83E20FB
S31508010DD813E03B68042B04D17B68022283F83F2081
S31508010DE80BE03B68082B04D17B68022283F8402074
S31508010DF803E07B68022283F841203B680C2B41D823
S31508010E0801A252F823F000BF450E01088D0E01080C
S31508010E188D0E01088D0E0108570E01088D0E010861
S31508010E288D0E01088D0E0108690E01088D0E01083F
S31508010E388D0E01088D0E01087B0E01087B681B685B
S31508010E48DA687B681B6842F00202DA601DE07B6893
S31508010E581B68DA687B681B6842F00402DA6014E0EA
S31508010E687B681B68DA687B681B6842F00802DA60E7
S31508010E780BE07B681B68DA687B681B6842F010021E
S31508010E88DA6002E00123FB7300BFFB7B002B46D126
S31508010E987B681B6801223968184600F083FE7B685F
S31508010EA81B68214A934207D17B681B685A6C7B6881
S31508010EB81B6842F400425A647B681B681A4A9342C3
S31508010EC813D07B681B68B3F1804F0ED07B681B680B
S31508010ED8164A934209D07B681B68154A934204D07F
S31508010EE87B681B68134A934211D17B681B689B6808
S31508010EF803F00703BB60BB68062B10D07B681B6829
S31508010F081A687B681B6842F001021A6007E07B6869
S31508010F181B681A687B681B6842F001021A60FB7B2A
S31508010F2818461037BD4680BD002C01400004004014
S31508010F3800080040000C004080B582B000AF786018
S31508010F487B68002B01D1012341E07B6893F83D308A
S31508010F58DBB2002B06D17B68002283F83C2078682F
S31508010F6800F039F87B68022283F83D207B681A6805
S31508010F787B6804331946104600F07EFB7B6801221C
S31508010F8883F846207B68012283F83E207B68012284
S31508010F9883F83F207B68012283F840207B68012279
S31508010FA883F841207B68012283F842207B68012265
S31508010FB883F843207B68012283F844207B68012251
S31508010FC883F845207B68012283F83D2000231846CB
S31508010FD80837BD4680BD80B483B000AF786000BFCE
S31508010FE80C37BD4680BC704780B584B000AF7860C1
S31508010FF839603B68002B09D17B6893F83E30DBB230
S31508011008012B14BF01230023DBB222E03B68042B22
S3150801101809D17B6893F83F30DBB2012B14BF012352
S315080110280023DBB215E03B68082B09D17B6893F8E6
S315080110384030DBB2012B14BF01230023DBB208E0E1
S315080110487B6893F84130DBB2012B14BF01230023D7
S31508011058DBB2002B01D0012363E03B68002B04D1E6
S315080110687B68022283F83E2013E03B68042B04D1EF
S315080110787B68022283F83F200BE03B68082B04D1E2
S315080110887B68022283F8402003E07B68022283F802
S3150801109841207B681B6801223968184600F082FDE1
S315080110A87B681B68214A934207D17B681B685A6C7F
S315080110B87B681B6842F400425A647B681B681B4AB2
S315080110C8934213D07B681B68B3F1804F0ED07B68B7
S315080110D81B68174A934209D07B681B68154A9342CD
S315080110E804D07B681B68144A934211D17B681B6834
S315080110F89B6803F00703FB60FB68062B10D07B6827
S315080111081B681A687B681B6842F001021A6007E0C7
S315080111187B681B681A687B681B6842F001021A60BB
S31508011128002318461037BD4680BD00BF002C014074
S315080111380004004000080040000C004080B584B057
S3150801114800AF78607B681B68DB68FB607B681B6897
S315080111581B69BB60BB6803F00203002B20D0FB6840
S3150801116803F00203002B1BD07B681B686FF0020291
S315080111781A617B6801221A777B681B689B6903F0E9
S315080111880303002B03D0786800F05AFA05E078685B
S31508011198F9F730F8786800F05CFA7B6800221A7764
S315080111A8BB6803F00403002B20D0FB6803F0040393
S315080111B8002B1BD07B681B686FF004021A617B68D9
S315080111C802221A777B681B689B6903F44073002B14
S315080111D803D0786800F034FA05E07868F9F70AF870
S315080111E8786800F036FA7B6800221A77BB6803F03C
S315080111F80803002B20D0FB6803F00803002B1BD03B
S315080112087B681B686FF008021A617B6804221A77E3
S315080112187B681B68DB6903F00303002B03D0786836
S3150801122800F00EFA05E07868F8F7E4FF786800F048
S3150801123810FA7B6800221A77BB6803F01003002BA3
S3150801124820D0FB6803F01003002B1BD07B681B68B2
S315080112586FF010021A617B6808221A777B681B6887
S31508011268DB6903F44073002B03D0786800F0E8F9CA
S3150801127805E07868F8F7BEFF786800F0EAF97B6850
S3150801128800221A77BB6803F00103002B0CD0FB6810
S3150801129803F00103002B07D07B681B686FF0010276
S315080112A81A61786800F0C3F9BB6803F08003002B5C
S315080112B80CD0FB6803F08003002B07D07B681B68FA
S315080112C86FF080021A61786800F0FFFCBB6803F0CA
S315080112D84003002B0CD0FB6803F04003002B07D012
S315080112E87B681B686FF040021A61786800F0BAF9E2
S315080112F8BB6803F02003002B0CD0FB6803F020031E
S31508011308002B07D07B681B686FF020021A61786882
S3150801131800F0D2FC00BF1037BD4680BD80B586B047
S3150801132800AFF860B9607A600023FB75FB6893F82B
S315080113383C30012B01D10223AEE0FB68012283F878
S315080113483C207B680C2B00F29F8001A252F823F0FF
S315080113588D130108911401089114010891140108C3
S31508011368CD13010891140108911401089114010873
S315080113780F14010891140108911401089114010820
S315080113884F140108FB681B68B968184600F0ECF9A0
S31508011398FB681B689A69FB681B6842F008029A6130
S315080113A8FB681B689A69FB681B6822F004029A6144
S315080113B8FB681B689969BB681A69FB681B680A4355
S315080113C89A6164E0FB681B68B968184600F032FA46
S315080113D8FB681B689A69FB681B6842F400629A6194
S315080113E8FB681B689A69FB681B6822F480629A6124
S315080113F8FB681B689969BB681B691A02FB681B6845
S315080114080A439A6143E0FB681B68B968184600F005
S315080114187BFAFB681B68DA69FB681B6842F00802F5
S31508011428DA61FB681B68DA69FB681B6822F0040243
S31508011438DA61FB681B68D969BB681A69FB681B68A6
S315080114480A43DA6123E0FB681B68B968184600F0A5
S31508011458C5FAFB681B68DA69FB681B6842F400620F
S31508011468DA61FB681B68DA69FB681B6822F4806223
S31508011478DA61FB681B68D969BB681B691A02FB68CC
S315080114881B680A43DA6102E00123FB7500BFFB68A2
S31508011498002283F83C20FB7D18461837BD4680BDD7
S315080114A880B584B000AF786039600023FB737B6828
S315080114B893F83C30012B01D10223B4E07B68012261
S315080114C883F83C207B68022283F83D207B681B68E9
S315080114D89B68BB60BB6823F07703BB60BB6823F4D2
S315080114E87F43BB607B681B68BA689A603B681B6860
S315080114F8B3F5005F3ED0B3F5005F00F28780B3F518
S31508011508805F00F08680B3F5805F7FD8702B1AD08C
S31508011518702B7BD8602B50D0602B77D8502B3CD0BA
S31508011528502B73D8402B58D0402B6FD8302B64D00A
S31508011538302B6BD8202B60D0202B67D8002B5CD09A
S31508011548102B5AD062E07B6818683B6899683B6833
S315080115585A683B68DB6800F006FB7B681B689B6872
S31508011568BB60BB6843F07703BB607B681B68BA68D6
S315080115789A604FE07B6818683B6899683B685A68BF
S315080115883B68DB6800F0EFFA7B681B689A687B683A
S315080115981B6842F480429A603CE07B6818683B689D
S315080115A859683B68DB681A4600F066FA7B681B6867
S315080115B85021184600F0BDFA2CE07B6818683B688C
S315080115C859683B68DB681A4600F084FA7B681B6829
S315080115D86021184600F0ADFA1CE07B6818683B687C
S315080115E859683B68DB681A4600F046FA7B681B6847
S315080115F84021184600F09DFA0CE07B681A683B689A
S315080116081B681946104600F094FA03E00123FB7398
S3150801161800E000BF7B68012283F83D207B68002231
S3150801162883F83C20FB7B18461037BD4680BD80B43D
S3150801163883B000AF786000BF0C37BD4680BC7047E1
S3150801164880B483B000AF786000BF0C37BD4680BC54
S31508011658704780B483B000AF786000BF0C37BD46C9
S3150801166880BC704780B483B000AF786000BF0C3780
S31508011678BD4680BC7047000080B485B000AF78606D
S3150801168839607B681B68FB607B68334A93420FD0D5
S315080116987B68B3F1804F0BD07B68304A934207D0F9
S315080116A87B682F4A934203D07B682E4A934208D116
S315080116B8FB6823F07003FB603B685B68FA681343B1
S315080116C8FB607B68244A93420FD07B68B3F1804F4D
S315080116D80BD07B68214A934207D07B68204A9342FC
S315080116E803D07B681F4A934208D1FB6823F44073E9
S315080116F8FB603B68DB68FA681343FB60FB6823F009
S3150801170880023B685B691343FB607B68FA681A6069
S315080117183B689A687B68DA623B681A687B689A62EA
S315080117287B680D4A934203D13B681A697B681A6339
S315080117387B6801225A617B681B6903F00103002B48
S3150801174805D07B681B6923F001027B681A6100BF13
S315080117581437BD4680BC7047002C01400004004080
S3150801176800080040000C004080B487B000AF7860DC
S3150801177839607B681B6A7B617B681B6A23F00102F7
S315080117887B681A627B685B683B617B689B69FB605F
S31508011798FB6823F07003FB60FB6823F00303FB6017
S315080117A83B681B68FA681343FB607B6923F00203ED
S315080117B87B613B689B687A6913437B617B681C4A32
S315080117C893420CD17B6923F008037B613B68DB688C
S315080117D87A6913437B617B6923F004037B617B6820
S315080117E8134A934211D13B6923F480733B613B69E0
S315080117F823F400733B613B685B693A6913433B61B0
S315080118083B689B693A6913433B617B683A695A6045
S315080118187B68FA689A613B685A687B685A637B6889
S315080118287A691A6200BF1C37BD4680BC704700BF7B
S31508011838002C014080B487B000AF786039607B68B6
S315080118481B6A7B617B681B6A23F010027B681A6234
S315080118587B685B683B617B689B69FB60FB6823F473
S31508011868E043FB60FB6823F44073FB603B681B6835
S315080118781B02FA681343FB607B6923F020037B612B
S315080118883B689B681B017A6913437B617B681D4A20
S3150801189893420DD17B6923F080037B613B68DB6842
S315080118A81B017A6913437B617B6923F040037B61DA
S315080118B87B68144A934213D13B6923F480633B61DD
S315080118C83B6923F400633B613B685B699B003A69A2
S315080118D813433B613B689B699B003A6913433B6128
S315080118E87B683A695A607B68FA689A613B685A68FC
S315080118F87B689A637B687A691A6200BF1C37BD469A
S3150801190880BC7047002C014080B487B000AF78606E
S3150801191839607B681B6A7B617B681B6A23F4807262
S315080119287B681A627B685B683B617B68DB69FB607D
S31508011938FB6823F07003FB60FB6823F00303FB6075
S315080119483B681B68FA681343FB607B6923F40073D9
S315080119587B613B689B681B027A6913437B617B68D9
S315080119681D4A93420DD17B6923F400637B613B6869
S31508011978DB681B027A6913437B617B6923F48063FD
S315080119887B617B68144A934213D13B6923F48053DC
S315080119983B613B6923F400533B613B685B691B0167
S315080119A83A6913433B613B689B691B013A691343CF
S315080119B83B617B683A695A607B68FA68DA613B6811
S315080119C85A687B68DA637B687A691A6200BF1C37CA
S315080119D8BD4680BC704700BF002C014080B487B063
S315080119E800AF786039607B681B6A3B617B681B6A54
S315080119F823F480527B681A627B685B687B617B6823
S31508011A08DB69FB60FB6823F4E043FB60FB6823F4AE
S31508011A184073FB603B681B681B02FA681343FB604B
S31508011A283B6923F400533B613B689B681B033A698E
S31508011A3813433B617B680F4A934209D17B6923F4B7
S31508011A4880437B613B685B699B017A6913437B61C8
S31508011A587B687A695A607B68FA68DA613B685A680A
S31508011A687B681A647B683A691A6200BF1C37BD46E7
S31508011A7880BC7047002C014080B487B000AFF8607D
S31508011A88B9607A60FB681B6A7B61FB681B6A23F08D
S31508011A980102FB681A62FB689B693B613B6923F093
S31508011AA8F0033B617B681B013A6913433B617B6918
S31508011AB823F00A037B617A69BB6813437B61FB6878
S31508011AC83A699A61FB687A691A6200BF1C37BD468A
S31508011AD880BC704780B487B000AFF860B9607A6097
S31508011AE8FB681B6A7B61FB681B6A23F01002FB68AB
S31508011AF81A62FB689B693B613B6923F470433B6146
S31508011B087B681B033A6913433B617B6923F0A0038E
S31508011B187B61BB681B017A6913437B61FB683A6978
S31508011B289A61FB687A691A6200BF1C37BD4680BC90
S31508011B38704780B485B000AF786039607B689B6868
S31508011B48FB60FB6823F07003FB603A68FB68134384
S31508011B5843F00703FB607B68FA689A6000BF14378D
S31508011B68BD4680BC704780B487B000AFF860B960DD
S31508011B787A603B60FB689B687B617B6923F47F43DA
S31508011B887B613B681A027B681A43BB6813437A6907
S31508011B9813437B61FB687A699A6000BF1C37BD46A7
S31508011BA880BC704780B487B000AFF860B9607A60C6
S31508011BB8BB6803F01F03012202FA03F37B61FB6882
S31508011BC81A6A7B69DB431A40FB681A62FB681A6A58
S31508011BD8BB6803F01F03796801FA03F31A43FB6824
S31508011BE81A6200BF1C37BD4680BC704780B485B0F1
S31508011BF800AF786039607B6893F83C30012B01D1D6
S31508011C0802234BE07B68012283F83C207B68022289
S31508011C1883F83D207B681B685B68FB607B681B68EB
S31508011C289B68BB60FB6823F07003FB603B681B6815
S31508011C38FA681343FB607B681B68FA685A607B6815
S31508011C481B68194A934213D07B681B68B3F1804F06
S31508011C580ED07B681B68154A934209D07B681B68B6
S31508011C68134A934204D07B681B68124A93420CD1E3
S31508011C78BB6823F08003BB603B685B68BA6813439B
S31508011C88BB607B681B68BA689A607B68012283F81F
S31508011C983D207B68002283F83C2000231846143728
S31508011CA8BD4680BC704700BF002C014000040040B7
S31508011CB800080040000C004080B483B000AF78608B
S31508011CC800BF0C37BD4680BC704780B483B000AFEF
S31508011CD8786000BF0C37BD4680BC704780B582B0B6
S31508011CE800AF78607B68002B01D1012342E07B684D
S31508011CF893F84130DBB2002B06D17B68002283F8C2
S31508011D0840207868FBF76CFC7B68242283F841201D
S31508011D187B681B68DA687B681B6822F40052DA60FC
S31508011D28786800F0B5FF7B681B681A697B681B68C9
S31508011D3822F490421A617B681B685A697B681B689A
S31508011D4822F02A025A617B681B68DA687B681B6875
S31508011D5842F40052DA607B6800225A647B682022C2
S31508011D6883F841207B68202283F842207B68002279
S31508011D785A63002318460837BD4680BD80B58AB020
S31508011D8802AFF860B9603B601346FB8000237B61AC
S31508011D98FB6893F84130DBB2202B75D1BB68002B61
S31508011DA802D0FB88002B01D101236EE0FB680022D3
S31508011DB85A64FB68212283F84120FBF7D9FD78612B
S31508011DC8FB68FA889A84FB68FA88DA84FB689B6850
S31508011DD8B3F5805F08D1FB681B69002B04D1002382
S31508011DE8FB61BB68BB6103E0BB68FB610023BB61A0
S31508011DF82EE03B6800937B6900228021F86800F091
S31508011E08B9FC0346002B05D0FB68202283F841203C
S31508011E1803233AE0FB69002B0BD1BB691B881A46D9
S31508011E28FB681B68C2F308025A60BB690233BB61C7
S31508011E3807E0FB691A78FB681B685A60FB69013376
S31508011E48FB61FB68DB8C9BB2013B9AB2FB68DA84BF
S31508011E58FB68DB8C9BB2002BCBD13B6800937B6973
S31508011E6800224021F86800F085FC0346002B05D0BE
S31508011E78FB68202283F84120032306E0FB68202219
S31508011E8883F84120002300E0022318462037BD467F
S31508011E9880BD80B485B000AFF860B9601346FB8091
S31508011EA8FB6893F84130DBB2202B21D1BB68002BA4
S31508011EB802D0FB88002B01D101231AE0FB68BA6816
S31508011EC81A62FB68FA889A84FB68FA88DA84FB68D6
S31508011ED800225A64FB68212283F84120FB681B68A3
S31508011EE8DA68FB681B6842F08002DA60002300E0C2
S31508011EF8022318461437BD4680BC704780B58CB096
S31508011F0800AFF860B9601346FB80FB6893F8423066
S31508011F18DBB2202B4AD1BB68002B02D0FB88002BE9
S31508011F2801D1012343E0FB6801221A63FB680022F9
S31508011F385A63FB881A46B968F86800F074FC0346C0
S31508011F4887F82F3097F82F30002B2CD1FB681B6B9D
S31508011F58012B25D100233B61FB681B681B683B6184
S31508011F68FB681B685B683B613B69FB681B680C334C
S31508011F78BB61BB6953E8003F7B617B6943F010038A
S31508011F88BB62FB681B680C33BA6A7A623B62396AB8
S31508011F987A6A41E80023FB61FB69002BE5D102E077
S31508011FA8012387F82F3097F82F3000E002231846C7
S31508011FB83037BD4680BD000080B5A2B000AF786055
S31508011FC80123C7F884307B681B680C333B663B6E74
S31508011FD853E8003FFB65FB6D23F4F073C7F88030BF
S31508011FE87B681B680C33D7F88020FA66BB66B96E1E
S31508011FF8FA6E41E800237B667B6E002BE3D17B688A
S315080120081B681433FB64FB6C53E8003FBB64BB6C69
S3150801201823F00103FB677B681B681433FA6FBA65FB
S315080120287B65796DBA6D41E800233B653B6D002BED
S31508012038E5D17B681B6B012B19D17B681B680C33AF
S31508012048BB63BB6B53E8003F7B637B6B23F01003D1
S31508012058BB677B681B680C33BA6F7A643B64396C57
S315080120687A6C41E80023FB63FB6B002BE5D17B689F
S315080120789B6B002B0FD07B681B685B6903F0800399
S31508012088002B04D07B689B6B534A5A6303E07B6831
S315080120989B6B00225A637B68DB6B002B0FD07B682E
S315080120A81B685B6903F04003002B04D07B68DB6B74
S315080120B84A4A5A6303E07B68DB6B00225A637B68EA
S315080120C81B685B6903F08003002B2DD07B681B68AE
S315080120D814337B627B6A53E8003F3B623B6A23F011
S315080120E880037B677B681B6814337A6F3A63FB62E4
S315080120F8F96A3A6B41E80023BB62BB6A002BE5D152
S315080121087B689B6B002B0FD07B689B6B1846FDF78A
S315080121189DF90346002B04D07B689B6B00225A6302
S3150801212802E00023C7F884307B681B685B6903F003
S315080121384003002B30D07B681B6814333B613B692D
S3150801214853E8003FFB60FB6823F040033B677B6865
S315080121581B6814333A6FFA61BB61B969FA6941E8D0
S3150801216800237B617B69002BE5D17B68DB6B002B40
S3150801217812D07B68DB6B1846FDF768F90346002B16
S3150801218807D07B68DB6B00225A630123C7F88430C2
S3150801219802E00023C7F88430D7F88430012B16D11A
S315080121A87B680022DA847B680022DA857B6800224C
S315080121B85A647B68202283F841207B68202283F8A9
S315080121C842207B6800221A63786800F0ADFA00237A
S315080121D818468837BD4680BD8D290108ED290108AD
S315080121E880B5BAB000AF78607B681B681B68C7F80A
S315080121F8E4307B681B68DB68C7F8E0307B681B68D6
S315080122085B69C7F8DC300023C7F8D8300023C7F85C
S31508012218D430D7F8E43003F00F03C7F8D830D7F825
S31508012228D830002B0FD1D7F8E43003F02003002B60
S3150801223809D0D7F8E03003F02003002B03D07868DB
S3150801224800F067FC5BE2D7F8D830002B00F0DE8097
S31508012258D7F8DC3003F00103002B06D1D7F8E030B4
S3150801226803F49073002B00F0D180D7F8E43003F01B
S315080122780103002B0BD0D7F8E03003F48073002B49
S3150801228805D07B685B6C43F001027B685A64D7F812
S31508012298E43003F00403002B0BD0D7F8DC3003F045
S315080122A80103002B05D07B685B6C43F002027B684F
S315080122B85A64D7F8E43003F00203002B0BD0D7F899
S315080122C8DC3003F00103002B05D07B685B6C43F017
S315080122D804027B685A64D7F8E43003F00803002B34
S315080122E811D0D7F8E03003F02003002B05D1D7F831
S315080122F8DC3003F00103002B05D07B685B6C43F0E7
S3150801230808027B685A647B685B6C002B00F0F281D3
S31508012318D7F8E43003F02003002B08D0D7F8E030CB
S3150801232803F02003002B02D0786800F0F2FB7B68E3
S315080123381B685B6903F04003002B14BF01230023C4
S31508012348DBB2C7F8D4307B685B6C03F00803002B53
S3150801235803D1D7F8D430002B4FD0786800F09CFA0F
S315080123687B681B685B6903F04003002B41D07B68D7
S315080123781B681433C7F89C30D7F89C3053E8003FDC
S31508012388C7F89830D7F8983023F04003C7F8D03003
S315080123987B681B681433D7F8D020C7F8A820C7F874
S315080123A8A430D7F8A410D7F8A82041E80023C7F81D
S315080123B8A030D7F8A030002BD9D17B68DB6B002B6E
S315080123C813D07B68DB6B7E4A5A637B68DB6B1846DE
S315080123D8FDF73CF80346002B16D07B68DB6B5B6B75
S315080123E87A68D26B104698470EE0786800F093F938
S315080123F80AE0786800F08FF906E0786800F08BF94A
S315080124087B6800225A6475E100BF73E17B681B6B20
S31508012418012B40F04F81D7F8E43003F01003002B65
S3150801242800F04881D7F8E03003F01003002B00F0DC
S3150801243841810023BB607B681B681B68BB607B689E
S315080124481B685B68BB60BB687B681B685B6903F0D4
S315080124584003002B00F0B6807B68DB6B1B685B6862
S31508012468A7F8BE30B7F8BE30002B00F045817B6867
S315080124789B8DB7F8BE209A4280F03E817B68B7F8F3
S31508012488BE20DA857B68DB6B9B69202B00F0888088
S315080124987B681B680C33C7F88830D7F8883053E847
S315080124A8003FC7F88430D7F8843023F48073C7F817
S315080124B8B8307B681B680C33D7F8B820C7F894205E
S315080124C8C7F89030D7F89010D7F8942041E8002338
S315080124D8C7F88C30D7F88C30002BD9D17B681B68A4
S315080124E814337B677B6F53E8003F3B673B6F23F0E9
S315080124F80103C7F8B4307B681B681433D7F8B420CE
S31508012508C7F88020FB67F96FD7F8802041E80023D0
S31508012518BB67BB6F002BE1D17B681B6814333B662D
S315080125283B6E53E8003FFB65FB6D23F04003C7F894
S31508012538B0307B681B681433D7F8B020FA66BB66D7
S31508012548B96EFA6E41E800237B667B6E002BE3D1F0
S315080125587B68202283F842207B6800221A637B68FD
S315080125681B680C33FB64FB6C53E8003FBB64BB6C0C
S3150801257823F01003C7F8AC307B681B680C33D7F80F
S31508012588AC20BA657B65796DBA6D41E800233B6570
S315080125983B6D002BE3D17B68DB6B1846FCF71BFF09
S315080125A87B6802225A637B689A8D7B68DB8D9BB2AE
S315080125B8D31A9BB219467868FAF702F89CE000BF65
S315080125C8652901087B689A8D7B68DB8D9BB2D31ACE
S315080125D8A7F8CE307B68DB8D9BB2002B00F08E8086
S315080125E8B7F8CE30002B00F089807B681B680C335E
S315080125F8BB63BB6B53E8003F7B637B6B23F4907328
S31508012608C7F8C8307B681B680C33D7F8C8207A64C2
S315080126183B64396C7A6C41E80023FB63FB6B002B3E
S31508012628E3D17B681B6814337B627B6A53E8003FF6
S315080126383B623B6A23F00103C7F8C4307B681B6811
S315080126481433D7F8C4203A63FB62F96A3A6B41E84E
S315080126580023BB62BB6A002BE3D17B68202283F87F
S3150801266842207B6800221A637B681B680C333B612E
S315080126783B6953E8003FFB60FB6823F01003C7F882
S31508012688C0307B681B680C33D7F8C020FA61BB6178
S31508012698B969FA6941E800237B617B69002BE3D1B3
S315080126A87B6802225A63B7F8CE3019467868F9F773
S315080126B887FF23E0D7F8E43003F08003002B09D01D
S315080126C8D7F8E03003F08003002B03D0786800F0D0
S315080126D8B9F914E0D7F8E43003F04003002B0ED01B
S315080126E8D7F8E03003F04003002B08D0786800F0EB
S315080126F8F8F904E000BF02E000BF00E000BFE837D0
S31508012708BD4680BD80B483B000AF786000BF0C3782
S31508012718BD4680BC704780B483B000AF786000BFFF
S315080127280C37BD4680BC704780B483B000AF78606B
S3150801273800BF0C37BD4680BC704780B485B000AF72
S3150801274878600023FB600023BB607B6893F84130FF
S31508012758DBB2FB607B6893F84230DBB2BB60FB688F
S31508012768DAB2BB68DBB21343DBB218461437BD4687
S3150801277880BC704780B586B000AFF860B9603B6029
S315080127881346FB713BE03B6AB3F1FF3F37D0FBF7D2
S31508012798EFF802463B68D31A3A6A9A4202D33B6A69
S315080127A8002B01D103233AE0FB681B68DB6803F0B9
S315080127B80403002B23D0BB68802B20D0BB68402B91
S315080127C81DD0FB681B681B6803F00803082B16D184
S315080127D800237B61FB681B681B687B61FB681B68B8
S315080127E85B687B617B69F86800F056F8FB68082224
S315080127F85A64FB68002283F8402001230FE0FB682E
S315080128081B681A68BB681340BA689A420CBF012349
S315080128180023DBB21A46FB799A42B4D0002318463C
S315080128281837BD4680BD80B485B000AFF860B96079
S315080128381346FB80FB68BA689A62FB68FA889A8528
S31508012848FB68FA88DA85FB6800225A64FB68222243
S3150801285883F84220FB681B69002B07D0FB681B68B5
S31508012868DA68FB681B6842F48072DA60FB681B68E1
S315080128785A69FB681B6842F001025A61FB681B68C2
S31508012888DA68FB681B6842F02002DA6000231846FA
S315080128981437BD4680BC704780B495B000AF7860E0
S315080128A87B681B680C337B637B6B53E8003F3B6390
S315080128B83B6B23F49073FB647B681B680C33FA6CD7
S315080128C83A64FB63F96B3A6C41E80023BB63BB6B5B
S315080128D8002BE5D17B681B6814333B623B6A53E8D6
S315080128E8003FFB61FB6923F00103BB647B681B6836
S315080128F81433BA6CFA62BB62B96AFA6A41E8002308
S315080129087B627B6A002BE5D17B681B6B012B19D18E
S315080129187B681B680C33FB60FB6853E8003FBB60A8
S31508012928BB6823F010037B647B681B680C337A6CDD
S31508012938BA617B617969BA6941E800233B613B69F8
S31508012948002BE5D17B68202283F842207B68002288
S315080129581A6300BF5437BD4680BC704780B584B03A
S3150801296800AF78607B685B6AFB60FB680022DA85E2
S31508012978FB680022DA84F868FFF7CDFE00BF103736
S31508012988BD4680BD80B584B000AF78607B685B6A58
S31508012998FB60FB689B6B00225A63FB68DB6B002BA9
S315080129A804D0FB68DB6B5B6B002B17D1FB68002235
S315080129B8DA84FB680022DA85FB6800225A64FB6818
S315080129C8202283F84120FB68202283F84220FB68ED
S315080129D800221A63F868FFF7A7FE00E000BF103760
S315080129E8BD4680BD80B584B000AF78607B685B6AF8
S315080129F8FB60FB68DB6B00225A63FB689B6B002B49
S31508012A0804D0FB689B6B5B6B002B17D1FB68002214
S31508012A18DA84FB680022DA85FB6800225A64FB68B7
S31508012A28202283F84120FB68202283F84220FB688C
S31508012A3800221A63F868FFF777FE00E000BF10372F
S31508012A48BD4680BD80B485B000AF78607B6893F8D1
S31508012A584130DBB2212B3ED17B689B68B3F5805F99
S31508012A6814D17B681B69002B10D17B681B6AFB6034
S31508012A78FB681B881A467B681B68C2F308025A60FA
S31508012A887B681B6A9A1C7B681A6208E07B681B6A62
S31508012A98591C7A6811621A787B681B685A607B68C0
S31508012AA8DB8C9BB2013B9BB27A681946D184002B11
S31508012AB80FD17B681B68DA687B681B6822F080027D
S31508012AC8DA607B681B68DA687B681B6842F0400233
S31508012AD8DA60002300E0022318461437BD4680BC95
S31508012AE8704780B582B000AF78607B681B68DA6882
S31508012AF87B681B6822F04002DA607B68202283F82B
S31508012B0841207868F9F7BCFD002318460837BD4601
S31508012B1880BD80B58CB000AF78607B6893F8423089
S31508012B28DBB2222B40F0AE807B689B68B3F5805FE9
S31508012B3817D17B681B69002B13D10023FB627B68BD
S31508012B489B6ABB627B681B685B689BB2C3F3080315
S31508012B589AB2BB6A1A807B689B6A9A1C7B689A62D6
S31508012B6826E07B689B6AFB620023BB627B689B68DD
S31508012B78B3F5805F07D07B689B68002B0AD17B6811
S31508012B881B69002B06D17B681B685B68DAB2FB6A8E
S31508012B981A7008E07B681B685B68DBB203F07F0381
S31508012BA8DAB2FB6A1A707B689B6A5A1C7B689A6256
S31508012BB87B68DB8D9BB2013B9BB27A681946D18546
S31508012BC8002B5DD17B681B68DA687B681B6822F075
S31508012BD82002DA607B681B68DA687B681B6822F45E
S31508012BE88072DA607B681B685A697B681B6822F001
S31508012BF801025A617B68202283F842207B680022F9
S31508012C085A637B681B6B012B35D17B6800221A63D3
S31508012C187B681B680C337B617B6953E8003F3B6122
S31508012C283B6923F010037B627B681B680C337A6A5D
S31508012C383A62FB61F9693A6A41E80023BB61BB69F3
S31508012C48002BE5D17B681B681B6803F01003102B62
S31508012C580AD10023FB607B681B681B68FB607B68DD
S31508012C681B685B68FB60FB687B689B8D19467868FF
S31508012C78F9F7A6FC02E07868FFF744FD002302E0AD
S31508012C88002300E0022318463037BD4680BD000000
S31508012C9880B584B000AF78607B681B681B6923F42C
S31508012CA840517B68DA687B681B680A431A617B6846
S31508012CB89A687B681B691A437B685B691343BB601F
S31508012CC87B681B68DB6823F4B05323F00C037A6826
S31508012CD81268B9680B43D3607B681B685B6923F480
S31508012CE840717B689A697B681B680A435A617B68E5
S31508012CF81B682C4A934203D1FDF71AFCF86002E0D7
S31508012D08FDF702FCF860FA6813469B0013449A001B
S31508012D181A447B685B689B00B2FBF3F3224AA2FB61
S31508012D2803235B091901FA6813469B0013449A00A1
S31508012D381A447B685B689B00B2FBF3F21A4BA3FB48
S31508012D4802035B09642000FB03F3D31A1B01323320
S31508012D58154AA2FB03235B0903F0F0031944FA6831
S31508012D6813469B0013449A001A447B685B689B00C8
S31508012D78B2FBF3F20C4BA3FB02035B09642000FBCD
S31508012D8803F3D31A1B013233074AA2FB03235B0950
S31508012D9803F00F027B681B680A449A6000BF103764
S31508012DA8BD4680BD003801401F85EB51002310B58B
S31508012DB80446C0E90033C0E9043383608181436668
S31508012DC8C2818361194608225C3000F043F90D4B2C
S31508012DD8246263620C4BA3620C4BE3620C4B2363BC
S31508012DE80C4B9C4206D003F16802944202D0D033B8
S31508012DF89C4205D104F15800BDE8104000F0A2B97B
S31508012E0810BD00BF5D2F01087F2F0108B72F0108E4
S31508012E18DB2F01087C100020024A0349034800F009
S31508012E2869B800BF78000020AD3C01088800002079
S31508012E3841680C4B10B59942044601D000F032FF9F
S31508012E48A168094B994202D0204600F02BFFE16898
S31508012E58064B994204D02046BDE8104000F022BF2F
S31508012E6810BD00BF7C100020E41000204C11002082
S31508012E7810B50B4B0B4C0C4A20461A60042100224C
S31508012E88FFF794FF04F1680001220921FFF78EFF75
S31508012E9804F1D0000222BDE810401221FFF786BFCF
S31508012EA8B41100207C100020212E0108014800F0E9
S31508012EB84AB900BFBD110020014800F045B900BF55
S31508012EC8BD11002010B50446FFF7F0FF236A1BB1B0
S31508012ED8BDE81040FFF7F0BF044B2362044B1B689B
S31508012EE8002BF5D1FFF7C4FFF2E700BF392E010819
S31508012EF8B41100202DE9F8430746884614460026EA
S31508012F08D4E90195B9F1010905D52468002CF7D149
S31508012F183046BDE8F883AB89012B07D9B5F90E30D8
S31508012F28013303D029463846C04706436835E9E7D9
S31508012F380FB407B5064904AB086853F8042B81682A
S31508012F48019300F087FB03B05DF804EB04B0704702
S31508012F588400002010B50C46B1F90E1000F0A4F84B
S31508012F680028ABBF636DA3891B1823F48053ACBF34
S31508012F786365A38110BD2DE9F0411F468B89054676
S31508012F88DB050C46164605D502230022B1F90E10B3
S31508012F9800F078F8A389324623F48053A38128469A
S31508012FA83B46B4F90E10BDE8F04100F08FB810B5EC
S31508012FB80C46B1F90E1000F065F8431CA38915BF34
S31508012FC8606523F4805343F48053A38118BFA38112
S31508012FD810BDB1F90E1000F045B830B51446002CED
S31508012FE805461A469BB005DA8B2303604FF0FF3076
S31508012FF81BB030BD4FF40273ADF80C304FF0000327
S3150801300819930CBF234604F1FF33029305934FF630
S31508013018FF7300910491ADF80E3069461E9B00F0C6
S31508013028F5F9431CBCBF8B232B60002CE0D000228A
S31508013038009B1A70DCE7000007B5009313460A4699
S31508013048014603480068FFF7C8FF03B05DF804FBAB
S315080130588400002003460244934200D1704703F8CE
S31508013068011BF9E738B50023054D044608462B60C8
S31508013078F9F7FFFF431C02D12B6803B1236038BD5A
S31508013088B811002038B50446084611460022054DF0
S315080130982A601A46FAF711F8431C02D12B6803B1BC
S315080130A8236038BDB811002038B5044608461146CC
S315080130B80022054D2A601A46F9F7BEFF431C02D1BC
S315080130C82B6803B1236038BDB811002038B504460A
S315080130D8084611460022054D2A601A46F7F7E4F80C
S315080130E8431C02D12B6803B1236038BDB8110020EF
S315080130F8014B1868704700BF8400002070B5002688
S315080131080C4D0D4C641BA410A64209D100F078FF9A
S3150801311800260A4D0A4C641BA410A64205D170BDA7
S3150801312855F8043B98470136EEE755F8043B9847A6
S315080131380136F2E7D4440108D4440108D444010805
S31508013148D84401087047704770470A44914200F10C
S31508013158FF3300D1704710B511F8014B914203F8B6
S31508013168014FF9D110BD000038B50546002940D0F0
S3150801317851F8043C0C1F002BB8BFE41800F0DEF820
S315080131881C4A136833B9636014602846BDE8384099
S3150801319800F0DAB8A34208D9206821188B4201BF82
S315080131A819685B6809182160EDE71A465B680BB16F
S315080131B8A342FAD911685018A0420BD120680144D4
S315080131C8501883421160E0D118685B68084410609A
S315080131D85360DAE702D90C232B60D6E72068211851
S315080131E88B4201BF19685B680918216063605460DE
S315080131F8CBE738BDC411002070B50F4E0C463168AF
S31508013208054611B900F024FE30602146284600F02B
S315080132181FFE431C03D14FF0FF34204670BDC41C62
S3150801322824F00304A042F8D0211A284600F010FE1B
S315080132380130F2D1EFE700BFC01100202DE9F843AC
S31508013248CD1C25F0030508350C2D38BF0C25002D96
S31508013258064601DBA94204D90C2333600020BDE8E0
S31508013268F883DFF8D48000F069F8D8F800301C46EE
S3150801327844BB29463046FFF7BFFF431C044658D1CD
S31508013288D8F800402746002F43D1002C4BD0236895
S315080132983946304604EB030900F0DAFD814542D187
S315080132A8216830466D1A2946FFF7A6FF01303AD03C
S315080132B823682B442360D8F800305A6862BBC8F8DB
S315080132C800700FE02268521B20D40B2A17D96119FE
S315080132D8A342256018BF5960636808BFC8F800107B
S315080132E862514B60304600F02FF804F10B00231D9C
S315080132F820F00700C21A1CBF1B1AA350AFE7626861
S31508013308A3420CBFC8F800205A60EBE72346646855
S31508013318AEE73C467F68B6E71A465B68A342FBD127
S3150801332800235360DEE70C233046336000F00CF8BF
S3150801333894E70560D6E700BFC41100200148FFF7E6
S3150801334802BF00BFBC1100200148FFF7FDBE00BF40
S31508013358BC1100202DE9F0471F468E688246BE42F9
S315080133680C4690460B682DD8B1F90C2012F4906FCB
S3150801337826D06569096905EB4505A3EB010905EB3E
S31508013388D5757B1C4B446D109D4238BF1D465305A8
S3150801339827D52946FFF752FF064660B34A462169EB
S315080133A8FFF7D3FEA38923F4906343F08003A3812F
S315080133B826614E4426603E466561A5EB0905A5606A
S315080133C8BE4200D93E4632464146206800F026FDEF
S315080133D80020A3689B1BA360236833442360BDE8C8
S315080133E8F0872A4600F052FD06460028E0D15046E5
S315080133F82169FFF7B9FE0C23CAF80030A3894FF0F3
S31508013408FF3043F04003A381E9E700002DE9F04FB7
S3150801341898468B8907461B060D4614469DB010D556
S315080134280B6973B94021FFF709FF2860286130B98C
S315080134380C233B604FF0FF301DB0BDE8F08F4023E9
S315080134486B610023099320238DF8293030234FF027
S315080134580109CDF80C80DFF898818DF82A302346C2
S315080134689A4613F8012B0AB1252AF9D1BAEB040BA6
S315080134780BD05B46224629463846FFF76BFF0130D3
S3150801348800F0A780099A5A4409929AF80030002B45
S3150801349800F09F8000234FF0FF32CDE905230AF19A
S315080134A8010A049307938DF853301A935446052253
S315080134B814F8011B4E4800F0DBFC049AD8B9D0066B
S315080134C844BF20238DF85330110744BF2B238DF8A9
S315080134D853309AF800302A2B15D0544600204FF05D
S315080134E80A0C079A214611F8013B303B092B4BD99F
S315080134F8B0B1079214E0A0EB080309FA03F31343E2
S31508013508A2460493D2E7039B191D1B680391002B56
S31508013518BBBF5B4242F0020207930793B8BF049206
S3150801352823782E2B0AD163782A2B32D1039B0234AE
S315080135381A1D1B68039243EAE3730593DFF8B4A0DF
S3150801354803225046217800F093FC38B14022049BA7
S31508013558A0EB0A00824013430134049314F8011BB3
S31508013568062225488DF8281000F082FC002836D056
S31508013578224B1BBB039B073323F00703083303932B
S31508013588099B334409936AE70C4601200CFB02326E
S31508013598A8E700234FF00A0C19460134059320467B
S315080135A810F8012B303A092A03D9002BC6D0059100
S315080135B8C4E7044601230CFB0121F0E703AB00939A
S315080135C82A4638460E4B04A9AFF30080421C064624
S315080135D8D6D1AB895B063FF52DAF09982CE703AB26
S315080135E800932A463846064B04A900F0BDF9EDE7CB
S315080135F8984401089E440108A244010800000000F5
S315080136085D330108936810B4013B002B936007DA10
S315080136189469A34201DB0A2902D110BC00F06ABBEE
S315080136281368581C10601970084610BC7047F8B51D
S3150801363806460F461446D518AC4201D1002007E0C4
S315080136483A46304614F8011BFFF7DCFF431CF3D151
S31508013658F8BD00002DE9F04F0D4614469846064672
S315080136689DB018B1036A0BB9FFF72CFC6B6ED90725
S3150801367805D4AB899A0502D4A86DFFF764FDAB8911
S315080136881B0701D52B699BB92946304600F070FB03
S3150801369870B16B6EDC0704D54FF0FF301DB0BDE87D
S315080136A8F08FAB899805F7D4A86DFFF74DFDF3E7B9
S315080136B80023099320238DF8293030234FF0010977
S315080136C8CDF80C80DFF8A8818DF82A3023469A466A
S315080136D813F8012B0AB1252AF9D1BAEB040B0BD039
S315080136E85B46224629463046FFF7A1FF013000F01E
S315080136F8A780099A5A4409929AF80030002B00F0D3
S315080137089F8000234FF0FF32CDE905230AF1010A0C
S31508013718049307938DF853301A935446052214F8DF
S31508013728011B534800F0A4FB049AD8B9D10644BF33
S3150801373820238DF85330130744BF2B238DF85330B4
S315080137489AF800302A2B15D0544600204FF00A0C57
S31508013758079A214611F8013B303B092B4BD9B0B1E1
S31508013768079214E0A0EB080309FA03F31343A246E8
S315080137780493D2E7039B191D1B680391002BBBBF52
S315080137885B4242F0020207930793B8BF0492237873
S315080137982E2B0AD163782A2B32D1039B02341A1DA0
S315080137A81B68039243EAE3730593DFF8C8A003226B
S315080137B85046217800F05CFB38B14022049BA0EB07
S315080137C80A00824013430134049314F8011B0622A4
S315080137D829488DF8281000F04BFB00283FD0274BC5
S315080137E81BBB039B073323F0070308330393099B82
S315080137F83B4409936AE70C4601200CFB0232A8E709
S3150801380800234FF00A0C194601340593204610F88F
S31508013818012B303A092A03D9002BC6D00591C4E7EA
S31508013828044601230CFB0121F0E703AB00932A4662
S315080138383046134B04A9AFF300800746781CD6D146
S315080138486B6ED90705D4AB899A0502D4A86DFFF71B
S315080138587BFCAB895B063FF51FAF09981EE703ABEF
S3150801386800932A463046064B04A900F07DF8E4E79A
S31508013878984401089E440108A24401080000000072
S31508013888373601082DE9F047164698468A680B69BE
S3150801389807469342B8BF1346336091F843200C464E
S315080138A8DDF820900AB1013333602368990642BFCF
S315080138B8336802333360256815F0060506D104F125
S315080138C8190AE36832689B1AAB422BDC94F8433031
S315080138D82268003B18BF0123920630D44146384670
S315080138E804F14302C847013023D02368226903F04B
S315080138F80603042B14BF002533684FF0000608BFDA
S31508013908E56804F11A0408BFED1A54F8123C08BF11
S3150801391825EAE5759342C4BF9B1AED18B5421AD133
S31508013928002008E00123524641463846C847013077
S3150801393803D14FF0FF30BDE8F0870135C1E73020E4
S31508013948E11881F843005A1C94F8451022440233B9
S3150801395882F84310C2E70123224641463846C8473A
S315080139680130E6D00136D9E72DE9FF470F7E9146A2
S31508013978782F80460C469A460C9E01F1430207D8D1
S31508013988622F0AD8002F00F0D180582F00F0B8808E
S3150801399804F1420684F842703AE0A7F16303152B4D
S315080139A8F6D801A151F823F0093A01081D3A010888
S315080139B89939010899390108993901089939010884
S315080139C81D3A0108993901089939010899390108EF
S315080139D8993901081B3B0108473A0108D53A0108F4
S315080139E899390108993901083D3B010899390108AE
S315080139F8473A01089939010899390108DD3A010850
S31508013A0833681A1D1B68326004F1420684F842308D
S31508013A1801239CE033682068191D3160060601D523
S31508013A281D6803E04506FBD5B3F90050002D03DAF6
S31508013A382D236D4284F843300A23584811E021683A
S31508013A483368080653F8045B02D4490648BFADB281
S31508013A586F2F336014BF0A2308235048002184F8BE
S31508013A6843106668002EA66005DB21682E4321F0FF
S31508013A78040121604BD01646B5FBF3F103FB115738
S31508013A88C75D06F8017D2F46BB420D46F4D9082BBA
S31508013A980BD12368DF0708D5236961689942DEBF18
S31508013AA8302306F8013C06F1FF36921B22614B4684
S31508013AB821464046CDF800A003AAFFF7E3FE0130E8
S31508013AC84AD14FF0FF3004B0BDE8F087236843F0C8
S31508013AD8200323607827324884F8457023683168BB
S31508013AE81F0651F8045B02D45F0648BFADB23160C0
S31508013AF8D90744BF43F0200323601DB11023ADE75E
S31508013B082648E9E7236823F020032360F6E71646E3
S31508013B18BDE733682568181D616930602E061B687C
S31508013B2801D5196002E06806FBD5198000231646F7
S31508013B382361BCE7336800211A1D32601E68626872
S31508013B48304600F095F908B1801B60606368236107
S31508013B58002384F84330AAE7324649464046236992
S31508013B68D0470130ADD023689B0713D4E068039B7F
S31508013B789842B8BF1846A6E7012332464946404641
S31508013B88D04701309DD00135E36803995B1AAB42EA
S31508013B98F2DCEBE7002504F11906F5E7A944010863
S31508013BA8BA440108B1F90C20F8B5160705460C46BA
S31508013BB854D44B68002B02DC0B6C002B48DDE66AF3
S31508013BC8002E45D0002312F480522F68216A2B60F3
S31508013BD830D0626DA389590705D56368D21A636B14
S31508013BE80BB1236CD21A00232846E66A216AB04724
S31508013BF8431CA38906D129681D292BD8284ACA40F6
S31508013C08D60727D5002262602269D904226004D51D
S31508013C18421C01D12B6803B96065616B2F60B9B184
S31508013C2804F14403994202D02846FFF79DFA002376
S31508013C3863630DE001232846B0470246501CC9D1E3
S31508013C482B68002BC6D01D2B01D0162B1DD12F6032
S31508013C58002021E043F040031BB21AE00F69002F48
S31508013C68F6D0930718BF00230E6808BF4B69F61BE1
S31508013C780F608B60002EEBDD33463A462846216AEB
S31508013C88D4F828C0E047002807DCB4F90C3043F01B
S31508013C9840034FF0FF30A381F8BD0744361AE9E718
S31508013CA80100402038B50B6905460C4613B90025AD
S31508013CB8284638BD18B1036A0BB9FFF703F9B4F9F1
S31508013CC80C30002BF3D0626ED00704D4990502D4C0
S31508013CD8A06DFFF738FA28462146FFF763FF636E9A
S31508013CE80546DA07E4D4A3899B05E1D4A06DFFF755
S31508013CF82BFADDE7F8B50E461446054618B1036AE8
S31508013D080BB9FFF7DFF8A369A360A3891A0701D5D9
S31508013D18236943B92146284600F02AF818B14FF015
S31508013D28FF373846F8BD23682269F6B2981A6369D7
S31508013D383746834205DC21462846FFF7B3FF0028A4
S31508013D48EDD1A368013BA36023685A1C22601E7043
S31508013D586269431C9A4204D0A389DB07E1D50A2E76
S31508013D68DFD121462846FFF79DFF0028D9D0D6E797
S31508013D7838B5294B054618680C4618B1036A0BB9B4
S31508013D88FFF7A0F8B4F90C30190722D4DA0607D4D4
S31508013D9809222A6043F040034FF0FF30A38133E03C
S31508013DA8580712D5616B41B104F14403994202D00F
S31508013DB82846FFF7D9F900236363A38923F0240367
S31508013DC8A3810023636023692360A38943F0080359
S31508013DD8A38123694BB9A38903F42073B3F5007F3B
S31508013DE803D02146284600F0A4F8B4F90C3013F09C
S31508013DF801020AD00022A26062695242A2612269BE
S31508013E0842B913F08000C5D138BD990758BF626910
S31508013E18A260F4E70020F7E784000020884210B57D
S31508013E2801EB020402D98442234607D8431EA1425C
S31508013E3808D011F8012B03F8012FF8E701460244C7
S31508013E488A4200D110BD13F8014D02F8014DF7E772
S31508013E5838B50023054D044608462B60F9F73AF9A3
S31508013E68431C02D12B6803B1236038BDB811002061
S31508013E78034610B5C9B202449342184601D1002037
S31508013E8803E0047801338C42F6D110BD2DE9F041DF
S31508013E98074614460D4621B91146BDE8F041FFF714
S31508013EA8CDB92AB9FFF760F925462846BDE8F08154
S31508013EB800F09EF88442064602D8B4EB500FF4D8AF
S31508013EC821463846FFF7BAF9804608B94546ECE768
S31508013ED8B4422246294628BF3246FFF736F929460B
S31508013EE83846FFF741F9F1E770B50C46B1F90E10F6
S31508013EF8154600291E4696B00CDAA389002113F047
S31508013F08800F14BF40234FF48063002031602B6073
S31508013F1816B070BD6A4600F049F80028EDDB01992C
S31508013F2801F47041A1F50053594259414FF4806390
S31508013F38EBE78B89F7B59D0706460C4607D504F1C5
S31508013F484703236023610123636103B0F0BD6A4611
S31508013F5801ABFFF7C9FF009F054639463046FFF70B
S31508013F686DF948B9B4F90C309A05EED423F0030370
S31508013F7843F00203A381E2E7A389C4E9040743F0EE
S31508013F888003A381019B20605BB13046B4F90E100A
S31508013F9800F01EF828B1A38923F0030343F00103AF
S31508013FA8A381A3891D43A581CFE7000038B500235E
S31508013FB8064D0446084611462B60F9F765F8431C71
S31508013FC802D12B6803B1236038BD00BFB8110020A0
S31508013FD838B50023054D044608462B60F9F763F8FA
S31508013FE8431C02D12B6803B1236038BDB8110020E0
S31508013FF851F8043C181F002BBCBF0B58C018704752
S31508014008F8B500BFF8BC08BC9E467047F8B500BFAE
S30D08014018F8BC08BC9E4670477E
S31508014020434F4E4E2564204572726F723A202564BD
S315080140300A000000436F6E6E6563746F723A20550D
S315080140406E6B6E6F776E0A00436F6E6E6563746F83
S31508014050723A20556E706C75676765640A000000D0
S31508014060436F6E6E6563746F723A20446973616259
S315080140706C65640A00000000436F6E6E6563746FB9
S31508014080723A20507265706172696E670A000000A3
S31508014090436F6E6E6563746F723A20417574685228
S315080140A0657175697265640A00000000436F6E6E7A
S315080140B06563746F723A2057616974696E67466FF2
S315080140C072456E657267790A00000000436F6E6E6D
S315080140D06563746F723A204368617267696E6750E7
S315080140E0617573656445560A00000000436F6E6E7C
S315080140F06563746F723A204368617267696E6750C7
S315080141006175736564455653450A0000436F6E6EC3
S315080141106563746F723A204368617267696E670AEC
S3150801412000000000436F6E6E6563746F723A20413A
S3150801413075746854696D656F75740A00436F6E6EA0
S315080141406563746F723A2046696E69736865640AB5
S3150801415000000000436F6E6E6563746F723A204605
S31508014160696E6973686564455653450A000000001F
S31508014170436F6E6E6563746F723A2046696E697332
S3150801418068656445560A0000436F6E6E6563746F11
S31508014190723A205265706C756767696E670A000026
S315080141A0434F4E4E2564204368617267696E6720E6
S315080141B046696E69736865643A0A00004368617204
S315080141C067696E6720456E657267793A2025640AC4
S315080141D000000000434353206D6F64756C652073BE
S315080141E0746172740A00000053657269616C206E0D
S315080141F0756D6265723A2025640A0000426F617224
S3150801420064207265766973696F6E3A2025640A00BF
S3150801421046572076657273696F6E3A2025642E2596
S31508014220642E25640A000000505355206F6E2074D1
S31508014230696D656F75740A00436F6E746163746F97
S3150801424072206572726F722C2073746F7070696E4A
S31508014250672E2E2E0A000000505355206F666620E1
S3150801426074696D656F75740A000000004553544FF3
S3150801427050207472696767657265640A00000000F8
S3150801428053746F7070696E67206368617267696ECF
S31508014290672E2E2E0A00000046696E6973686564EA
S315080142A045562C2073746F7070696E672E2E2E0A10
S315080142B0000000004368617267696E672065727263
S315080142C06F722025642C207374617465202D3E203D
S315080142D064697361626C65640A000000436861720F
S315080142E067696E67207065726D69747465642C20E0
S315080142F07374617274206368617267696E670A0014
S3150801430043617220756E706C75676765640A000093
S315080143105265706C756767696E672E2E2E0A0000E6
S315080143205265706C756767696E672066696E697331
S315080143306865642C206275742063617220756E70DD
S315080143406C75676765640A005265706C756767699D
S315080143506E672066696E69736865642C206361728D
S3150801436020706C75676765642C20737461746520A9
S315080143702D3E206175746820726571756972656470
S315080143800A000000457665726573742074696D6567
S315080143906F75740A0000000043435320696E6974FF
S315080143A00A00000045766572657374207265736547
S315080143B07420636F6D6D616E640A00005061636BF2
S315080143C0657420435243206572726F720A000000B9
S315080143D0556E6B6E6F776E20636D6420307825306D
S315080143E032780A005061636B6574206C656E206DC6
S315080143F069736D6174636820636D643D3078253037
S3150801440032780A0053657420436F6E6669673A20ED
S3150801441025732025640A0000506F776572206C6940
S315080144206D69743A2025640A0000000043686172C8
S315080144306765207065726D69743A2025640A000003
S315080144400000000000000000010203040607080935
S31508014450000000000102030400000405060708091C
S3150801446000000000000D000001020304050607080C
S31508014470090A0B0C0D0E0F100000040506070809A2
S3150801448000000000000D00000102030405060708EC
S31508014490090A0B0C0D0E0F10232D302B2000686C0A
S315080144A04C00656667454647003031323334353648
S315080144B03738394142434445460030313233343581
S311080144C0363738396162636465660000AE
S30D080144CCBC4BFF7F0100000053
S309080144D40D8200083E
S309080144D8E98100085F
S315080144DCE401000006060600400000320A320040DC
S315080144EC00000000008000320A3200008000000043
S315080144FC0000FA320A32000000FA000000FF00320E
S3150801450C0A32000020000000FFFFFF320A3200FFCA
S3150801451CFFFF0000FF0000320A320020000064068B
S3150801452C0100000000FFFF00000000000000000071
S3150801453C52555301000000FE529E66000024F400F9
S3150801454C100000000100000000000000030000003C
S3150801455C7C10002088000020000000007C10002040
S3150801456CE41000204C11002000000000000000009F
S3150801457C0000000000000000000000000000000020
S3150801458C0000000000000000000000000000000010
S3150801459C0000000000000000000000000000000000
S309080145AC00000000FC
S7050800D87D9D
